Component: ARM Compiler 5.06 update 7 (build 960) Tool: armlink [4d3601]

==============================================================================

Section Cross References

    stm32f4xx_it.o(i.DMA1_Stream3_IRQHandler) refers to md_connect.o(i.MD_Connect_DMATX4_IRQHandler) for MD_Connect_DMATX4_IRQHandler
    stm32f4xx_it.o(i.DMA1_Stream4_IRQHandler) refers to md_connect.o(i.MD_Connect_DMATX2_IRQHandler) for MD_Connect_DMATX2_IRQHandler
    stm32f4xx_it.o(i.DMA1_Stream6_IRQHandler) refers to md_connect.o(i.MD_Connect_DMATX1_IRQHandler) for MD_Connect_DMATX1_IRQHandler
    stm32f4xx_it.o(i.DMA1_Stream7_IRQHandler) refers to md_connect.o(i.MD_Connect_DMATX3_IRQHandler) for MD_Connect_DMATX3_IRQHandler
    stm32f4xx_it.o(i.DMA2_Stream6_IRQHandler) refers to multiplex_port.o(i.Multiplex_Port_DMATX_IRQHandler) for Multiplex_Port_DMATX_IRQHandler
    stm32f4xx_it.o(i.DMA2_Stream7_IRQHandler) refers to pos_connect.o(i.POS_Connect_DMATX_IRQHandler) for POS_Connect_DMATX_IRQHandler
    stm32f4xx_it.o(i.EXTI0_IRQHandler) refers to pluse_input.o(i.Pluse_InPut_IRQHandler) for Pluse_InPut_IRQHandler
    stm32f4xx_it.o(i.EXTI15_10_IRQHandler) refers to pluse_input.o(i.Pluse_InPut_IRQHandler) for Pluse_InPut_IRQHandler
    stm32f4xx_it.o(i.EXTI1_IRQHandler) refers to pluse_input.o(i.Pluse_InPut_IRQHandler) for Pluse_InPut_IRQHandler
    stm32f4xx_it.o(i.TIM2_IRQHandler) refers to time_count.o(i.SYSTimer_IRQHandler) for SYSTimer_IRQHandler
    stm32f4xx_it.o(i.UART4_IRQHandler) refers to md_connect.o(i.MD_Connect_DMARX2_IRQHandler) for MD_Connect_DMARX2_IRQHandler
    stm32f4xx_it.o(i.UART5_IRQHandler) refers to md_connect.o(i.MD_Connect_DMARX3_IRQHandler) for MD_Connect_DMARX3_IRQHandler
    stm32f4xx_it.o(i.USART1_IRQHandler) refers to pos_connect.o(i.POS_Connect_DMARX_IRQHandler) for POS_Connect_DMARX_IRQHandler
    stm32f4xx_it.o(i.USART2_IRQHandler) refers to md_connect.o(i.MD_Connect_DMARX1_IRQHandler) for MD_Connect_DMARX1_IRQHandler
    stm32f4xx_it.o(i.USART3_IRQHandler) refers to md_connect.o(i.MD_Connect_DMARX4_IRQHandler) for MD_Connect_DMARX4_IRQHandler
    stm32f4xx_it.o(i.USART6_IRQHandler) refers to multiplex_port.o(i.Multiplex_Port_DMARX_IRQHandler) for Multiplex_Port_DMARX_IRQHandler
    main.o(i.main) refers to misc.o(i.NVIC_SetVectorTable) for NVIC_SetVectorTable
    main.o(i.main) refers to stm32f4xx_tim.o(i.TIM_DeInit) for TIM_DeInit
    main.o(i.main) refers to stm32f4xx_usart.o(i.USART_DeInit) for USART_DeInit
    main.o(i.main) refers to stm32f4xx_dma.o(i.DMA_DeInit) for DMA_DeInit
    main.o(i.main) refers to stm32f4xx_gpio.o(i.GPIO_DeInit) for GPIO_DeInit
    main.o(i.main) refers to stm32f4xx_iwdg.o(i.IWDG_ReloadCounter) for IWDG_ReloadCounter
    main.o(i.main) refers to delay.o(i.delay_init) for delay_init
    main.o(i.main) refers to txh.o(i.TXH_Init) for TXH_Init
    main.o(i.main) refers to txh.o(i.TXH_Task) for TXH_Task
    txh.o(i.TXH_Init) refers to pluse_input.o(i.Pluse_InPut_Init) for Pluse_InPut_Init
    txh.o(i.TXH_Init) refers to time_count.o(i.Timer_Init) for Timer_Init
    txh.o(i.TXH_Init) refers to fram.o(i.FM_Init) for FM_Init
    txh.o(i.TXH_Init) refers to fram.o(i.FMItemWrite) for FMItemWrite
    txh.o(i.TXH_Init) refers to at45db.o(i.AT45DB_Init) for AT45DB_Init
    txh.o(i.TXH_Init) refers to ds1307.o(i.DS1307_Init) for DS1307_Init
    txh.o(i.TXH_Init) refers to log.o(i.Log_Init) for Log_Init
    txh.o(i.TXH_Init) refers to oled.o(i.OLED_Init) for OLED_Init
    txh.o(i.TXH_Init) refers to surface.o(i.Surface_Init) for Surface_Init
    txh.o(i.TXH_Init) refers to log.o(i.FindSysconfigFile) for FindSysconfigFile
    txh.o(i.TXH_Init) refers to md_connect.o(i.MD_Connect_Init) for MD_Connect_Init
    txh.o(i.TXH_Init) refers to multiplex_port.o(i.Multiplex_Port_Init) for Multiplex_Port_Init
    txh.o(i.TXH_Init) refers to pos_connect.o(i.POS_Connect_Init) for POS_Connect_Init
    txh.o(i.TXH_Init) refers to pluse_putout.o(i.Pluse_Putout_Init) for Pluse_Putout_Init
    txh.o(i.TXH_Init) refers to fram.o(i.PCBEncryption_Check) for PCBEncryption_Check
    txh.o(i.TXH_Init) refers to txh.o(.bss) for TXHData
    txh.o(i.TXH_Task) refers to ds1307.o(i.DS1307_Read) for DS1307_Read
    txh.o(i.TXH_Task) refers to md_connect.o(i.MD_ConnectTXTask) for MD_ConnectTXTask
    txh.o(i.TXH_Task) refers to txh.o(.bss) for TXHData
    txh.o(i.TXH_Task) refers to multiplex_port.o(i.Multiplex_PortTXTask) for Multiplex_PortTXTask
    txh.o(i.TXH_Task) refers to pos_connect.o(i.POS_ConnectTXTask) for POS_ConnectTXTask
    txh.o(i.TXH_Task) refers to md_connect.o(i.MD_ConnectRXTask) for MD_ConnectRXTask
    txh.o(i.TXH_Task) refers to multiplex_port.o(i.Multiplex_PortRXTask) for Multiplex_PortRXTask
    txh.o(i.TXH_Task) refers to pos_connect.o(i.POS_ConnectRXTask) for POS_ConnectRXTask
    txh.o(i.TXH_Task) refers to surface.o(i.SurfaceTast) for SurfaceTast
    system_stm32f4xx.o(i.SystemCoreClockUpdate) refers to system_stm32f4xx.o(.data) for SystemCoreClock
    system_stm32f4xx.o(i.SystemInit) refers to system_stm32f4xx.o(i.SetSysClock) for SetSysClock
    startup_stm32f4xx.o(RESET) refers to startup_stm32f4xx.o(STACK) for __initial_sp
    startup_stm32f4xx.o(RESET) refers to startup_stm32f4xx.o(.text) for Reset_Handler
    startup_stm32f4xx.o(RESET) refers to stm32f4xx_it.o(i.HardFault_Handler) for HardFault_Handler
    startup_stm32f4xx.o(RESET) refers to stm32f4xx_it.o(i.EXTI0_IRQHandler) for EXTI0_IRQHandler
    startup_stm32f4xx.o(RESET) refers to stm32f4xx_it.o(i.EXTI1_IRQHandler) for EXTI1_IRQHandler
    startup_stm32f4xx.o(RESET) refers to stm32f4xx_it.o(i.DMA1_Stream3_IRQHandler) for DMA1_Stream3_IRQHandler
    startup_stm32f4xx.o(RESET) refers to stm32f4xx_it.o(i.DMA1_Stream4_IRQHandler) for DMA1_Stream4_IRQHandler
    startup_stm32f4xx.o(RESET) refers to stm32f4xx_it.o(i.DMA1_Stream6_IRQHandler) for DMA1_Stream6_IRQHandler
    startup_stm32f4xx.o(RESET) refers to stm32f4xx_it.o(i.TIM2_IRQHandler) for TIM2_IRQHandler
    startup_stm32f4xx.o(RESET) refers to stm32f4xx_it.o(i.USART1_IRQHandler) for USART1_IRQHandler
    startup_stm32f4xx.o(RESET) refers to stm32f4xx_it.o(i.USART2_IRQHandler) for USART2_IRQHandler
    startup_stm32f4xx.o(RESET) refers to stm32f4xx_it.o(i.USART3_IRQHandler) for USART3_IRQHandler
    startup_stm32f4xx.o(RESET) refers to stm32f4xx_it.o(i.EXTI15_10_IRQHandler) for EXTI15_10_IRQHandler
    startup_stm32f4xx.o(RESET) refers to stm32f4xx_it.o(i.DMA1_Stream7_IRQHandler) for DMA1_Stream7_IRQHandler
    startup_stm32f4xx.o(RESET) refers to stm32f4xx_it.o(i.UART4_IRQHandler) for UART4_IRQHandler
    startup_stm32f4xx.o(RESET) refers to stm32f4xx_it.o(i.UART5_IRQHandler) for UART5_IRQHandler
    startup_stm32f4xx.o(RESET) refers to stm32f4xx_it.o(i.DMA2_Stream6_IRQHandler) for DMA2_Stream6_IRQHandler
    startup_stm32f4xx.o(RESET) refers to stm32f4xx_it.o(i.DMA2_Stream7_IRQHandler) for DMA2_Stream7_IRQHandler
    startup_stm32f4xx.o(RESET) refers to stm32f4xx_it.o(i.USART6_IRQHandler) for USART6_IRQHandler
    startup_stm32f4xx.o(.text) refers to system_stm32f4xx.o(i.SystemInit) for SystemInit
    startup_stm32f4xx.o(.text) refers to entry.o(.ARM.Collect$$$$00000000) for __main
    stm32f4xx_adc.o(i.ADC_DeInit) refers to stm32f4xx_rcc.o(i.RCC_APB2PeriphResetCmd) for RCC_APB2PeriphResetCmd
    stm32f4xx_flash.o(i.FLASH_EraseAllSectors) refers to stm32f4xx_flash.o(i.FLASH_WaitForLastOperation) for FLASH_WaitForLastOperation
    stm32f4xx_flash.o(i.FLASH_EraseSector) refers to stm32f4xx_flash.o(i.FLASH_WaitForLastOperation) for FLASH_WaitForLastOperation
    stm32f4xx_flash.o(i.FLASH_OB_Launch) refers to stm32f4xx_flash.o(i.FLASH_WaitForLastOperation) for FLASH_WaitForLastOperation
    stm32f4xx_flash.o(i.FLASH_OB_RDPConfig) refers to stm32f4xx_flash.o(i.FLASH_WaitForLastOperation) for FLASH_WaitForLastOperation
    stm32f4xx_flash.o(i.FLASH_OB_UserConfig) refers to stm32f4xx_flash.o(i.FLASH_WaitForLastOperation) for FLASH_WaitForLastOperation
    stm32f4xx_flash.o(i.FLASH_OB_WRPConfig) refers to stm32f4xx_flash.o(i.FLASH_WaitForLastOperation) for FLASH_WaitForLastOperation
    stm32f4xx_flash.o(i.FLASH_ProgramByte) refers to stm32f4xx_flash.o(i.FLASH_WaitForLastOperation) for FLASH_WaitForLastOperation
    stm32f4xx_flash.o(i.FLASH_ProgramDoubleWord) refers to stm32f4xx_flash.o(i.FLASH_WaitForLastOperation) for FLASH_WaitForLastOperation
    stm32f4xx_flash.o(i.FLASH_ProgramHalfWord) refers to stm32f4xx_flash.o(i.FLASH_WaitForLastOperation) for FLASH_WaitForLastOperation
    stm32f4xx_flash.o(i.FLASH_ProgramWord) refers to stm32f4xx_flash.o(i.FLASH_WaitForLastOperation) for FLASH_WaitForLastOperation
    stm32f4xx_flash.o(i.FLASH_WaitForLastOperation) refers to stm32f4xx_flash.o(i.FLASH_GetStatus) for FLASH_GetStatus
    stm32f4xx_gpio.o(i.GPIO_DeInit) refers to stm32f4xx_rcc.o(i.RCC_AHB1PeriphResetCmd) for RCC_AHB1PeriphResetCmd
    stm32f4xx_rcc.o(i.RCC_GetClocksFreq) refers to stm32f4xx_rcc.o(.data) for APBAHBPrescTable
    stm32f4xx_rcc.o(i.RCC_WaitForHSEStartUp) refers to stm32f4xx_rcc.o(i.RCC_GetFlagStatus) for RCC_GetFlagStatus
    stm32f4xx_spi.o(i.SPI_I2S_DeInit) refers to stm32f4xx_rcc.o(i.RCC_APB2PeriphResetCmd) for RCC_APB2PeriphResetCmd
    stm32f4xx_spi.o(i.SPI_I2S_DeInit) refers to stm32f4xx_rcc.o(i.RCC_APB1PeriphResetCmd) for RCC_APB1PeriphResetCmd
    stm32f4xx_syscfg.o(i.SYSCFG_DeInit) refers to stm32f4xx_rcc.o(i.RCC_APB2PeriphResetCmd) for RCC_APB2PeriphResetCmd
    stm32f4xx_tim.o(i.TIM_DeInit) refers to stm32f4xx_rcc.o(i.RCC_APB2PeriphResetCmd) for RCC_APB2PeriphResetCmd
    stm32f4xx_tim.o(i.TIM_DeInit) refers to stm32f4xx_rcc.o(i.RCC_APB1PeriphResetCmd) for RCC_APB1PeriphResetCmd
    stm32f4xx_tim.o(i.TIM_ETRClockMode1Config) refers to stm32f4xx_tim.o(i.TIM_ETRConfig) for TIM_ETRConfig
    stm32f4xx_tim.o(i.TIM_ETRClockMode2Config) refers to stm32f4xx_tim.o(i.TIM_ETRConfig) for TIM_ETRConfig
    stm32f4xx_tim.o(i.TIM_ICInit) refers to stm32f4xx_tim.o(i.TI1_Config) for TI1_Config
    stm32f4xx_tim.o(i.TIM_ICInit) refers to stm32f4xx_tim.o(i.TIM_SetIC1Prescaler) for TIM_SetIC1Prescaler
    stm32f4xx_tim.o(i.TIM_ICInit) refers to stm32f4xx_tim.o(i.TI2_Config) for TI2_Config
    stm32f4xx_tim.o(i.TIM_ICInit) refers to stm32f4xx_tim.o(i.TIM_SetIC2Prescaler) for TIM_SetIC2Prescaler
    stm32f4xx_tim.o(i.TIM_ICInit) refers to stm32f4xx_tim.o(i.TI3_Config) for TI3_Config
    stm32f4xx_tim.o(i.TIM_ICInit) refers to stm32f4xx_tim.o(i.TIM_SetIC3Prescaler) for TIM_SetIC3Prescaler
    stm32f4xx_tim.o(i.TIM_ICInit) refers to stm32f4xx_tim.o(i.TI4_Config) for TI4_Config
    stm32f4xx_tim.o(i.TIM_ICInit) refers to stm32f4xx_tim.o(i.TIM_SetIC4Prescaler) for TIM_SetIC4Prescaler
    stm32f4xx_tim.o(i.TIM_ITRxExternalClockConfig) refers to stm32f4xx_tim.o(i.TIM_SelectInputTrigger) for TIM_SelectInputTrigger
    stm32f4xx_tim.o(i.TIM_PWMIConfig) refers to stm32f4xx_tim.o(i.TI1_Config) for TI1_Config
    stm32f4xx_tim.o(i.TIM_PWMIConfig) refers to stm32f4xx_tim.o(i.TIM_SetIC1Prescaler) for TIM_SetIC1Prescaler
    stm32f4xx_tim.o(i.TIM_PWMIConfig) refers to stm32f4xx_tim.o(i.TI2_Config) for TI2_Config
    stm32f4xx_tim.o(i.TIM_PWMIConfig) refers to stm32f4xx_tim.o(i.TIM_SetIC2Prescaler) for TIM_SetIC2Prescaler
    stm32f4xx_tim.o(i.TIM_TIxExternalClockConfig) refers to stm32f4xx_tim.o(i.TI2_Config) for TI2_Config
    stm32f4xx_tim.o(i.TIM_TIxExternalClockConfig) refers to stm32f4xx_tim.o(i.TI1_Config) for TI1_Config
    stm32f4xx_tim.o(i.TIM_TIxExternalClockConfig) refers to stm32f4xx_tim.o(i.TIM_SelectInputTrigger) for TIM_SelectInputTrigger
    stm32f4xx_usart.o(i.USART_DeInit) refers to stm32f4xx_rcc.o(i.RCC_APB2PeriphResetCmd) for RCC_APB2PeriphResetCmd
    stm32f4xx_usart.o(i.USART_DeInit) refers to stm32f4xx_rcc.o(i.RCC_APB1PeriphResetCmd) for RCC_APB1PeriphResetCmd
    stm32f4xx_usart.o(i.USART_Init) refers to stm32f4xx_rcc.o(i.RCC_GetClocksFreq) for RCC_GetClocksFreq
    stm32f4xx_rng.o(i.RNG_DeInit) refers to stm32f4xx_rcc.o(i.RCC_AHB2PeriphResetCmd) for RCC_AHB2PeriphResetCmd
    stm32f4xx_wwdg.o(i.WWDG_DeInit) refers to stm32f4xx_rcc.o(i.RCC_APB1PeriphResetCmd) for RCC_APB1PeriphResetCmd
    time_count.o(i.SYSTimer_IRQHandler) refers to stm32f4xx_tim.o(i.TIM_GetITStatus) for TIM_GetITStatus
    time_count.o(i.SYSTimer_IRQHandler) refers to stm32f4xx_tim.o(i.TIM_ClearFlag) for TIM_ClearFlag
    time_count.o(i.SYSTimer_IRQHandler) refers to txh.o(.bss) for TXHData
    time_count.o(i.Timer_Init) refers to stm32f4xx_rcc.o(i.RCC_APB1PeriphClockCmd) for RCC_APB1PeriphClockCmd
    time_count.o(i.Timer_Init) refers to stm32f4xx_tim.o(i.TIM_TimeBaseInit) for TIM_TimeBaseInit
    time_count.o(i.Timer_Init) refers to stm32f4xx_tim.o(i.TIM_Cmd) for TIM_Cmd
    time_count.o(i.Timer_Init) refers to stm32f4xx_tim.o(i.TIM_ITConfig) for TIM_ITConfig
    time_count.o(i.Timer_Init) refers to time_count.o(i.Timer_NVIC_Configuration) for Timer_NVIC_Configuration
    time_count.o(i.Timer_Init) refers to txh.o(.bss) for TXHData
    time_count.o(i.Timer_NVIC_Configuration) refers to misc.o(i.NVIC_Init) for NVIC_Init
    fram.o(i.FMItemRead) refers to fram.o(i.FM_ReadData) for FM_ReadData
    fram.o(i.FMItemRead) refers to fram.o(i.FRamDataCheck) for FRamDataCheck
    fram.o(i.FMItemRead) refers to delay.o(i.delay_ms) for delay_ms
    fram.o(i.FMItemRead) refers to fram.o(.constdata) for FDITab
    fram.o(i.FMItemRead) refers to fram.o(.bss) for s_uniGlobal
    fram.o(i.FMItemWrite) refers to fram.o(i.FMItemRead) for FMItemRead
    fram.o(i.FMItemWrite) refers to fram.o(i.FM_WriteData) for FM_WriteData
    fram.o(i.FMItemWrite) refers to fram.o(i.FRamDataCheck) for FRamDataCheck
    fram.o(i.FMItemWrite) refers to delay.o(i.delay_ms) for delay_ms
    fram.o(i.FMItemWrite) refers to fram.o(.constdata) for FDITab
    fram.o(i.FMItemWrite) refers to txh.o(.bss) for TXHData
    fram.o(i.FMItemWrite) refers to fram.o(.bss) for s_uniGlobal
    fram.o(i.FM_Data_Init) refers to fram.o(i.FMItemRead) for FMItemRead
    fram.o(i.FM_Data_Init) refers to fram.o(i.FRamDataCheck) for FRamDataCheck
    fram.o(i.FM_Data_Init) refers to fram.o(i.FM_WriteData) for FM_WriteData
    fram.o(i.FM_Data_Init) refers to fram.o(i.FMItemWrite) for FMItemWrite
    fram.o(i.FM_Data_Init) refers to txh.o(.bss) for TXHData
    fram.o(i.FM_Data_Init) refers to fram.o(.data) for iiii
    fram.o(i.FM_Data_Init) refers to fram.o(.constdata) for FDITab
    fram.o(i.FM_Data_Init) refers to fram.o(.bss) for s_uniGlobal
    fram.o(i.FM_IO_Configuration) refers to stm32f4xx_rcc.o(i.RCC_AHB1PeriphClockCmd) for RCC_AHB1PeriphClockCmd
    fram.o(i.FM_IO_Configuration) refers to stm32f4xx_gpio.o(i.GPIO_Init) for GPIO_Init
    fram.o(i.FM_IO_Configuration) refers to stm32f4xx_gpio.o(i.GPIO_PinAFConfig) for GPIO_PinAFConfig
    fram.o(i.FM_Init) refers to fram.o(i.FM_IO_Configuration) for FM_IO_Configuration
    fram.o(i.FM_Init) refers to fram.o(i.FM_SPI_Configuration) for FM_SPI_Configuration
    fram.o(i.FM_Init) refers to delay.o(i.delay_ms) for delay_ms
    fram.o(i.FM_Init) refers to stm32f4xx_gpio.o(i.GPIO_ResetBits) for GPIO_ResetBits
    fram.o(i.FM_Init) refers to stm32f4xx_gpio.o(i.GPIO_SetBits) for GPIO_SetBits
    fram.o(i.FM_Init) refers to fram.o(i.FM_SPI1_SendByte) for FM_SPI1_SendByte
    fram.o(i.FM_Init) refers to fram.o(i.FM_Data_Init) for FM_Data_Init
    fram.o(i.FM_Init) refers to fram.o(i.FMItemRead) for FMItemRead
    fram.o(i.FM_Init) refers to fram.o(.constdata) for FDITab
    fram.o(i.FM_Init) refers to fram.o(.data) for iiii
    fram.o(i.FM_Init) refers to txh.o(.bss) for TXHData
    fram.o(i.FM_ReadData) refers to fram.o(i.__set_PRIMASK) for __set_PRIMASK
    fram.o(i.FM_ReadData) refers to stm32f4xx_gpio.o(i.GPIO_ResetBits) for GPIO_ResetBits
    fram.o(i.FM_ReadData) refers to stm32f4xx_gpio.o(i.GPIO_SetBits) for GPIO_SetBits
    fram.o(i.FM_ReadData) refers to fram.o(i.FM_SPI1_SendByte) for FM_SPI1_SendByte
    fram.o(i.FM_SPI1_SendByte) refers to stm32f4xx_spi.o(i.SPI_I2S_GetFlagStatus) for SPI_I2S_GetFlagStatus
    fram.o(i.FM_SPI1_SendByte) refers to stm32f4xx_spi.o(i.SPI_I2S_SendData) for SPI_I2S_SendData
    fram.o(i.FM_SPI1_SendByte) refers to stm32f4xx_spi.o(i.SPI_I2S_ReceiveData) for SPI_I2S_ReceiveData
    fram.o(i.FM_SPI_Configuration) refers to stm32f4xx_rcc.o(i.RCC_APB2PeriphClockCmd) for RCC_APB2PeriphClockCmd
    fram.o(i.FM_SPI_Configuration) refers to stm32f4xx_spi.o(i.SPI_I2S_DeInit) for SPI_I2S_DeInit
    fram.o(i.FM_SPI_Configuration) refers to stm32f4xx_spi.o(i.SPI_Init) for SPI_Init
    fram.o(i.FM_SPI_Configuration) refers to stm32f4xx_spi.o(i.SPI_Cmd) for SPI_Cmd
    fram.o(i.FM_WriteData) refers to fram.o(i.__set_PRIMASK) for __set_PRIMASK
    fram.o(i.FM_WriteData) refers to stm32f4xx_gpio.o(i.GPIO_ResetBits) for GPIO_ResetBits
    fram.o(i.FM_WriteData) refers to stm32f4xx_gpio.o(i.GPIO_SetBits) for GPIO_SetBits
    fram.o(i.FM_WriteData) refers to fram.o(i.FM_SPI1_SendByte) for FM_SPI1_SendByte
    fram.o(i.PCBEncryption) refers to pos_connect.o(i.CRC_Check) for CRC_Check
    fram.o(i.PCBEncryption) refers to fram.o(i.FM_WriteData) for FM_WriteData
    fram.o(i.PCBEncryption) refers to txh.o(.bss) for STM32CPU
    fram.o(i.PCBEncryption_Check) refers to fram.o(i.FM_ReadData) for FM_ReadData
    fram.o(i.PCBEncryption_Check) refers to pos_connect.o(i.CRC_Check) for CRC_Check
    fram.o(i.PCBEncryption_Check) refers to txh.o(.bss) for STM32CPU
    fram.o(.constdata) refers to fram.o(.bss) for s_uniGlobal
    fram.o(.constdata) refers to txh.o(.bss) for TXHData
    pluse_input.o(i.Pluse_InPut_EXTI_Configuration) refers to stm32f4xx_rcc.o(i.RCC_APB2PeriphClockCmd) for RCC_APB2PeriphClockCmd
    pluse_input.o(i.Pluse_InPut_EXTI_Configuration) refers to stm32f4xx_syscfg.o(i.SYSCFG_EXTILineConfig) for SYSCFG_EXTILineConfig
    pluse_input.o(i.Pluse_InPut_EXTI_Configuration) refers to stm32f4xx_exti.o(i.EXTI_Init) for EXTI_Init
    pluse_input.o(i.Pluse_InPut_IO_Configuration) refers to stm32f4xx_rcc.o(i.RCC_AHB1PeriphClockCmd) for RCC_AHB1PeriphClockCmd
    pluse_input.o(i.Pluse_InPut_IO_Configuration) refers to stm32f4xx_gpio.o(i.GPIO_Init) for GPIO_Init
    pluse_input.o(i.Pluse_InPut_IO_Configuration) refers to stm32f4xx_gpio.o(i.GPIO_ResetBits) for GPIO_ResetBits
    pluse_input.o(i.Pluse_InPut_IO_Configuration) refers to stm32f4xx_gpio.o(i.GPIO_SetBits) for GPIO_SetBits
    pluse_input.o(i.Pluse_InPut_IO_Configuration) refers to txh.o(.bss) for TXHData
    pluse_input.o(i.Pluse_InPut_IRQHandler) refers to stm32f4xx_exti.o(i.EXTI_GetITStatus) for EXTI_GetITStatus
    pluse_input.o(i.Pluse_InPut_IRQHandler) refers to stm32f4xx_exti.o(i.EXTI_ClearITPendingBit) for EXTI_ClearITPendingBit
    pluse_input.o(i.Pluse_InPut_IRQHandler) refers to txh.o(.bss) for TXHData
    pluse_input.o(i.Pluse_InPut_Init) refers to pluse_input.o(i.Pluse_InPut_IO_Configuration) for Pluse_InPut_IO_Configuration
    pluse_input.o(i.Pluse_InPut_Init) refers to delay.o(i.delay_ms) for delay_ms
    pluse_input.o(i.Pluse_InPut_Init) refers to pluse_input.o(i.Pluse_InPut_EXTI_Configuration) for Pluse_InPut_EXTI_Configuration
    pluse_input.o(i.Pluse_InPut_Init) refers to pluse_input.o(i.Pluse_InPut_NVIC_Configuration) for Pluse_InPut_NVIC_Configuration
    pluse_input.o(i.Pluse_InPut_Init) refers to txh.o(.bss) for TXHData
    pluse_input.o(i.Pluse_InPut_NVIC_Configuration) refers to misc.o(i.NVIC_Init) for NVIC_Init
    md_connect.o(i.Bluesky_Decrypt) refers to md_connect.o(i.Bluesky_Encrypt) for Bluesky_Encrypt
    md_connect.o(i.MD_ConnectRXTask) refers to stm32f4xx_dma.o(i.DMA_Cmd) for DMA_Cmd
    md_connect.o(i.MD_ConnectRXTask) refers to stm32f4xx_dma.o(i.DMA_ClearFlag) for DMA_ClearFlag
    md_connect.o(i.MD_ConnectRXTask) refers to stm32f4xx_gpio.o(i.GPIO_ResetBits) for GPIO_ResetBits
    md_connect.o(i.MD_ConnectRXTask) refers to log.o(i.Log_Task) for Log_Task
    md_connect.o(i.MD_ConnectRXTask) refers to md_connect.o(i.MD_Connect_BCDTou64) for MD_Connect_BCDTou64
    md_connect.o(i.MD_ConnectRXTask) refers to txh.o(.bss) for TXHData
    md_connect.o(i.MD_ConnectRXTask) refers to md_connect.o(.data) for MD_ConnectRX1Task_Flag
    md_connect.o(i.MD_ConnectRXTask) refers to md_connect.o(.bss) for MD_Connect_RX_Buff
    md_connect.o(i.MD_ConnectRXTask) refers to md_connect.o(i.MD_Connect_TXDataCheck) for MD_Connect_TXDataCheck
    md_connect.o(i.MD_ConnectRXTask) refers to fram.o(i.FMItemWrite) for FMItemWrite
    md_connect.o(i.MD_ConnectRXTask) refers to memcpya.o(.text) for __aeabi_memcpy
    md_connect.o(i.MD_ConnectRXTask) refers to at45db.o(i.AT45DBItemWrite) for AT45DBItemWrite
    md_connect.o(i.MD_ConnectRXTask) refers to md_connect.o(i.MD_Connect_USART_Configuration) for MD_Connect_USART_Configuration
    md_connect.o(i.MD_ConnectRXTask) refers to md_connect.o(i.do_crc) for do_crc
    md_connect.o(i.MD_ConnectRXTask) refers to ldiv.o(.text) for __aeabi_ldivmod
    md_connect.o(i.MD_ConnectRXTask) refers to md_connect.o(i.CheckSum) for CheckSum
    md_connect.o(i.MD_ConnectRXTask) refers to md_connect.o(i.StrToInt) for StrToInt
    md_connect.o(i.MD_ConnectRXTask) refers to md_connect.o(i.StrToFloat) for StrToFloat
    md_connect.o(i.MD_ConnectRXTask) refers to pos_connect.o(i.CRC_Check) for CRC_Check
    md_connect.o(i.MD_ConnectRXTask) refers to f2d.o(.text) for __aeabi_f2d
    md_connect.o(i.MD_ConnectRXTask) refers to ddiv.o(.text) for __aeabi_ddiv
    md_connect.o(i.MD_ConnectRXTask) refers to dadd.o(.text) for __aeabi_drsub
    md_connect.o(i.MD_ConnectRXTask) refers to d2f.o(.text) for __aeabi_d2f
    md_connect.o(i.MD_ConnectRXTask) refers to dfltui.o(.text) for __aeabi_ui2d
    md_connect.o(i.MD_ConnectRXTask) refers to pow.o(i.__hardfp_pow) for __hardfp_pow
    md_connect.o(i.MD_ConnectRXTask) refers to md_connect.o(i.BCC_CheckSum) for BCC_CheckSum
    md_connect.o(i.MD_ConnectRXTask) refers to dflti.o(.text) for __aeabi_i2d
    md_connect.o(i.MD_ConnectRXTask) refers to dfixl.o(.text) for __aeabi_d2lz
    md_connect.o(i.MD_ConnectRXTask) refers to md_connect.o(i.MD_Connect_u64ToBCD) for MD_Connect_u64ToBCD
    md_connect.o(i.MD_ConnectRXTask) refers to md_connect.o(i.InteiHEXCheck) for InteiHEXCheck
    md_connect.o(i.MD_ConnectRXTask) refers to md_connect.o(i.Bluesky_Decrypt) for Bluesky_Decrypt
    md_connect.o(i.MD_ConnectRXTask) refers to multiplex_port.o(i.Price_DataCheck) for Price_DataCheck
    md_connect.o(i.MD_ConnectRXTask) refers to multiplex_port.o(i.mystrstr) for mystrstr
    md_connect.o(i.MD_ConnectTXTask) refers to md_connect.o(.data) for MD_Connect_TX_Flag
    md_connect.o(i.MD_ConnectTXTask) refers to txh.o(.bss) for TXHData
    md_connect.o(i.MD_ConnectTXTask) refers to md_connect.o(i.MD_Connect_u64ToBCD) for MD_Connect_u64ToBCD
    md_connect.o(i.MD_ConnectTXTask) refers to md_connect.o(i.MD_Connect_USART_Configuration) for MD_Connect_USART_Configuration
    md_connect.o(i.MD_ConnectTXTask) refers to md_connect.o(i.MD_Connect_TXDataCheck) for MD_Connect_TXDataCheck
    md_connect.o(i.MD_ConnectTXTask) refers to md_connect.o(.bss) for MD_Connect_TX_Buff
    md_connect.o(i.MD_ConnectTXTask) refers to llsshr.o(.text) for __aeabi_lasr
    md_connect.o(i.MD_ConnectTXTask) refers to at45db.o(i.AT45DBItemRead) for AT45DBItemRead
    md_connect.o(i.MD_ConnectTXTask) refers to stm32f4xx_rng.o(i.RNG_GetRandomNumber) for RNG_GetRandomNumber
    md_connect.o(i.MD_ConnectTXTask) refers to md_connect.o(i.Bluesky_Encrypt) for Bluesky_Encrypt
    md_connect.o(i.MD_ConnectTXTask) refers to pos_connect.o(i.CRC_Check) for CRC_Check
    md_connect.o(i.MD_ConnectTXTask) refers to md_connect.o(i.BCC_CheckSum) for BCC_CheckSum
    md_connect.o(i.MD_ConnectTXTask) refers to pos_connect.o(i.DartCRC16) for DartCRC16
    md_connect.o(i.MD_ConnectTXTask) refers to md_connect.o(i.MD_Connect_BCDTou64) for MD_Connect_BCDTou64
    md_connect.o(i.MD_ConnectTXTask) refers to ldiv.o(.text) for __aeabi_ldivmod
    md_connect.o(i.MD_ConnectTXTask) refers to md_connect.o(i.InteiHEXCheck) for InteiHEXCheck
    md_connect.o(i.MD_ConnectTXTask) refers to md_connect.o(i.CheckSum8) for CheckSum8
    md_connect.o(i.MD_ConnectTXTask) refers to fram.o(i.FMItemWrite) for FMItemWrite
    md_connect.o(i.MD_ConnectTXTask) refers to multiplex_port.o(i.Price_DataCheck) for Price_DataCheck
    md_connect.o(i.MD_ConnectTXTask) refers to stm32f4xx_gpio.o(i.GPIO_ResetBits) for GPIO_ResetBits
    md_connect.o(i.MD_ConnectTXTask) refers to stm32f4xx_dma.o(i.DMA_Cmd) for DMA_Cmd
    md_connect.o(i.MD_ConnectTXTask) refers to log.o(i.Log_Task) for Log_Task
    md_connect.o(i.MD_ConnectTXTask) refers to strlen.o(.text) for strlen
    md_connect.o(i.MD_ConnectTXTask) refers to md_connect.o(.constdata) for MD_ATRec
    md_connect.o(i.MD_Connect_BCDTou64) refers to llsshr.o(.text) for __aeabi_lasr
    md_connect.o(i.MD_Connect_BCDTou64) refers to dfltui.o(.text) for __aeabi_ui2d
    md_connect.o(i.MD_Connect_BCDTou64) refers to pow.o(i.__hardfp_pow) for __hardfp_pow
    md_connect.o(i.MD_Connect_BCDTou64) refers to dflti.o(.text) for __aeabi_i2d
    md_connect.o(i.MD_Connect_BCDTou64) refers to dmul.o(.text) for __aeabi_dmul
    md_connect.o(i.MD_Connect_BCDTou64) refers to dfltl.o(.text) for __aeabi_l2d
    md_connect.o(i.MD_Connect_BCDTou64) refers to dadd.o(.text) for __aeabi_dadd
    md_connect.o(i.MD_Connect_BCDTou64) refers to dfixl.o(.text) for __aeabi_d2lz
    md_connect.o(i.MD_Connect_DMARX1_IRQHandler) refers to stm32f4xx_usart.o(i.USART_GetITStatus) for USART_GetITStatus
    md_connect.o(i.MD_Connect_DMARX1_IRQHandler) refers to stm32f4xx_usart.o(i.USART_ClearFlag) for USART_ClearFlag
    md_connect.o(i.MD_Connect_DMARX1_IRQHandler) refers to txh.o(.bss) for TXHData
    md_connect.o(i.MD_Connect_DMARX2_IRQHandler) refers to stm32f4xx_usart.o(i.USART_GetITStatus) for USART_GetITStatus
    md_connect.o(i.MD_Connect_DMARX2_IRQHandler) refers to txh.o(.bss) for TXHData
    md_connect.o(i.MD_Connect_DMARX3_IRQHandler) refers to stm32f4xx_usart.o(i.USART_GetITStatus) for USART_GetITStatus
    md_connect.o(i.MD_Connect_DMARX3_IRQHandler) refers to txh.o(.bss) for TXHData
    md_connect.o(i.MD_Connect_DMARX4_IRQHandler) refers to stm32f4xx_usart.o(i.USART_GetITStatus) for USART_GetITStatus
    md_connect.o(i.MD_Connect_DMARX4_IRQHandler) refers to txh.o(.bss) for TXHData
    md_connect.o(i.MD_Connect_DMATX1_IRQHandler) refers to stm32f4xx_dma.o(i.DMA_ClearFlag) for DMA_ClearFlag
    md_connect.o(i.MD_Connect_DMATX1_IRQHandler) refers to stm32f4xx_dma.o(i.DMA_Cmd) for DMA_Cmd
    md_connect.o(i.MD_Connect_DMATX1_IRQHandler) refers to stm32f4xx_usart.o(i.USART_GetFlagStatus) for USART_GetFlagStatus
    md_connect.o(i.MD_Connect_DMATX1_IRQHandler) refers to stm32f4xx_gpio.o(i.GPIO_SetBits) for GPIO_SetBits
    md_connect.o(i.MD_Connect_DMATX1_IRQHandler) refers to md_connect.o(.data) for MD_Connect_TX_Flag
    md_connect.o(i.MD_Connect_DMATX2_IRQHandler) refers to stm32f4xx_dma.o(i.DMA_ClearFlag) for DMA_ClearFlag
    md_connect.o(i.MD_Connect_DMATX2_IRQHandler) refers to stm32f4xx_dma.o(i.DMA_Cmd) for DMA_Cmd
    md_connect.o(i.MD_Connect_DMATX2_IRQHandler) refers to stm32f4xx_usart.o(i.USART_GetFlagStatus) for USART_GetFlagStatus
    md_connect.o(i.MD_Connect_DMATX2_IRQHandler) refers to stm32f4xx_gpio.o(i.GPIO_SetBits) for GPIO_SetBits
    md_connect.o(i.MD_Connect_DMATX2_IRQHandler) refers to md_connect.o(.data) for MD_Connect_TX_Flag
    md_connect.o(i.MD_Connect_DMATX3_IRQHandler) refers to stm32f4xx_dma.o(i.DMA_ClearFlag) for DMA_ClearFlag
    md_connect.o(i.MD_Connect_DMATX3_IRQHandler) refers to stm32f4xx_dma.o(i.DMA_Cmd) for DMA_Cmd
    md_connect.o(i.MD_Connect_DMATX3_IRQHandler) refers to stm32f4xx_usart.o(i.USART_GetFlagStatus) for USART_GetFlagStatus
    md_connect.o(i.MD_Connect_DMATX3_IRQHandler) refers to stm32f4xx_gpio.o(i.GPIO_SetBits) for GPIO_SetBits
    md_connect.o(i.MD_Connect_DMATX3_IRQHandler) refers to md_connect.o(.data) for MD_Connect_TX_Flag
    md_connect.o(i.MD_Connect_DMATX4_IRQHandler) refers to stm32f4xx_dma.o(i.DMA_ClearFlag) for DMA_ClearFlag
    md_connect.o(i.MD_Connect_DMATX4_IRQHandler) refers to stm32f4xx_dma.o(i.DMA_Cmd) for DMA_Cmd
    md_connect.o(i.MD_Connect_DMATX4_IRQHandler) refers to stm32f4xx_usart.o(i.USART_GetFlagStatus) for USART_GetFlagStatus
    md_connect.o(i.MD_Connect_DMATX4_IRQHandler) refers to stm32f4xx_gpio.o(i.GPIO_SetBits) for GPIO_SetBits
    md_connect.o(i.MD_Connect_DMATX4_IRQHandler) refers to md_connect.o(.data) for MD_Connect_TX_Flag
    md_connect.o(i.MD_Connect_DMA_Configuration) refers to stm32f4xx_rcc.o(i.RCC_AHB1PeriphClockCmd) for RCC_AHB1PeriphClockCmd
    md_connect.o(i.MD_Connect_DMA_Configuration) refers to stm32f4xx_dma.o(i.DMA_DeInit) for DMA_DeInit
    md_connect.o(i.MD_Connect_DMA_Configuration) refers to stm32f4xx_dma.o(i.DMA_Init) for DMA_Init
    md_connect.o(i.MD_Connect_DMA_Configuration) refers to stm32f4xx_dma.o(i.DMA_ITConfig) for DMA_ITConfig
    md_connect.o(i.MD_Connect_DMA_Configuration) refers to stm32f4xx_dma.o(i.DMA_Cmd) for DMA_Cmd
    md_connect.o(i.MD_Connect_DMA_Configuration) refers to md_connect.o(.bss) for MD_Connect_TX_Buff
    md_connect.o(i.MD_Connect_IO_Configuration) refers to stm32f4xx_rcc.o(i.RCC_AHB1PeriphClockCmd) for RCC_AHB1PeriphClockCmd
    md_connect.o(i.MD_Connect_IO_Configuration) refers to stm32f4xx_gpio.o(i.GPIO_PinAFConfig) for GPIO_PinAFConfig
    md_connect.o(i.MD_Connect_IO_Configuration) refers to stm32f4xx_gpio.o(i.GPIO_Init) for GPIO_Init
    md_connect.o(i.MD_Connect_IO_Configuration) refers to stm32f4xx_gpio.o(i.GPIO_ResetBits) for GPIO_ResetBits
    md_connect.o(i.MD_Connect_Init) refers to md_connect.o(i.MD_Connect_IO_Configuration) for MD_Connect_IO_Configuration
    md_connect.o(i.MD_Connect_Init) refers to md_connect.o(i.MD_Connect_DMA_Configuration) for MD_Connect_DMA_Configuration
    md_connect.o(i.MD_Connect_Init) refers to md_connect.o(i.MD_Port_Init) for MD_Port_Init
    md_connect.o(i.MD_Connect_Init) refers to md_connect.o(i.MD_Connect_NVIC_Configuration) for MD_Connect_NVIC_Configuration
    md_connect.o(i.MD_Connect_Init) refers to txh.o(.bss) for TXHData
    md_connect.o(i.MD_Connect_NVIC_Configuration) refers to misc.o(i.NVIC_Init) for NVIC_Init
    md_connect.o(i.MD_Connect_USART_Configuration) refers to stm32f4xx_rcc.o(i.RCC_APB1PeriphClockCmd) for RCC_APB1PeriphClockCmd
    md_connect.o(i.MD_Connect_USART_Configuration) refers to stm32f4xx_usart.o(i.USART_Init) for USART_Init
    md_connect.o(i.MD_Connect_USART_Configuration) refers to stm32f4xx_usart.o(i.USART_Cmd) for USART_Cmd
    md_connect.o(i.MD_Connect_USART_Configuration) refers to stm32f4xx_usart.o(i.USART_ITConfig) for USART_ITConfig
    md_connect.o(i.MD_Connect_USART_Configuration) refers to stm32f4xx_usart.o(i.USART_ClearFlag) for USART_ClearFlag
    md_connect.o(i.MD_Connect_USART_Configuration) refers to stm32f4xx_usart.o(i.USART_DMACmd) for USART_DMACmd
    md_connect.o(i.MD_Connect_u64ToBCD) refers to ldiv.o(.text) for __aeabi_ldivmod
    md_connect.o(i.MD_Port_Init) refers to md_connect.o(i.MD_Port_LORASet) for MD_Port_LORASet
    md_connect.o(i.MD_Port_Init) refers to md_connect.o(i.MD_Connect_DMA_Configuration) for MD_Connect_DMA_Configuration
    md_connect.o(i.MD_Port_Init) refers to md_connect.o(i.MD_Connect_USART_Configuration) for MD_Connect_USART_Configuration
    md_connect.o(i.MD_Port_Init) refers to stm32f4xx_gpio.o(i.GPIO_SetBits) for GPIO_SetBits
    md_connect.o(i.MD_Port_Init) refers to txh.o(.bss) for TXHData
    md_connect.o(i.MD_Port_LORASet) refers to stm32f4xx_gpio.o(i.GPIO_SetBits) for GPIO_SetBits
    md_connect.o(i.MD_Port_LORASet) refers to stm32f4xx_gpio.o(i.GPIO_ResetBits) for GPIO_ResetBits
    md_connect.o(i.MD_Port_LORASet) refers to delay.o(i.delay_ms) for delay_ms
    md_connect.o(i.MD_Port_LORASet) refers to md_connect.o(i.MD_Connect_USART_Configuration) for MD_Connect_USART_Configuration
    md_connect.o(i.MD_Port_LORASet) refers to stm32f4xx_dma.o(i.DMA_Cmd) for DMA_Cmd
    md_connect.o(i.MD_Port_LORASet) refers to log.o(i.Log_Task) for Log_Task
    md_connect.o(i.MD_Port_LORASet) refers to txh.o(.bss) for TXHData
    md_connect.o(i.MD_Port_LORASet) refers to md_connect.o(.bss) for LORA_Set
    md_connect.o(i.do_crc) refers to md_connect.o(.data) for crc16_ccitt_table
    pos_connect.o(i.CRC_Check) refers to pos_connect.o(.constdata) for auchCRCHi
    pos_connect.o(i.DartCRC16) refers to pos_connect.o(.constdata) for auchCRCHi
    pos_connect.o(i.POS_ConnectRXTask) refers to md_connect.o(i.MD_Connect_BCDTou64) for MD_Connect_BCDTou64
    pos_connect.o(i.POS_ConnectRXTask) refers to ds1307.o(i.DS1307_Write) for DS1307_Write
    pos_connect.o(i.POS_ConnectRXTask) refers to pos_connect.o(i.CRC_Check) for CRC_Check
    pos_connect.o(i.POS_ConnectRXTask) refers to log.o(i.Log_Task) for Log_Task
    pos_connect.o(i.POS_ConnectRXTask) refers to pos_connect.o(i.Decode_Data) for Decode_Data
    pos_connect.o(i.POS_ConnectRXTask) refers to txh.o(.bss) for TXHData
    pos_connect.o(i.POS_ConnectRXTask) refers to pos_connect.o(.bss) for POS_Connect_RX_Buff
    pos_connect.o(i.POS_ConnectRXTask) refers to pos_connect.o(.data) for POS_RX_RNGData
    pos_connect.o(i.POS_ConnectRXTask) refers to fram.o(i.FMItemWrite) for FMItemWrite
    pos_connect.o(i.POS_ConnectRXTask) refers to md_connect.o(i.MD_Port_Init) for MD_Port_Init
    pos_connect.o(i.POS_ConnectRXTask) refers to multiplex_port.o(i.Multiplex_Port_Init) for Multiplex_Port_Init
    pos_connect.o(i.POS_ConnectRXTask) refers to ds1307.o(i.DS1307_Read) for DS1307_Read
    pos_connect.o(i.POS_ConnectRXTask) refers to ds1307.o(i.DS1307_Init) for DS1307_Init
    pos_connect.o(i.POS_ConnectRXTask) refers to stm32f4xx_rng.o(i.RNG_GetRandomNumber) for RNG_GetRandomNumber
    pos_connect.o(i.POS_ConnectRXTask) refers to at45db.o(i.AT45DBItemWrite) for AT45DBItemWrite
    pos_connect.o(i.POS_ConnectRXTask) refers to multiplex_port.o(i.mystrstr) for mystrstr
    pos_connect.o(i.POS_ConnectTXTask) refers to memcpya.o(.text) for __aeabi_memcpy
    pos_connect.o(i.POS_ConnectTXTask) refers to pos_connect.o(.data) for POS_Connect_TX_Buff
    pos_connect.o(i.POS_ConnectTXTask) refers to txh.o(.bss) for TXHData
    pos_connect.o(i.POS_ConnectTXTask) refers to at45db.o(i.AT45DBItemWrite) for AT45DBItemWrite
    pos_connect.o(i.POS_ConnectTXTask) refers to fram.o(i.FMItemWrite) for FMItemWrite
    pos_connect.o(i.POS_ConnectTXTask) refers to stm32f4xx_rng.o(i.RNG_GetRandomNumber) for RNG_GetRandomNumber
    pos_connect.o(i.POS_ConnectTXTask) refers to txh.o(.constdata) for BoxVersion
    pos_connect.o(i.POS_ConnectTXTask) refers to llsshr.o(.text) for __aeabi_lasr
    pos_connect.o(i.POS_ConnectTXTask) refers to at45db.o(i.AT45DBItemRead) for AT45DBItemRead
    pos_connect.o(i.POS_ConnectTXTask) refers to pos_connect.o(i.Encrypt_Data) for Encrypt_Data
    pos_connect.o(i.POS_ConnectTXTask) refers to log.o(i.Log_Task) for Log_Task
    pos_connect.o(i.POS_ConnectTXTask) refers to pos_connect.o(i.CRC_Check) for CRC_Check
    pos_connect.o(i.POS_ConnectTXTask) refers to pos_connect.o(i.SUMCRC) for SUMCRC
    pos_connect.o(i.POS_ConnectTXTask) refers to stm32f4xx_dma.o(i.DMA_Cmd) for DMA_Cmd
    pos_connect.o(i.POS_ConnectTXTask) refers to strlen.o(.text) for strlen
    pos_connect.o(i.POS_ConnectTXTask) refers to strcat.o(.text) for strcat
    pos_connect.o(i.POS_ConnectTXTask) refers to pos_connect.o(.constdata) for CMD_Model_NET
    pos_connect.o(i.POS_ConnectTXTask) refers to multiplex_port.o(i.mystrstr) for mystrstr
    pos_connect.o(i.POS_Connect_DMARX_IRQHandler) refers to stm32f4xx_usart.o(i.USART_GetITStatus) for USART_GetITStatus
    pos_connect.o(i.POS_Connect_DMARX_IRQHandler) refers to stm32f4xx_usart.o(i.USART_ClearFlag) for USART_ClearFlag
    pos_connect.o(i.POS_Connect_DMARX_IRQHandler) refers to stm32f4xx_dma.o(i.DMA_Cmd) for DMA_Cmd
    pos_connect.o(i.POS_Connect_DMARX_IRQHandler) refers to stm32f4xx_dma.o(i.DMA_ClearFlag) for DMA_ClearFlag
    pos_connect.o(i.POS_Connect_DMARX_IRQHandler) refers to txh.o(.bss) for TXHData
    pos_connect.o(i.POS_Connect_DMATX_IRQHandler) refers to stm32f4xx_dma.o(i.DMA_ClearFlag) for DMA_ClearFlag
    pos_connect.o(i.POS_Connect_DMATX_IRQHandler) refers to stm32f4xx_dma.o(i.DMA_Cmd) for DMA_Cmd
    pos_connect.o(i.POS_Connect_DMA_Configuration) refers to stm32f4xx_rcc.o(i.RCC_AHB1PeriphClockCmd) for RCC_AHB1PeriphClockCmd
    pos_connect.o(i.POS_Connect_DMA_Configuration) refers to stm32f4xx_dma.o(i.DMA_DeInit) for DMA_DeInit
    pos_connect.o(i.POS_Connect_DMA_Configuration) refers to stm32f4xx_dma.o(i.DMA_Init) for DMA_Init
    pos_connect.o(i.POS_Connect_DMA_Configuration) refers to stm32f4xx_dma.o(i.DMA_ITConfig) for DMA_ITConfig
    pos_connect.o(i.POS_Connect_DMA_Configuration) refers to stm32f4xx_dma.o(i.DMA_Cmd) for DMA_Cmd
    pos_connect.o(i.POS_Connect_DMA_Configuration) refers to pos_connect.o(.data) for POS_Connect_TX_Buff
    pos_connect.o(i.POS_Connect_DMA_Configuration) refers to pos_connect.o(.bss) for POS_Connect_RX_Buff
    pos_connect.o(i.POS_Connect_IO_Configuration) refers to stm32f4xx_rcc.o(i.RCC_AHB1PeriphClockCmd) for RCC_AHB1PeriphClockCmd
    pos_connect.o(i.POS_Connect_IO_Configuration) refers to stm32f4xx_gpio.o(i.GPIO_PinAFConfig) for GPIO_PinAFConfig
    pos_connect.o(i.POS_Connect_IO_Configuration) refers to stm32f4xx_gpio.o(i.GPIO_Init) for GPIO_Init
    pos_connect.o(i.POS_Connect_Init) refers to pos_connect.o(i.POS_Connect_IO_Configuration) for POS_Connect_IO_Configuration
    pos_connect.o(i.POS_Connect_Init) refers to pos_connect.o(i.POS_Connect_DMA_Configuration) for POS_Connect_DMA_Configuration
    pos_connect.o(i.POS_Connect_Init) refers to pos_connect.o(i.POS_Connect_USART_Configuration) for POS_Connect_USART_Configuration
    pos_connect.o(i.POS_Connect_Init) refers to pos_connect.o(i.POS_Connect_NVIC_Configuration) for POS_Connect_NVIC_Configuration
    pos_connect.o(i.POS_Connect_Init) refers to stm32f4xx_rcc.o(i.RCC_AHB2PeriphClockCmd) for RCC_AHB2PeriphClockCmd
    pos_connect.o(i.POS_Connect_Init) refers to stm32f4xx_rng.o(i.RNG_Cmd) for RNG_Cmd
    pos_connect.o(i.POS_Connect_Init) refers to delay.o(i.delay_ms) for delay_ms
    pos_connect.o(i.POS_Connect_Init) refers to stm32f4xx_gpio.o(i.GPIO_SetBits) for GPIO_SetBits
    pos_connect.o(i.POS_Connect_Init) refers to stm32f4xx_gpio.o(i.GPIO_ResetBits) for GPIO_ResetBits
    pos_connect.o(i.POS_Connect_Init) refers to printf8.o(i.__0sprintf$8) for __2sprintf
    pos_connect.o(i.POS_Connect_Init) refers to fram.o(i.FMItemWrite) for FMItemWrite
    pos_connect.o(i.POS_Connect_Init) refers to txh.o(.bss) for TXHData
    pos_connect.o(i.POS_Connect_NVIC_Configuration) refers to misc.o(i.NVIC_Init) for NVIC_Init
    pos_connect.o(i.POS_Connect_USART_Configuration) refers to stm32f4xx_rcc.o(i.RCC_APB2PeriphClockCmd) for RCC_APB2PeriphClockCmd
    pos_connect.o(i.POS_Connect_USART_Configuration) refers to stm32f4xx_usart.o(i.USART_Init) for USART_Init
    pos_connect.o(i.POS_Connect_USART_Configuration) refers to stm32f4xx_usart.o(i.USART_Cmd) for USART_Cmd
    pos_connect.o(i.POS_Connect_USART_Configuration) refers to stm32f4xx_usart.o(i.USART_ITConfig) for USART_ITConfig
    pos_connect.o(i.POS_Connect_USART_Configuration) refers to stm32f4xx_usart.o(i.USART_ClearFlag) for USART_ClearFlag
    pos_connect.o(i.POS_Connect_USART_Configuration) refers to stm32f4xx_usart.o(i.USART_DMACmd) for USART_DMACmd
    pos_connect.o(i.POS_Connect_u64ToBCD) refers to ldiv.o(.text) for __aeabi_ldivmod
    pos_connect.o(i.POS_Network_APN_Set) refers to memcpya.o(.text) for __aeabi_memcpy4
    pos_connect.o(i.POS_Network_APN_Set) refers to strlen.o(.text) for strlen
    pos_connect.o(i.POS_Network_APN_Set) refers to stm32f4xx_dma.o(i.DMA_Cmd) for DMA_Cmd
    pos_connect.o(i.POS_Network_APN_Set) refers to delay.o(i.delay_ms) for delay_ms
    pos_connect.o(i.POS_Network_APN_Set) refers to strcat.o(.text) for strcat
    pos_connect.o(i.POS_Network_APN_Set) refers to pos_connect.o(.constdata) for .constdata
    pos_connect.o(i.POS_Network_APN_Set) refers to txh.o(.bss) for TXHData
    pos_connect.o(i.POS_Network_APN_Set) refers to pos_connect.o(.data) for POS_Connect_TX_Buff
    pos_connect.o(i.POS_WIFIReconnect) refers to strlen.o(.text) for strlen
    pos_connect.o(i.POS_WIFIReconnect) refers to strcat.o(.text) for strcat
    pos_connect.o(i.POS_WIFIReconnect) refers to stm32f4xx_dma.o(i.DMA_Cmd) for DMA_Cmd
    pos_connect.o(i.POS_WIFIReconnect) refers to delay.o(i.delay_ms) for delay_ms
    pos_connect.o(i.POS_WIFIReconnect) refers to pos_connect.o(.data) for POS_Connect_TX_Buff
    pos_connect.o(i.POS_WIFIReconnect) refers to txh.o(.bss) for TXHData
    pos_connect.o(i.POS_WIFIReconnect) refers to pos_connect.o(.constdata) for CMD_WifiWSSSID
    ds1307.o(i.DS1307_Init) refers to stm32f4xx_rcc.o(i.RCC_AHB1PeriphClockCmd) for RCC_AHB1PeriphClockCmd
    ds1307.o(i.DS1307_Init) refers to stm32f4xx_gpio.o(i.GPIO_Init) for GPIO_Init
    ds1307.o(i.DS1307_Init) refers to stm32f4xx_gpio.o(i.GPIO_SetBits) for GPIO_SetBits
    ds1307.o(i.DS1307_Init) refers to ds1307.o(i.DS1307_Read) for DS1307_Read
    ds1307.o(i.DS1307_Init) refers to ds1307.o(i.DS1307_Write) for DS1307_Write
    ds1307.o(i.DS1307_Init) refers to txh.o(.bss) for TXHData
    ds1307.o(i.DS1307_Read) refers to ds1307.o(i.iic_start) for iic_start
    ds1307.o(i.DS1307_Read) refers to ds1307.o(i.iic_sendbyte) for iic_sendbyte
    ds1307.o(i.DS1307_Read) refers to ds1307.o(i.iic_wait4ack) for iic_wait4ack
    ds1307.o(i.DS1307_Read) refers to ds1307.o(i.iic_readbyte) for iic_readbyte
    ds1307.o(i.DS1307_Read) refers to ds1307.o(i.iic_stop) for iic_stop
    ds1307.o(i.DS1307_Read) refers to txh.o(.bss) for TXHData
    ds1307.o(i.DS1307_Write) refers to ds1307.o(i.iic_start) for iic_start
    ds1307.o(i.DS1307_Write) refers to ds1307.o(i.iic_sendbyte) for iic_sendbyte
    ds1307.o(i.DS1307_Write) refers to ds1307.o(i.iic_wait4ack) for iic_wait4ack
    ds1307.o(i.DS1307_Write) refers to ds1307.o(i.iic_stop) for iic_stop
    ds1307.o(i.DS1307_Write) refers to txh.o(.bss) for TXHData
    ds1307.o(i.iic_ack) refers to stm32f4xx_gpio.o(i.GPIO_ResetBits) for GPIO_ResetBits
    ds1307.o(i.iic_ack) refers to delay.o(i.delay_us) for delay_us
    ds1307.o(i.iic_ack) refers to stm32f4xx_gpio.o(i.GPIO_SetBits) for GPIO_SetBits
    ds1307.o(i.iic_noack) refers to stm32f4xx_gpio.o(i.GPIO_ResetBits) for GPIO_ResetBits
    ds1307.o(i.iic_noack) refers to stm32f4xx_gpio.o(i.GPIO_SetBits) for GPIO_SetBits
    ds1307.o(i.iic_noack) refers to delay.o(i.delay_us) for delay_us
    ds1307.o(i.iic_readbyte) refers to stm32f4xx_gpio.o(i.GPIO_ResetBits) for GPIO_ResetBits
    ds1307.o(i.iic_readbyte) refers to delay.o(i.delay_us) for delay_us
    ds1307.o(i.iic_readbyte) refers to stm32f4xx_gpio.o(i.GPIO_SetBits) for GPIO_SetBits
    ds1307.o(i.iic_readbyte) refers to stm32f4xx_gpio.o(i.GPIO_ReadInputDataBit) for GPIO_ReadInputDataBit
    ds1307.o(i.iic_readbyte) refers to ds1307.o(i.iic_ack) for iic_ack
    ds1307.o(i.iic_readbyte) refers to ds1307.o(i.iic_noack) for iic_noack
    ds1307.o(i.iic_sendbyte) refers to stm32f4xx_gpio.o(i.GPIO_ResetBits) for GPIO_ResetBits
    ds1307.o(i.iic_sendbyte) refers to stm32f4xx_gpio.o(i.GPIO_SetBits) for GPIO_SetBits
    ds1307.o(i.iic_sendbyte) refers to delay.o(i.delay_us) for delay_us
    ds1307.o(i.iic_start) refers to stm32f4xx_gpio.o(i.GPIO_SetBits) for GPIO_SetBits
    ds1307.o(i.iic_start) refers to delay.o(i.delay_us) for delay_us
    ds1307.o(i.iic_start) refers to stm32f4xx_gpio.o(i.GPIO_ResetBits) for GPIO_ResetBits
    ds1307.o(i.iic_stop) refers to stm32f4xx_gpio.o(i.GPIO_ResetBits) for GPIO_ResetBits
    ds1307.o(i.iic_stop) refers to delay.o(i.delay_us) for delay_us
    ds1307.o(i.iic_stop) refers to stm32f4xx_gpio.o(i.GPIO_SetBits) for GPIO_SetBits
    ds1307.o(i.iic_wait4ack) refers to stm32f4xx_gpio.o(i.GPIO_SetBits) for GPIO_SetBits
    ds1307.o(i.iic_wait4ack) refers to delay.o(i.delay_us) for delay_us
    ds1307.o(i.iic_wait4ack) refers to ds1307.o(i.iic_stop) for iic_stop
    ds1307.o(i.iic_wait4ack) refers to stm32f4xx_gpio.o(i.GPIO_ReadInputDataBit) for GPIO_ReadInputDataBit
    ds1307.o(i.iic_wait4ack) refers to stm32f4xx_gpio.o(i.GPIO_ResetBits) for GPIO_ResetBits
    at45db.o(i.AT45DBItemRead) refers to at45db.o(i.AT45DB_ReadPage) for AT45DB_ReadPage
    at45db.o(i.AT45DBItemRead) refers to at45db.o(i.AT45DBDataCheck) for AT45DBDataCheck
    at45db.o(i.AT45DBItemRead) refers to delay.o(i.delay_ms) for delay_ms
    at45db.o(i.AT45DBItemRead) refers to at45db.o(.constdata) for AT45DBTab
    at45db.o(i.AT45DBItemRead) refers to at45db.o(.bss) for F_uniGlobal
    at45db.o(i.AT45DBItemRead) refers to at45db.o(.data) for CRCTemp
    at45db.o(i.AT45DBItemWrite) refers to at45db.o(i.AT45DBDataCheck) for AT45DBDataCheck
    at45db.o(i.AT45DBItemWrite) refers to at45db.o(i.AT45DB_WritePage) for AT45DB_WritePage
    at45db.o(i.AT45DBItemWrite) refers to at45db.o(i.AT45DBItemRead) for AT45DBItemRead
    at45db.o(i.AT45DBItemWrite) refers to delay.o(i.delay_ms) for delay_ms
    at45db.o(i.AT45DBItemWrite) refers to at45db.o(.constdata) for AT45DBTab
    at45db.o(i.AT45DB_Data_Init) refers to at45db.o(i.AT45DBDataCheck) for AT45DBDataCheck
    at45db.o(i.AT45DB_Data_Init) refers to at45db.o(i.AT45DB_WritePage) for AT45DB_WritePage
    at45db.o(i.AT45DB_Data_Init) refers to at45db.o(.constdata) for AT45DBTab
    at45db.o(i.AT45DB_Init) refers to at45db.o(i.ReadDriverID) for ReadDriverID
    at45db.o(i.AT45DB_Init) refers to at45db.o(i.AT45DB_SetPageByte) for AT45DB_SetPageByte
    at45db.o(i.AT45DB_Init) refers to at45db.o(.data) for FlashType
    at45db.o(i.AT45DB_Init) refers to txh.o(.bss) for TXHData
    at45db.o(i.AT45DB_ReadPage) refers to at45db.o(i.__set_PRIMASK) for __set_PRIMASK
    at45db.o(i.AT45DB_ReadPage) refers to at45db.o(i.ReadDFStatus) for ReadDFStatus
    at45db.o(i.AT45DB_ReadPage) refers to delay.o(i.delay_ms) for delay_ms
    at45db.o(i.AT45DB_ReadPage) refers to stm32f4xx_gpio.o(i.GPIO_ResetBits) for GPIO_ResetBits
    at45db.o(i.AT45DB_ReadPage) refers to stm32f4xx_gpio.o(i.GPIO_SetBits) for GPIO_SetBits
    at45db.o(i.AT45DB_ReadPage) refers to at45db.o(i.AT45DB_SendByte) for AT45DB_SendByte
    at45db.o(i.AT45DB_ReadPage) refers to at45db.o(.data) for ii
    at45db.o(i.AT45DB_SendByte) refers to stm32f4xx_spi.o(i.SPI_I2S_GetFlagStatus) for SPI_I2S_GetFlagStatus
    at45db.o(i.AT45DB_SendByte) refers to stm32f4xx_spi.o(i.SPI_I2S_SendData) for SPI_I2S_SendData
    at45db.o(i.AT45DB_SendByte) refers to stm32f4xx_spi.o(i.SPI_I2S_ReceiveData) for SPI_I2S_ReceiveData
    at45db.o(i.AT45DB_SetPageByte) refers to at45db.o(i.__set_PRIMASK) for __set_PRIMASK
    at45db.o(i.AT45DB_SetPageByte) refers to at45db.o(i.ReadDFStatus) for ReadDFStatus
    at45db.o(i.AT45DB_SetPageByte) refers to delay.o(i.delay_ms) for delay_ms
    at45db.o(i.AT45DB_SetPageByte) refers to stm32f4xx_gpio.o(i.GPIO_ResetBits) for GPIO_ResetBits
    at45db.o(i.AT45DB_SetPageByte) refers to stm32f4xx_gpio.o(i.GPIO_SetBits) for GPIO_SetBits
    at45db.o(i.AT45DB_SetPageByte) refers to at45db.o(i.AT45DB_SendByte) for AT45DB_SendByte
    at45db.o(i.AT45DB_SetPageByte) refers to at45db.o(.data) for ii
    at45db.o(i.AT45DB_WriteBuff) refers to at45db.o(i.__set_PRIMASK) for __set_PRIMASK
    at45db.o(i.AT45DB_WriteBuff) refers to at45db.o(i.ReadDFStatus) for ReadDFStatus
    at45db.o(i.AT45DB_WriteBuff) refers to delay.o(i.delay_ms) for delay_ms
    at45db.o(i.AT45DB_WriteBuff) refers to stm32f4xx_gpio.o(i.GPIO_ResetBits) for GPIO_ResetBits
    at45db.o(i.AT45DB_WriteBuff) refers to stm32f4xx_gpio.o(i.GPIO_SetBits) for GPIO_SetBits
    at45db.o(i.AT45DB_WriteBuff) refers to at45db.o(i.AT45DB_SendByte) for AT45DB_SendByte
    at45db.o(i.AT45DB_WriteBuff) refers to at45db.o(.data) for ii
    at45db.o(i.AT45DB_WritePage) refers to at45db.o(i.__set_PRIMASK) for __set_PRIMASK
    at45db.o(i.AT45DB_WritePage) refers to at45db.o(i.AT45DB_WriteBuff) for AT45DB_WriteBuff
    at45db.o(i.AT45DB_WritePage) refers to at45db.o(i.ReadDFStatus) for ReadDFStatus
    at45db.o(i.AT45DB_WritePage) refers to delay.o(i.delay_ms) for delay_ms
    at45db.o(i.AT45DB_WritePage) refers to stm32f4xx_gpio.o(i.GPIO_ResetBits) for GPIO_ResetBits
    at45db.o(i.AT45DB_WritePage) refers to stm32f4xx_gpio.o(i.GPIO_SetBits) for GPIO_SetBits
    at45db.o(i.AT45DB_WritePage) refers to at45db.o(i.AT45DB_SendByte) for AT45DB_SendByte
    at45db.o(i.AT45DB_WritePage) refers to at45db.o(.data) for ii
    at45db.o(i.ReadDFStatus) refers to at45db.o(i.__set_PRIMASK) for __set_PRIMASK
    at45db.o(i.ReadDFStatus) refers to stm32f4xx_gpio.o(i.GPIO_ResetBits) for GPIO_ResetBits
    at45db.o(i.ReadDFStatus) refers to stm32f4xx_gpio.o(i.GPIO_SetBits) for GPIO_SetBits
    at45db.o(i.ReadDFStatus) refers to at45db.o(i.AT45DB_SendByte) for AT45DB_SendByte
    at45db.o(i.ReadDriverID) refers to at45db.o(i.__set_PRIMASK) for __set_PRIMASK
    at45db.o(i.ReadDriverID) refers to at45db.o(i.ReadDFStatus) for ReadDFStatus
    at45db.o(i.ReadDriverID) refers to delay.o(i.delay_ms) for delay_ms
    at45db.o(i.ReadDriverID) refers to stm32f4xx_gpio.o(i.GPIO_ResetBits) for GPIO_ResetBits
    at45db.o(i.ReadDriverID) refers to stm32f4xx_gpio.o(i.GPIO_SetBits) for GPIO_SetBits
    at45db.o(i.ReadDriverID) refers to at45db.o(i.AT45DB_SendByte) for AT45DB_SendByte
    at45db.o(i.ReadDriverID) refers to at45db.o(.data) for ii
    at45db.o(.constdata) refers to at45db.o(.bss) for F_uniGlobal
    at45db.o(.constdata) refers to txh.o(.bss) for TXHData
    pluse_putout.o(i.Pluse_Putout_IO_Configuration) refers to stm32f4xx_rcc.o(i.RCC_AHB1PeriphClockCmd) for RCC_AHB1PeriphClockCmd
    pluse_putout.o(i.Pluse_Putout_IO_Configuration) refers to stm32f4xx_gpio.o(i.GPIO_Init) for GPIO_Init
    pluse_putout.o(i.Pluse_Putout_IO_Configuration) refers to stm32f4xx_gpio.o(i.GPIO_ResetBits) for GPIO_ResetBits
    pluse_putout.o(i.Pluse_Putout_IO_Configuration) refers to txh.o(.bss) for TXHData
    pluse_putout.o(i.Pluse_Putout_Init) refers to pluse_putout.o(i.Pluse_Putout_IO_Configuration) for Pluse_Putout_IO_Configuration
    analog.o(i.Pressure_ADCDMA_IRQHandler) refers to stm32f4xx_dma.o(i.DMA_ClearFlag) for DMA_ClearFlag
    analog.o(i.Pressure_ADCDMA_IRQHandler) refers to analog.o(.data) for PrssureTask_Flag
    analog.o(i.Pressure_ADC_Configuration) refers to stm32f4xx_rcc.o(i.RCC_APB2PeriphClockCmd) for RCC_APB2PeriphClockCmd
    analog.o(i.Pressure_ADC_Configuration) refers to stm32f4xx_rcc.o(i.RCC_APB2PeriphResetCmd) for RCC_APB2PeriphResetCmd
    analog.o(i.Pressure_ADC_Configuration) refers to stm32f4xx_adc.o(i.ADC_CommonInit) for ADC_CommonInit
    analog.o(i.Pressure_ADC_Configuration) refers to stm32f4xx_adc.o(i.ADC_Init) for ADC_Init
    analog.o(i.Pressure_ADC_Configuration) refers to stm32f4xx_adc.o(i.ADC_RegularChannelConfig) for ADC_RegularChannelConfig
    analog.o(i.Pressure_ADC_Configuration) refers to stm32f4xx_adc.o(i.ADC_DMACmd) for ADC_DMACmd
    analog.o(i.Pressure_ADC_Configuration) refers to stm32f4xx_adc.o(i.ADC_Cmd) for ADC_Cmd
    analog.o(i.Pressure_ADC_Configuration) refers to stm32f4xx_adc.o(i.ADC_DMARequestAfterLastTransferCmd) for ADC_DMARequestAfterLastTransferCmd
    analog.o(i.Pressure_ADC_Configuration) refers to stm32f4xx_adc.o(i.ADC_SoftwareStartConv) for ADC_SoftwareStartConv
    analog.o(i.Pressure_DMA_Configuration) refers to stm32f4xx_rcc.o(i.RCC_AHB1PeriphClockCmd) for RCC_AHB1PeriphClockCmd
    analog.o(i.Pressure_DMA_Configuration) refers to stm32f4xx_dma.o(i.DMA_DeInit) for DMA_DeInit
    analog.o(i.Pressure_DMA_Configuration) refers to stm32f4xx_dma.o(i.DMA_Init) for DMA_Init
    analog.o(i.Pressure_DMA_Configuration) refers to stm32f4xx_dma.o(i.DMA_ITConfig) for DMA_ITConfig
    analog.o(i.Pressure_DMA_Configuration) refers to stm32f4xx_dma.o(i.DMA_ClearFlag) for DMA_ClearFlag
    analog.o(i.Pressure_DMA_Configuration) refers to stm32f4xx_dma.o(i.DMA_Cmd) for DMA_Cmd
    analog.o(i.Pressure_DMA_Configuration) refers to analog.o(.bss) for PressureAdcBuf
    analog.o(i.Pressure_IO_Configuration) refers to stm32f4xx_rcc.o(i.RCC_AHB1PeriphClockCmd) for RCC_AHB1PeriphClockCmd
    analog.o(i.Pressure_IO_Configuration) refers to stm32f4xx_gpio.o(i.GPIO_Init) for GPIO_Init
    analog.o(i.Pressure_Init) refers to analog.o(i.Pressure_IO_Configuration) for Pressure_IO_Configuration
    analog.o(i.Pressure_Init) refers to analog.o(i.Pressure_ADC_Configuration) for Pressure_ADC_Configuration
    analog.o(i.Pressure_Init) refers to analog.o(i.Pressure_DMA_Configuration) for Pressure_DMA_Configuration
    analog.o(i.Pressure_Init) refers to analog.o(i.Pressure_NVIC_Configuration) for Pressure_NVIC_Configuration
    analog.o(i.Pressure_Init) refers to txh.o(.bss) for TXHData
    analog.o(i.Pressure_NVIC_Configuration) refers to misc.o(i.NVIC_Init) for NVIC_Init
    analog.o(i.PrssureTask) refers to analog.o(.bss) for PressureAdcBuf
    analog.o(i.PrssureTask) refers to analog.o(.data) for PrssureTask_Flag
    file_sys.o(i.CH376ByteLocate) refers to file_sys.o(i.xWriteCH376Cmd) for xWriteCH376Cmd
    file_sys.o(i.CH376ByteLocate) refers to file_sys.o(i.xWriteCH376Data) for xWriteCH376Data
    file_sys.o(i.CH376ByteLocate) refers to stm32f4xx_gpio.o(i.GPIO_SetBits) for GPIO_SetBits
    file_sys.o(i.CH376ByteLocate) refers to file_sys.o(i.Wait376Interrupt) for Wait376Interrupt
    file_sys.o(i.CH376ByteRead) refers to file_sys.o(i.xWriteCH376Cmd) for xWriteCH376Cmd
    file_sys.o(i.CH376ByteRead) refers to file_sys.o(i.xWriteCH376Data) for xWriteCH376Data
    file_sys.o(i.CH376ByteRead) refers to stm32f4xx_gpio.o(i.GPIO_SetBits) for GPIO_SetBits
    file_sys.o(i.CH376ByteRead) refers to file_sys.o(i.Wait376Interrupt) for Wait376Interrupt
    file_sys.o(i.CH376ByteRead) refers to file_sys.o(i.CH376ReadBlock) for CH376ReadBlock
    file_sys.o(i.CH376ByteWrite) refers to file_sys.o(i.xWriteCH376Cmd) for xWriteCH376Cmd
    file_sys.o(i.CH376ByteWrite) refers to file_sys.o(i.xWriteCH376Data) for xWriteCH376Data
    file_sys.o(i.CH376ByteWrite) refers to stm32f4xx_gpio.o(i.GPIO_SetBits) for GPIO_SetBits
    file_sys.o(i.CH376ByteWrite) refers to file_sys.o(i.Wait376Interrupt) for Wait376Interrupt
    file_sys.o(i.CH376ByteWrite) refers to file_sys.o(i.CH376WriteReqBlock) for CH376WriteReqBlock
    file_sys.o(i.CH376DirCreate) refers to file_sys.o(i.CH376SetFileName) for CH376SetFileName
    file_sys.o(i.CH376DirCreate) refers to file_sys.o(i.CH376WriteVar32) for CH376WriteVar32
    file_sys.o(i.CH376DirCreate) refers to file_sys.o(i.CH376SendCmdWaitInt) for CH376SendCmdWaitInt
    file_sys.o(i.CH376DirInfoRead) refers to file_sys.o(i.CH376SendCmdDatWaitInt) for CH376SendCmdDatWaitInt
    file_sys.o(i.CH376DirInfoSave) refers to file_sys.o(i.CH376SendCmdWaitInt) for CH376SendCmdWaitInt
    file_sys.o(i.CH376DiskCapacity) refers to file_sys.o(i.CH376SendCmdWaitInt) for CH376SendCmdWaitInt
    file_sys.o(i.CH376DiskCapacity) refers to file_sys.o(i.xWriteCH376Cmd) for xWriteCH376Cmd
    file_sys.o(i.CH376DiskCapacity) refers to file_sys.o(i.xReadCH376Data) for xReadCH376Data
    file_sys.o(i.CH376DiskCapacity) refers to file_sys.o(i.CH376Read32bitDat) for CH376Read32bitDat
    file_sys.o(i.CH376DiskConnect) refers to file_sys.o(i.Query376Interrupt) for Query376Interrupt
    file_sys.o(i.CH376DiskConnect) refers to file_sys.o(i.CH376GetIntStatus) for CH376GetIntStatus
    file_sys.o(i.CH376DiskConnect) refers to file_sys.o(i.CH376SendCmdWaitInt) for CH376SendCmdWaitInt
    file_sys.o(i.CH376DiskMount) refers to file_sys.o(i.CH376SendCmdWaitInt) for CH376SendCmdWaitInt
    file_sys.o(i.CH376DiskQuery) refers to file_sys.o(i.xWriteCH376Cmd) for xWriteCH376Cmd
    file_sys.o(i.CH376DiskQuery) refers to file_sys.o(i.xReadCH376Data) for xReadCH376Data
    file_sys.o(i.CH376DiskQuery) refers to file_sys.o(i.CH376ReadVar8) for CH376ReadVar8
    file_sys.o(i.CH376DiskQuery) refers to file_sys.o(i.CH376WriteVar8) for CH376WriteVar8
    file_sys.o(i.CH376DiskQuery) refers to file_sys.o(i.CH376SendCmdWaitInt) for CH376SendCmdWaitInt
    file_sys.o(i.CH376DiskQuery) refers to stm32f4xx_gpio.o(i.GPIO_SetBits) for GPIO_SetBits
    file_sys.o(i.CH376DiskReqSense) refers to delay.o(i.delay_us) for delay_us
    file_sys.o(i.CH376DiskReqSense) refers to file_sys.o(i.CH376SendCmdWaitInt) for CH376SendCmdWaitInt
    file_sys.o(i.CH376EndDirInfo) refers to file_sys.o(i.CH376WriteVar8) for CH376WriteVar8
    file_sys.o(i.CH376FileClose) refers to file_sys.o(i.CH376SendCmdDatWaitInt) for CH376SendCmdDatWaitInt
    file_sys.o(i.CH376FileCreate) refers to file_sys.o(i.CH376SetFileName) for CH376SetFileName
    file_sys.o(i.CH376FileCreate) refers to file_sys.o(i.CH376SendCmdWaitInt) for CH376SendCmdWaitInt
    file_sys.o(i.CH376FileCreatePath) refers to file_sys.o(i.CH376SeparatePath) for CH376SeparatePath
    file_sys.o(i.CH376FileCreatePath) refers to file_sys.o(i.CH376FileOpenDir) for CH376FileOpenDir
    file_sys.o(i.CH376FileCreatePath) refers to file_sys.o(i.CH376FileCreate) for CH376FileCreate
    file_sys.o(i.CH376FileErase) refers to file_sys.o(i.CH376FileOpenPath) for CH376FileOpenPath
    file_sys.o(i.CH376FileErase) refers to file_sys.o(i.CH376SetFileName) for CH376SetFileName
    file_sys.o(i.CH376FileErase) refers to file_sys.o(i.CH376SendCmdWaitInt) for CH376SendCmdWaitInt
    file_sys.o(i.CH376FileOpen) refers to file_sys.o(i.CH376SetFileName) for CH376SetFileName
    file_sys.o(i.CH376FileOpen) refers to file_sys.o(i.CH376WriteVar32) for CH376WriteVar32
    file_sys.o(i.CH376FileOpen) refers to file_sys.o(i.CH376SendCmdWaitInt) for CH376SendCmdWaitInt
    file_sys.o(i.CH376FileOpenDir) refers to file_sys.o(i.CH376FileOpen) for CH376FileOpen
    file_sys.o(i.CH376FileOpenPath) refers to file_sys.o(i.CH376FileOpenDir) for CH376FileOpenDir
    file_sys.o(i.CH376GetDiskStatus) refers to file_sys.o(i.CH376ReadVar8) for CH376ReadVar8
    file_sys.o(i.CH376GetFileSize) refers to file_sys.o(i.CH376ReadVar32) for CH376ReadVar32
    file_sys.o(i.CH376GetIntStatus) refers to file_sys.o(i.xWriteCH376Cmd) for xWriteCH376Cmd
    file_sys.o(i.CH376GetIntStatus) refers to file_sys.o(i.xReadCH376Data) for xReadCH376Data
    file_sys.o(i.CH376GetIntStatus) refers to stm32f4xx_gpio.o(i.GPIO_SetBits) for GPIO_SetBits
    file_sys.o(i.CH376Read32bitDat) refers to file_sys.o(i.xReadCH376Data) for xReadCH376Data
    file_sys.o(i.CH376Read32bitDat) refers to stm32f4xx_gpio.o(i.GPIO_SetBits) for GPIO_SetBits
    file_sys.o(i.CH376ReadBlock) refers to file_sys.o(i.xWriteCH376Cmd) for xWriteCH376Cmd
    file_sys.o(i.CH376ReadBlock) refers to file_sys.o(i.xReadCH376Data) for xReadCH376Data
    file_sys.o(i.CH376ReadBlock) refers to stm32f4xx_gpio.o(i.GPIO_SetBits) for GPIO_SetBits
    file_sys.o(i.CH376ReadVar32) refers to file_sys.o(i.xWriteCH376Cmd) for xWriteCH376Cmd
    file_sys.o(i.CH376ReadVar32) refers to file_sys.o(i.xWriteCH376Data) for xWriteCH376Data
    file_sys.o(i.CH376ReadVar32) refers to file_sys.o(i.CH376Read32bitDat) for CH376Read32bitDat
    file_sys.o(i.CH376ReadVar8) refers to file_sys.o(i.xWriteCH376Cmd) for xWriteCH376Cmd
    file_sys.o(i.CH376ReadVar8) refers to file_sys.o(i.xWriteCH376Data) for xWriteCH376Data
    file_sys.o(i.CH376ReadVar8) refers to file_sys.o(i.xReadCH376Data) for xReadCH376Data
    file_sys.o(i.CH376ReadVar8) refers to stm32f4xx_gpio.o(i.GPIO_SetBits) for GPIO_SetBits
    file_sys.o(i.CH376SecLocate) refers to file_sys.o(i.xWriteCH376Cmd) for xWriteCH376Cmd
    file_sys.o(i.CH376SecLocate) refers to file_sys.o(i.xWriteCH376Data) for xWriteCH376Data
    file_sys.o(i.CH376SecLocate) refers to stm32f4xx_gpio.o(i.GPIO_SetBits) for GPIO_SetBits
    file_sys.o(i.CH376SecLocate) refers to file_sys.o(i.Wait376Interrupt) for Wait376Interrupt
    file_sys.o(i.CH376SendCmdDatWaitInt) refers to file_sys.o(i.xWriteCH376Cmd) for xWriteCH376Cmd
    file_sys.o(i.CH376SendCmdDatWaitInt) refers to file_sys.o(i.xWriteCH376Data) for xWriteCH376Data
    file_sys.o(i.CH376SendCmdDatWaitInt) refers to stm32f4xx_gpio.o(i.GPIO_SetBits) for GPIO_SetBits
    file_sys.o(i.CH376SendCmdDatWaitInt) refers to file_sys.o(i.Wait376Interrupt) for Wait376Interrupt
    file_sys.o(i.CH376SendCmdWaitInt) refers to file_sys.o(i.xWriteCH376Cmd) for xWriteCH376Cmd
    file_sys.o(i.CH376SendCmdWaitInt) refers to stm32f4xx_gpio.o(i.GPIO_SetBits) for GPIO_SetBits
    file_sys.o(i.CH376SendCmdWaitInt) refers to file_sys.o(i.Wait376Interrupt) for Wait376Interrupt
    file_sys.o(i.CH376SetFileName) refers to file_sys.o(i.xWriteCH376Cmd) for xWriteCH376Cmd
    file_sys.o(i.CH376SetFileName) refers to file_sys.o(i.xReadCH376Data) for xReadCH376Data
    file_sys.o(i.CH376SetFileName) refers to file_sys.o(i.CH376ReadVar8) for CH376ReadVar8
    file_sys.o(i.CH376SetFileName) refers to file_sys.o(i.xWriteCH376Data) for xWriteCH376Data
    file_sys.o(i.CH376SetFileName) refers to file_sys.o(i.CH376SendCmdWaitInt) for CH376SendCmdWaitInt
    file_sys.o(i.CH376SetFileName) refers to file_sys.o(i.CH376ReadVar32) for CH376ReadVar32
    file_sys.o(i.CH376SetFileName) refers to file_sys.o(i.CH376WriteVar32) for CH376WriteVar32
    file_sys.o(i.CH376SetFileName) refers to stm32f4xx_gpio.o(i.GPIO_SetBits) for GPIO_SetBits
    file_sys.o(i.CH376WriteHostBlock) refers to file_sys.o(i.xWriteCH376Cmd) for xWriteCH376Cmd
    file_sys.o(i.CH376WriteHostBlock) refers to file_sys.o(i.xWriteCH376Data) for xWriteCH376Data
    file_sys.o(i.CH376WriteHostBlock) refers to stm32f4xx_gpio.o(i.GPIO_SetBits) for GPIO_SetBits
    file_sys.o(i.CH376WriteOfsBlock) refers to file_sys.o(i.xWriteCH376Cmd) for xWriteCH376Cmd
    file_sys.o(i.CH376WriteOfsBlock) refers to file_sys.o(i.xWriteCH376Data) for xWriteCH376Data
    file_sys.o(i.CH376WriteOfsBlock) refers to stm32f4xx_gpio.o(i.GPIO_SetBits) for GPIO_SetBits
    file_sys.o(i.CH376WriteReqBlock) refers to file_sys.o(i.xWriteCH376Cmd) for xWriteCH376Cmd
    file_sys.o(i.CH376WriteReqBlock) refers to file_sys.o(i.xReadCH376Data) for xReadCH376Data
    file_sys.o(i.CH376WriteReqBlock) refers to file_sys.o(i.xWriteCH376Data) for xWriteCH376Data
    file_sys.o(i.CH376WriteReqBlock) refers to stm32f4xx_gpio.o(i.GPIO_SetBits) for GPIO_SetBits
    file_sys.o(i.CH376WriteVar32) refers to file_sys.o(i.xWriteCH376Cmd) for xWriteCH376Cmd
    file_sys.o(i.CH376WriteVar32) refers to file_sys.o(i.xWriteCH376Data) for xWriteCH376Data
    file_sys.o(i.CH376WriteVar32) refers to stm32f4xx_gpio.o(i.GPIO_SetBits) for GPIO_SetBits
    file_sys.o(i.CH376WriteVar8) refers to file_sys.o(i.xWriteCH376Cmd) for xWriteCH376Cmd
    file_sys.o(i.CH376WriteVar8) refers to file_sys.o(i.xWriteCH376Data) for xWriteCH376Data
    file_sys.o(i.CH376WriteVar8) refers to stm32f4xx_gpio.o(i.GPIO_SetBits) for GPIO_SetBits
    file_sys.o(i.Query376Interrupt) refers to stm32f4xx_gpio.o(i.GPIO_ReadInputDataBit) for GPIO_ReadInputDataBit
    file_sys.o(i.SPI2_Init) refers to stm32f4xx_rcc.o(i.RCC_APB1PeriphClockCmd) for RCC_APB1PeriphClockCmd
    file_sys.o(i.SPI2_Init) refers to stm32f4xx_rcc.o(i.RCC_AHB1PeriphClockCmd) for RCC_AHB1PeriphClockCmd
    file_sys.o(i.SPI2_Init) refers to stm32f4xx_gpio.o(i.GPIO_Init) for GPIO_Init
    file_sys.o(i.SPI2_Init) refers to stm32f4xx_gpio.o(i.GPIO_PinAFConfig) for GPIO_PinAFConfig
    file_sys.o(i.SPI2_Init) refers to stm32f4xx_spi.o(i.SPI_I2S_DeInit) for SPI_I2S_DeInit
    file_sys.o(i.SPI2_Init) refers to stm32f4xx_spi.o(i.SPI_Init) for SPI_Init
    file_sys.o(i.SPI2_Init) refers to stm32f4xx_spi.o(i.SPI_Cmd) for SPI_Cmd
    file_sys.o(i.SPI2_ReadWriteByte) refers to stm32f4xx_spi.o(i.SPI_I2S_GetFlagStatus) for SPI_I2S_GetFlagStatus
    file_sys.o(i.SPI2_ReadWriteByte) refers to stm32f4xx_spi.o(i.SPI_I2S_SendData) for SPI_I2S_SendData
    file_sys.o(i.SPI2_ReadWriteByte) refers to stm32f4xx_spi.o(i.SPI_I2S_ReceiveData) for SPI_I2S_ReceiveData
    file_sys.o(i.Spi376OutByte) refers to file_sys.o(i.SPI2_ReadWriteByte) for SPI2_ReadWriteByte
    file_sys.o(i.Wait376Interrupt) refers to file_sys.o(i.Query376Interrupt) for Query376Interrupt
    file_sys.o(i.Wait376Interrupt) refers to file_sys.o(i.CH376GetIntStatus) for CH376GetIntStatus
    file_sys.o(i.mInitCH376Host) refers to file_sys.o(i.SPI2_Init) for SPI2_Init
    file_sys.o(i.mInitCH376Host) refers to file_sys.o(i.xWriteCH376Cmd) for xWriteCH376Cmd
    file_sys.o(i.mInitCH376Host) refers to file_sys.o(i.xWriteCH376Data) for xWriteCH376Data
    file_sys.o(i.mInitCH376Host) refers to file_sys.o(i.xReadCH376Data) for xReadCH376Data
    file_sys.o(i.mInitCH376Host) refers to stm32f4xx_gpio.o(i.GPIO_ResetBits) for GPIO_ResetBits
    file_sys.o(i.mInitCH376Host) refers to stm32f4xx_gpio.o(i.GPIO_SetBits) for GPIO_SetBits
    file_sys.o(i.mInitCH376Host) refers to delay.o(i.delay_us) for delay_us
    file_sys.o(i.xReadCH376Data) refers to delay.o(i.delay_us) for delay_us
    file_sys.o(i.xReadCH376Data) refers to file_sys.o(i.SPI2_ReadWriteByte) for SPI2_ReadWriteByte
    file_sys.o(i.xWriteCH376Cmd) refers to stm32f4xx_gpio.o(i.GPIO_SetBits) for GPIO_SetBits
    file_sys.o(i.xWriteCH376Cmd) refers to delay.o(i.delay_us) for delay_us
    file_sys.o(i.xWriteCH376Cmd) refers to stm32f4xx_gpio.o(i.GPIO_ResetBits) for GPIO_ResetBits
    file_sys.o(i.xWriteCH376Cmd) refers to file_sys.o(i.Spi376OutByte) for Spi376OutByte
    file_sys.o(i.xWriteCH376Data) refers to file_sys.o(i.Spi376OutByte) for Spi376OutByte
    file_sys.o(i.xWriteCH376Data) refers to delay.o(i.delay_us) for delay_us
    log.o(i.FindSysconfigFile) refers to file_sys.o(i.CH376DiskConnect) for CH376DiskConnect
    log.o(i.FindSysconfigFile) refers to file_sys.o(i.CH376FileOpen) for CH376FileOpen
    log.o(i.FindSysconfigFile) refers to file_sys.o(i.CH376GetFileSize) for CH376GetFileSize
    log.o(i.FindSysconfigFile) refers to file_sys.o(i.CH376ByteLocate) for CH376ByteLocate
    log.o(i.FindSysconfigFile) refers to file_sys.o(i.CH376ByteRead) for CH376ByteRead
    log.o(i.FindSysconfigFile) refers to multiplex_port.o(i.mystrstr) for mystrstr
    log.o(i.FindSysconfigFile) refers to fram.o(i.FMItemWrite) for FMItemWrite
    log.o(i.FindSysconfigFile) refers to file_sys.o(i.CH376FileClose) for CH376FileClose
    log.o(i.FindSysconfigFile) refers to file_sys.o(i.CH376FileCreate) for CH376FileCreate
    log.o(i.FindSysconfigFile) refers to file_sys.o(i.mInitCH376Host) for mInitCH376Host
    log.o(i.FindSysconfigFile) refers to log.o(.data) for SysconfigFileName
    log.o(i.FindSysconfigFile) refers to txh.o(.bss) for TXHData
    log.o(i.Log_Init) refers to file_sys.o(i.mInitCH376Host) for mInitCH376Host
    log.o(i.Log_Init) refers to delay.o(i.delay_ms) for delay_ms
    log.o(i.Log_Task) refers to file_sys.o(i.CH376DiskConnect) for CH376DiskConnect
    log.o(i.Log_Task) refers to file_sys.o(i.CH376FileOpen) for CH376FileOpen
    log.o(i.Log_Task) refers to file_sys.o(i.CH376GetFileSize) for CH376GetFileSize
    log.o(i.Log_Task) refers to file_sys.o(i.CH376ByteLocate) for CH376ByteLocate
    log.o(i.Log_Task) refers to file_sys.o(i.CH376ByteWrite) for CH376ByteWrite
    log.o(i.Log_Task) refers to file_sys.o(i.CH376FileClose) for CH376FileClose
    log.o(i.Log_Task) refers to file_sys.o(i.CH376FileCreate) for CH376FileCreate
    log.o(i.Log_Task) refers to file_sys.o(i.mInitCH376Host) for mInitCH376Host
    log.o(i.Log_Task) refers to txh.o(.bss) for TXHData
    log.o(i.Log_Task) refers to log.o(.data) for LogName
    oled.o(i.OLED_Clear) refers to oled.o(.bss) for OLED_GRAM
    oled.o(i.OLED_ColorTurn) refers to oled.o(i.OLED_WR_Byte) for OLED_WR_Byte
    oled.o(i.OLED_DisPlay_Off) refers to oled.o(i.OLED_WR_Byte) for OLED_WR_Byte
    oled.o(i.OLED_DisPlay_On) refers to oled.o(i.OLED_WR_Byte) for OLED_WR_Byte
    oled.o(i.OLED_DisplayTurn) refers to oled.o(i.OLED_WR_Byte) for OLED_WR_Byte
    oled.o(i.OLED_DrawArc) refers to dflti.o(.text) for __aeabi_i2d
    oled.o(i.OLED_DrawArc) refers to dmul.o(.text) for __aeabi_dmul
    oled.o(i.OLED_DrawArc) refers to d2f.o(.text) for __aeabi_d2f
    oled.o(i.OLED_DrawArc) refers to f2d.o(.text) for __aeabi_f2d
    oled.o(i.OLED_DrawArc) refers to ddiv.o(.text) for __aeabi_ddiv
    oled.o(i.OLED_DrawArc) refers to sin.o(i.__hardfp_sin) for __hardfp_sin
    oled.o(i.OLED_DrawArc) refers to dadd.o(.text) for __aeabi_dadd
    oled.o(i.OLED_DrawArc) refers to cos.o(i.__hardfp_cos) for __hardfp_cos
    oled.o(i.OLED_DrawArc) refers to oled.o(i.OLED_DrawPoint) for OLED_DrawPoint
    oled.o(i.OLED_DrawCircle) refers to oled.o(i.OLED_DrawPoint) for OLED_DrawPoint
    oled.o(i.OLED_DrawLine) refers to oled.o(i.OLED_DrawPoint) for OLED_DrawPoint
    oled.o(i.OLED_DrawPoint) refers to oled.o(.bss) for OLED_GRAM
    oled.o(i.OLED_Init) refers to stm32f4xx_rcc.o(i.RCC_AHB1PeriphClockCmd) for RCC_AHB1PeriphClockCmd
    oled.o(i.OLED_Init) refers to stm32f4xx_gpio.o(i.GPIO_Init) for GPIO_Init
    oled.o(i.OLED_Init) refers to delay.o(i.delay_ms) for delay_ms
    oled.o(i.OLED_Init) refers to stm32f4xx_gpio.o(i.GPIO_ResetBits) for GPIO_ResetBits
    oled.o(i.OLED_Init) refers to stm32f4xx_gpio.o(i.GPIO_SetBits) for GPIO_SetBits
    oled.o(i.OLED_Init) refers to oled.o(i.OLED_WR_Byte) for OLED_WR_Byte
    oled.o(i.OLED_Init) refers to oled.o(i.OLED_Clear) for OLED_Clear
    oled.o(i.OLED_Init) refers to oled.o(i.OLED_Refresh) for OLED_Refresh
    oled.o(i.OLED_Init) refers to txh.o(.bss) for TXHData
    oled.o(i.OLED_ProgressBar) refers to oled.o(i.OLED_DrawLine) for OLED_DrawLine
    oled.o(i.OLED_Refresh) refers to oled.o(i.OLED_WR_Byte) for OLED_WR_Byte
    oled.o(i.OLED_Refresh) refers to oled.o(.bss) for OLED_GRAM
    oled.o(i.OLED_SPI2_SendByte) refers to stm32f4xx_spi.o(i.SPI_I2S_GetFlagStatus) for SPI_I2S_GetFlagStatus
    oled.o(i.OLED_SPI2_SendByte) refers to stm32f4xx_spi.o(i.SPI_I2S_SendData) for SPI_I2S_SendData
    oled.o(i.OLED_SPI2_SendByte) refers to stm32f4xx_spi.o(i.SPI_I2S_ReceiveData) for SPI_I2S_ReceiveData
    oled.o(i.OLED_ShowChar) refers to oled.o(i.OLED_DrawPoint) for OLED_DrawPoint
    oled.o(i.OLED_ShowChar) refers to oled.o(.constdata) for asc2_0806
    oled.o(i.OLED_ShowNum) refers to dfltui.o(.text) for __aeabi_ui2d
    oled.o(i.OLED_ShowNum) refers to log10.o(i.__hardfp_log10) for __hardfp_log10
    oled.o(i.OLED_ShowNum) refers to dadd.o(.text) for __aeabi_dadd
    oled.o(i.OLED_ShowNum) refers to dfixi.o(.text) for __aeabi_d2iz
    oled.o(i.OLED_ShowNum) refers to oled.o(i.OLED_ShowChar) for OLED_ShowChar
    oled.o(i.OLED_ShowNum) refers to oled.o(i.OLED_Pow) for OLED_Pow
    oled.o(i.OLED_ShowPicture) refers to oled.o(i.OLED_DrawPoint) for OLED_DrawPoint
    oled.o(i.OLED_ShowString) refers to oled.o(i.OLED_ShowChar) for OLED_ShowChar
    oled.o(i.OLED_WR_Byte) refers to stm32f4xx_gpio.o(i.GPIO_SetBits) for GPIO_SetBits
    oled.o(i.OLED_WR_Byte) refers to stm32f4xx_gpio.o(i.GPIO_ResetBits) for GPIO_ResetBits
    oled.o(i.OLED_WR_Byte) refers to oled.o(i.OLED_SPI2_SendByte) for OLED_SPI2_SendByte
    surface.o(i.FindKey) refers to txh.o(.bss) for TXHData
    surface.o(i.FindKey) refers to surface.o(.data) for KeyNumconfirm_Flag
    surface.o(i.GetKeyNum) refers to txh.o(.bss) for TXHData
    surface.o(i.Sureface_Wait_TimeUpData) refers to md_connect.o(i.MD_Connect_BCDTou64) for MD_Connect_BCDTou64
    surface.o(i.Sureface_Wait_TimeUpData) refers to oled.o(i.OLED_ShowNum) for OLED_ShowNum
    surface.o(i.Sureface_Wait_TimeUpData) refers to oled.o(i.OLED_ShowChar) for OLED_ShowChar
    surface.o(i.Sureface_Wait_TimeUpData) refers to txh.o(.bss) for TXHData
    surface.o(i.SurfaceJump) refers to txh.o(.bss) for TXHData
    surface.o(i.SurfaceTast) refers to surface.o(i.FindKey) for FindKey
    surface.o(i.SurfaceTast) refers to oled.o(i.OLED_Clear) for OLED_Clear
    surface.o(i.SurfaceTast) refers to surface.o(i.GetKeyNum) for GetKeyNum
    surface.o(i.SurfaceTast) refers to surface.o(i.SurfaceJump) for SurfaceJump
    surface.o(i.SurfaceTast) refers to oled.o(i.OLED_ShowString) for OLED_ShowString
    surface.o(i.SurfaceTast) refers to oled.o(i.OLED_ShowNum) for OLED_ShowNum
    surface.o(i.SurfaceTast) refers to oled.o(i.OLED_ProgressBar) for OLED_ProgressBar
    surface.o(i.SurfaceTast) refers to oled.o(i.OLED_ShowChar) for OLED_ShowChar
    surface.o(i.SurfaceTast) refers to oled.o(i.OLED_ShowPicture) for OLED_ShowPicture
    surface.o(i.SurfaceTast) refers to surface.o(i.Sureface_Wait_TimeUpData) for Sureface_Wait_TimeUpData
    surface.o(i.SurfaceTast) refers to txh.o(.bss) for TXHData
    surface.o(i.SurfaceTast) refers to surface.o(.constdata) for BMP_Bluetooth_9
    surface.o(i.SurfaceTast) refers to printf8.o(i.__0sprintf$8) for __2sprintf
    surface.o(i.SurfaceTast) refers to surface.o(i.Surface_Copy_16) for Surface_Copy_16
    surface.o(i.SurfaceTast) refers to md_connect.o(i.MD_Connect_BCDTou64) for MD_Connect_BCDTou64
    surface.o(i.SurfaceTast) refers to pos_connect.o(.constdata) for TsatURL
    surface.o(i.SurfaceTast) refers to txh.o(.constdata) for BoxVersion
    surface.o(i.SurfaceTast) refers to fram.o(i.FMItemWrite) for FMItemWrite
    surface.o(i.SurfaceTast) refers to md_connect.o(i.MD_Port_Init) for MD_Port_Init
    surface.o(i.SurfaceTast) refers to md_connect.o(i.MD_Port_LORASet) for MD_Port_LORASet
    surface.o(i.SurfaceTast) refers to file_sys.o(i.CH376DiskConnect) for CH376DiskConnect
    surface.o(i.SurfaceTast) refers to fram.o(i.FM_Data_Init) for FM_Data_Init
    surface.o(i.SurfaceTast) refers to pos_connect.o(i.POS_Connect_Init) for POS_Connect_Init
    surface.o(i.SurfaceTast) refers to oled.o(i.OLED_Refresh) for OLED_Refresh
    surface.o(i.Surface_Copy_16) refers to oled.o(i.OLED_ShowChar) for OLED_ShowChar
    surface.o(i.Surface_Init) refers to surface.o(i.SurfaceJump) for SurfaceJump
    surface.o(i.Surface_Init) refers to txh.o(.bss) for TXHData
    printf.o(i.Print_Num) refers to llsshr.o(.text) for __aeabi_lasr
    printf.o(i.Print_Num) refers to txh.o(.bss) for TXHData
    multiplex_port.o(i.Multiplex_PortRXTask) refers to stm32f4xx_dma.o(i.DMA_Cmd) for DMA_Cmd
    multiplex_port.o(i.Multiplex_PortRXTask) refers to stm32f4xx_dma.o(i.DMA_ClearFlag) for DMA_ClearFlag
    multiplex_port.o(i.Multiplex_PortRXTask) refers to md_connect.o(i.CheckSum) for CheckSum
    multiplex_port.o(i.Multiplex_PortRXTask) refers to md_connect.o(i.StrToInt) for StrToInt
    multiplex_port.o(i.Multiplex_PortRXTask) refers to md_connect.o(i.StrToFloat) for StrToFloat
    multiplex_port.o(i.Multiplex_PortRXTask) refers to multiplex_port.o(i.Price_DataCheck) for Price_DataCheck
    multiplex_port.o(i.Multiplex_PortRXTask) refers to txh.o(.bss) for TXHData
    multiplex_port.o(i.Multiplex_PortRXTask) refers to multiplex_port.o(.data) for Multiplex_Port_RX_Flag
    multiplex_port.o(i.Multiplex_PortRXTask) refers to multiplex_port.o(i.mystrstr) for mystrstr
    multiplex_port.o(i.Multiplex_PortRXTask) refers to atof.o(i.__hardfp_atof) for __hardfp_atof
    multiplex_port.o(i.Multiplex_PortRXTask) refers to d2f.o(.text) for __aeabi_d2f
    multiplex_port.o(i.Multiplex_PortRXTask) refers to ffixl.o(.text) for __aeabi_f2lz
    multiplex_port.o(i.Multiplex_PortRXTask) refers to ffltl.o(.text) for __aeabi_l2f
    multiplex_port.o(i.Multiplex_PortTXTask) refers to multiplex_port.o(i.Multiplex_Port_Choose) for Multiplex_Port_Choose
    multiplex_port.o(i.Multiplex_PortTXTask) refers to multiplex_port.o(i.Multiplex_Port_USART_Configuration) for Multiplex_Port_USART_Configuration
    multiplex_port.o(i.Multiplex_PortTXTask) refers to md_connect.o(i.MD_Connect_u64ToBCD) for MD_Connect_u64ToBCD
    multiplex_port.o(i.Multiplex_PortTXTask) refers to printf.o(i.Print_Num) for Print_Num
    multiplex_port.o(i.Multiplex_PortTXTask) refers to multiplex_port.o(.data) for Multiplex_Port_TX_Flag
    multiplex_port.o(i.Multiplex_PortTXTask) refers to txh.o(.bss) for TXHData
    multiplex_port.o(i.Multiplex_PortTXTask) refers to stm32f4xx_gpio.o(i.GPIO_SetBits) for GPIO_SetBits
    multiplex_port.o(i.Multiplex_PortTXTask) refers to multiplex_port.o(i.Price_DataCheck) for Price_DataCheck
    multiplex_port.o(i.Multiplex_PortTXTask) refers to stm32f4xx_dma.o(i.DMA_Cmd) for DMA_Cmd
    multiplex_port.o(i.Multiplex_Port_Choose) refers to stm32f4xx_gpio.o(i.GPIO_ResetBits) for GPIO_ResetBits
    multiplex_port.o(i.Multiplex_Port_Choose) refers to stm32f4xx_gpio.o(i.GPIO_SetBits) for GPIO_SetBits
    multiplex_port.o(i.Multiplex_Port_DMARX_IRQHandler) refers to stm32f4xx_usart.o(i.USART_GetITStatus) for USART_GetITStatus
    multiplex_port.o(i.Multiplex_Port_DMARX_IRQHandler) refers to stm32f4xx_usart.o(i.USART_ClearFlag) for USART_ClearFlag
    multiplex_port.o(i.Multiplex_Port_DMARX_IRQHandler) refers to txh.o(.bss) for TXHData
    multiplex_port.o(i.Multiplex_Port_DMATX_IRQHandler) refers to stm32f4xx_dma.o(i.DMA_ClearFlag) for DMA_ClearFlag
    multiplex_port.o(i.Multiplex_Port_DMATX_IRQHandler) refers to stm32f4xx_dma.o(i.DMA_Cmd) for DMA_Cmd
    multiplex_port.o(i.Multiplex_Port_DMATX_IRQHandler) refers to stm32f4xx_usart.o(i.USART_GetFlagStatus) for USART_GetFlagStatus
    multiplex_port.o(i.Multiplex_Port_DMATX_IRQHandler) refers to stm32f4xx_gpio.o(i.GPIO_ResetBits) for GPIO_ResetBits
    multiplex_port.o(i.Multiplex_Port_DMATX_IRQHandler) refers to multiplex_port.o(.data) for Multiplex_Port_TX_Flag
    multiplex_port.o(i.Multiplex_Port_DMA_Configuration) refers to stm32f4xx_rcc.o(i.RCC_AHB1PeriphClockCmd) for RCC_AHB1PeriphClockCmd
    multiplex_port.o(i.Multiplex_Port_DMA_Configuration) refers to stm32f4xx_dma.o(i.DMA_DeInit) for DMA_DeInit
    multiplex_port.o(i.Multiplex_Port_DMA_Configuration) refers to stm32f4xx_dma.o(i.DMA_Init) for DMA_Init
    multiplex_port.o(i.Multiplex_Port_DMA_Configuration) refers to stm32f4xx_dma.o(i.DMA_ITConfig) for DMA_ITConfig
    multiplex_port.o(i.Multiplex_Port_DMA_Configuration) refers to stm32f4xx_dma.o(i.DMA_Cmd) for DMA_Cmd
    multiplex_port.o(i.Multiplex_Port_DMA_Configuration) refers to multiplex_port.o(.data) for Multiplex_Port_TX_Buff
    multiplex_port.o(i.Multiplex_Port_IO_Configuration) refers to stm32f4xx_rcc.o(i.RCC_AHB1PeriphClockCmd) for RCC_AHB1PeriphClockCmd
    multiplex_port.o(i.Multiplex_Port_IO_Configuration) refers to stm32f4xx_gpio.o(i.GPIO_PinAFConfig) for GPIO_PinAFConfig
    multiplex_port.o(i.Multiplex_Port_IO_Configuration) refers to stm32f4xx_gpio.o(i.GPIO_Init) for GPIO_Init
    multiplex_port.o(i.Multiplex_Port_IO_Configuration) refers to stm32f4xx_gpio.o(i.GPIO_ResetBits) for GPIO_ResetBits
    multiplex_port.o(i.Multiplex_Port_Init) refers to multiplex_port.o(i.Multiplex_Port_IO_Configuration) for Multiplex_Port_IO_Configuration
    multiplex_port.o(i.Multiplex_Port_Init) refers to multiplex_port.o(i.Multiplex_Port_USART_Configuration) for Multiplex_Port_USART_Configuration
    multiplex_port.o(i.Multiplex_Port_Init) refers to multiplex_port.o(i.Multiplex_Port_DMA_Configuration) for Multiplex_Port_DMA_Configuration
    multiplex_port.o(i.Multiplex_Port_Init) refers to multiplex_port.o(i.Multiplex_Port_NVIC_Configuration) for Multiplex_Port_NVIC_Configuration
    multiplex_port.o(i.Multiplex_Port_Init) refers to txh.o(.bss) for TXHData
    multiplex_port.o(i.Multiplex_Port_NVIC_Configuration) refers to misc.o(i.NVIC_Init) for NVIC_Init
    multiplex_port.o(i.Multiplex_Port_USART_Configuration) refers to stm32f4xx_rcc.o(i.RCC_APB2PeriphClockCmd) for RCC_APB2PeriphClockCmd
    multiplex_port.o(i.Multiplex_Port_USART_Configuration) refers to stm32f4xx_usart.o(i.USART_Init) for USART_Init
    multiplex_port.o(i.Multiplex_Port_USART_Configuration) refers to stm32f4xx_usart.o(i.USART_Cmd) for USART_Cmd
    multiplex_port.o(i.Multiplex_Port_USART_Configuration) refers to stm32f4xx_usart.o(i.USART_ITConfig) for USART_ITConfig
    multiplex_port.o(i.Multiplex_Port_USART_Configuration) refers to stm32f4xx_usart.o(i.USART_ClearFlag) for USART_ClearFlag
    multiplex_port.o(i.Multiplex_Port_USART_Configuration) refers to stm32f4xx_usart.o(i.USART_DMACmd) for USART_DMACmd
    multiplex_port.o(i.mystrstr) refers to strlen.o(.text) for strlen
    multiplex_port.o(i.mystrstr) refers to strncmp.o(.text) for strncmp
    delay.o(i.delay_init) refers to misc.o(i.SysTick_CLKSourceConfig) for SysTick_CLKSourceConfig
    atof.o(i.__hardfp_atof) refers (Special) to iusefp.o(.text) for __I$use$fp
    atof.o(i.__hardfp_atof) refers to errno.o(i.__read_errno) for __read_errno
    atof.o(i.__hardfp_atof) refers to strtod.o(.text) for __strtod_int
    atof.o(i.__hardfp_atof) refers to errno.o(i.__set_errno) for __set_errno
    atof.o(i.__softfp_atof) refers (Special) to iusefp.o(.text) for __I$use$fp
    atof.o(i.__softfp_atof) refers to errno.o(i.__read_errno) for __read_errno
    atof.o(i.__softfp_atof) refers to strtod.o(.text) for __strtod_int
    atof.o(i.__softfp_atof) refers to errno.o(i.__set_errno) for __set_errno
    atof.o(i.atof) refers (Special) to iusefp.o(.text) for __I$use$fp
    atof.o(i.atof) refers to errno.o(i.__read_errno) for __read_errno
    atof.o(i.atof) refers to strtod.o(.text) for __strtod_int
    atof.o(i.atof) refers to errno.o(i.__set_errno) for __set_errno
    cos.o(i.__hardfp_cos) refers (Special) to iusefp.o(.text) for __I$use$fp
    cos.o(i.__hardfp_cos) refers to errno.o(i.__set_errno) for __set_errno
    cos.o(i.__hardfp_cos) refers to dunder.o(i.__mathlib_dbl_invalid) for __mathlib_dbl_invalid
    cos.o(i.__hardfp_cos) refers to dunder.o(i.__mathlib_dbl_infnan) for __mathlib_dbl_infnan
    cos.o(i.__hardfp_cos) refers to rred.o(i.__ieee754_rem_pio2) for __ieee754_rem_pio2
    cos.o(i.__hardfp_cos) refers to sin_i.o(i.__kernel_sin) for __kernel_sin
    cos.o(i.__hardfp_cos) refers to cos_i.o(i.__kernel_cos) for __kernel_cos
    cos.o(i.__softfp_cos) refers (Special) to iusefp.o(.text) for __I$use$fp
    cos.o(i.__softfp_cos) refers to cos.o(i.__hardfp_cos) for __hardfp_cos
    cos.o(i.cos) refers (Special) to iusefp.o(.text) for __I$use$fp
    cos.o(i.cos) refers to cos.o(i.__hardfp_cos) for __hardfp_cos
    cos_x.o(i.____hardfp_cos$lsc) refers (Special) to iusefp.o(.text) for __I$use$fp
    cos_x.o(i.____hardfp_cos$lsc) refers to errno.o(i.__set_errno) for __set_errno
    cos_x.o(i.____hardfp_cos$lsc) refers to dunder.o(i.__mathlib_dbl_infnan) for __mathlib_dbl_infnan
    cos_x.o(i.____hardfp_cos$lsc) refers to rred.o(i.__ieee754_rem_pio2) for __ieee754_rem_pio2
    cos_x.o(i.____hardfp_cos$lsc) refers to sin_i.o(i.__kernel_sin) for __kernel_sin
    cos_x.o(i.____hardfp_cos$lsc) refers to cos_i.o(i.__kernel_cos) for __kernel_cos
    cos_x.o(i.____softfp_cos$lsc) refers (Special) to iusefp.o(.text) for __I$use$fp
    cos_x.o(i.____softfp_cos$lsc) refers to cos_x.o(i.____hardfp_cos$lsc) for ____hardfp_cos$lsc
    cos_x.o(i.__cos$lsc) refers (Special) to iusefp.o(.text) for __I$use$fp
    cos_x.o(i.__cos$lsc) refers to cos_x.o(i.____hardfp_cos$lsc) for ____hardfp_cos$lsc
    log10.o(i.__hardfp_log10) refers (Special) to iusefp.o(.text) for __I$use$fp
    log10.o(i.__hardfp_log10) refers to dunder.o(i.__mathlib_dbl_infnan) for __mathlib_dbl_infnan
    log10.o(i.__hardfp_log10) refers to errno.o(i.__set_errno) for __set_errno
    log10.o(i.__hardfp_log10) refers to dunder.o(i.__mathlib_dbl_invalid) for __mathlib_dbl_invalid
    log10.o(i.__hardfp_log10) refers to dunder.o(i.__mathlib_dbl_divzero) for __mathlib_dbl_divzero
    log10.o(i.__hardfp_log10) refers to dmul.o(.text) for __aeabi_dmul
    log10.o(i.__hardfp_log10) refers to dflti.o(.text) for __aeabi_i2d
    log10.o(i.__hardfp_log10) refers to log.o(i.log) for log
    log10.o(i.__hardfp_log10) refers to dadd.o(.text) for __aeabi_dadd
    log10.o(i.__softfp_log10) refers (Special) to iusefp.o(.text) for __I$use$fp
    log10.o(i.__softfp_log10) refers to log10.o(i.__hardfp_log10) for __hardfp_log10
    log10.o(i.log10) refers (Special) to iusefp.o(.text) for __I$use$fp
    log10.o(i.log10) refers to log10.o(i.__hardfp_log10) for __hardfp_log10
    log10_x.o(i.____hardfp_log10$lsc) refers (Special) to iusefp.o(.text) for __I$use$fp
    log10_x.o(i.____hardfp_log10$lsc) refers to dunder.o(i.__mathlib_dbl_infnan) for __mathlib_dbl_infnan
    log10_x.o(i.____hardfp_log10$lsc) refers to errno.o(i.__set_errno) for __set_errno
    log10_x.o(i.____hardfp_log10$lsc) refers to dmul.o(.text) for __aeabi_dmul
    log10_x.o(i.____hardfp_log10$lsc) refers to dflti.o(.text) for __aeabi_i2d
    log10_x.o(i.____hardfp_log10$lsc) refers to log.o(i.log) for log
    log10_x.o(i.____hardfp_log10$lsc) refers to dadd.o(.text) for __aeabi_dadd
    log10_x.o(i.____softfp_log10$lsc) refers (Special) to iusefp.o(.text) for __I$use$fp
    log10_x.o(i.____softfp_log10$lsc) refers to log10_x.o(i.____hardfp_log10$lsc) for ____hardfp_log10$lsc
    log10_x.o(i.__log10$lsc) refers (Special) to iusefp.o(.text) for __I$use$fp
    log10_x.o(i.__log10$lsc) refers to log10_x.o(i.____hardfp_log10$lsc) for ____hardfp_log10$lsc
    pow.o(i.__hardfp_pow) refers (Special) to iusefp.o(.text) for __I$use$fp
    pow.o(i.__hardfp_pow) refers to dunder.o(i.__mathlib_dbl_infnan2) for __mathlib_dbl_infnan2
    pow.o(i.__hardfp_pow) refers to errno.o(i.__set_errno) for __set_errno
    pow.o(i.__hardfp_pow) refers to dunder.o(i.__mathlib_dbl_divzero) for __mathlib_dbl_divzero
    pow.o(i.__hardfp_pow) refers to dunder.o(i.__mathlib_dbl_overflow) for __mathlib_dbl_overflow
    pow.o(i.__hardfp_pow) refers to ddiv.o(.text) for __aeabi_ddiv
    pow.o(i.__hardfp_pow) refers to sqrt.o(i.sqrt) for sqrt
    pow.o(i.__hardfp_pow) refers to fabs.o(i.fabs) for fabs
    pow.o(i.__hardfp_pow) refers to dflti.o(.text) for __aeabi_i2d
    pow.o(i.__hardfp_pow) refers to dunder.o(i.__mathlib_dbl_invalid) for __mathlib_dbl_invalid
    pow.o(i.__hardfp_pow) refers to dmul.o(.text) for __aeabi_dmul
    pow.o(i.__hardfp_pow) refers to dunder.o(i.__mathlib_dbl_underflow) for __mathlib_dbl_underflow
    pow.o(i.__hardfp_pow) refers to dadd.o(.text) for __aeabi_dsub
    pow.o(i.__hardfp_pow) refers to qnan.o(.constdata) for __mathlib_zero
    pow.o(i.__hardfp_pow) refers to poly.o(i.__kernel_poly) for __kernel_poly
    pow.o(i.__hardfp_pow) refers to pow.o(.constdata) for .constdata
    pow.o(i.__hardfp_pow) refers to cdrcmple.o(.text) for __aeabi_cdrcmple
    pow.o(i.__hardfp_pow) refers to dscalb.o(.text) for __ARM_scalbn
    pow.o(i.__hardfp_pow) refers to fpclassify.o(i.__ARM_fpclassify) for __ARM_fpclassify
    pow.o(i.__softfp_pow) refers (Special) to iusefp.o(.text) for __I$use$fp
    pow.o(i.__softfp_pow) refers to pow.o(i.__hardfp_pow) for __hardfp_pow
    pow.o(i.pow) refers (Special) to iusefp.o(.text) for __I$use$fp
    pow.o(i.pow) refers to pow.o(i.__hardfp_pow) for __hardfp_pow
    pow.o(.constdata) refers (Special) to iusefp.o(.text) for __I$use$fp
    pow_x.o(i.____hardfp_pow$lsc) refers (Special) to iusefp.o(.text) for __I$use$fp
    pow_x.o(i.____hardfp_pow$lsc) refers to dunder.o(i.__mathlib_dbl_infnan2) for __mathlib_dbl_infnan2
    pow_x.o(i.____hardfp_pow$lsc) refers to errno.o(i.__set_errno) for __set_errno
    pow_x.o(i.____hardfp_pow$lsc) refers to ddiv.o(.text) for __aeabi_ddiv
    pow_x.o(i.____hardfp_pow$lsc) refers to sqrt.o(i.sqrt) for sqrt
    pow_x.o(i.____hardfp_pow$lsc) refers to fabs.o(i.fabs) for fabs
    pow_x.o(i.____hardfp_pow$lsc) refers to dflti.o(.text) for __aeabi_i2d
    pow_x.o(i.____hardfp_pow$lsc) refers to dmul.o(.text) for __aeabi_dmul
    pow_x.o(i.____hardfp_pow$lsc) refers to dadd.o(.text) for __aeabi_dsub
    pow_x.o(i.____hardfp_pow$lsc) refers to qnan.o(.constdata) for __mathlib_zero
    pow_x.o(i.____hardfp_pow$lsc) refers to poly.o(i.__kernel_poly) for __kernel_poly
    pow_x.o(i.____hardfp_pow$lsc) refers to pow_x.o(.constdata) for .constdata
    pow_x.o(i.____hardfp_pow$lsc) refers to cdrcmple.o(.text) for __aeabi_cdrcmple
    pow_x.o(i.____hardfp_pow$lsc) refers to dscalb.o(.text) for __ARM_scalbn
    pow_x.o(i.____softfp_pow$lsc) refers (Special) to iusefp.o(.text) for __I$use$fp
    pow_x.o(i.____softfp_pow$lsc) refers to pow_x.o(i.____hardfp_pow$lsc) for ____hardfp_pow$lsc
    pow_x.o(i.__pow$lsc) refers (Special) to iusefp.o(.text) for __I$use$fp
    pow_x.o(i.__pow$lsc) refers to pow_x.o(i.____hardfp_pow$lsc) for ____hardfp_pow$lsc
    pow_x.o(.constdata) refers (Special) to iusefp.o(.text) for __I$use$fp
    sin.o(i.__hardfp_sin) refers (Special) to iusefp.o(.text) for __I$use$fp
    sin.o(i.__hardfp_sin) refers to errno.o(i.__set_errno) for __set_errno
    sin.o(i.__hardfp_sin) refers to dunder.o(i.__mathlib_dbl_invalid) for __mathlib_dbl_invalid
    sin.o(i.__hardfp_sin) refers to dunder.o(i.__mathlib_dbl_infnan) for __mathlib_dbl_infnan
    sin.o(i.__hardfp_sin) refers to rred.o(i.__ieee754_rem_pio2) for __ieee754_rem_pio2
    sin.o(i.__hardfp_sin) refers to cos_i.o(i.__kernel_cos) for __kernel_cos
    sin.o(i.__hardfp_sin) refers to sin_i.o(i.__kernel_sin) for __kernel_sin
    sin.o(i.__softfp_sin) refers (Special) to iusefp.o(.text) for __I$use$fp
    sin.o(i.__softfp_sin) refers to sin.o(i.__hardfp_sin) for __hardfp_sin
    sin.o(i.sin) refers (Special) to iusefp.o(.text) for __I$use$fp
    sin.o(i.sin) refers to sin.o(i.__hardfp_sin) for __hardfp_sin
    sin_x.o(i.____hardfp_sin$lsc) refers (Special) to iusefp.o(.text) for __I$use$fp
    sin_x.o(i.____hardfp_sin$lsc) refers to errno.o(i.__set_errno) for __set_errno
    sin_x.o(i.____hardfp_sin$lsc) refers to dunder.o(i.__mathlib_dbl_infnan) for __mathlib_dbl_infnan
    sin_x.o(i.____hardfp_sin$lsc) refers to rred.o(i.__ieee754_rem_pio2) for __ieee754_rem_pio2
    sin_x.o(i.____hardfp_sin$lsc) refers to cos_i.o(i.__kernel_cos) for __kernel_cos
    sin_x.o(i.____hardfp_sin$lsc) refers to sin_i.o(i.__kernel_sin) for __kernel_sin
    sin_x.o(i.____softfp_sin$lsc) refers (Special) to iusefp.o(.text) for __I$use$fp
    sin_x.o(i.____softfp_sin$lsc) refers to sin_x.o(i.____hardfp_sin$lsc) for ____hardfp_sin$lsc
    sin_x.o(i.__sin$lsc) refers (Special) to iusefp.o(.text) for __I$use$fp
    sin_x.o(i.__sin$lsc) refers to sin_x.o(i.____hardfp_sin$lsc) for ____hardfp_sin$lsc
    entry.o(.ARM.Collect$$$$00000000) refers (Special) to entry10a.o(.ARM.Collect$$$$0000000F) for __rt_final_cpp
    entry.o(.ARM.Collect$$$$00000000) refers (Special) to entry11a.o(.ARM.Collect$$$$00000011) for __rt_final_exit
    entry.o(.ARM.Collect$$$$00000000) refers (Special) to entry12b.o(.ARM.Collect$$$$0000000E) for __rt_lib_shutdown_fini
    entry.o(.ARM.Collect$$$$00000000) refers (Special) to entry7b.o(.ARM.Collect$$$$00000008) for _main_clock
    entry.o(.ARM.Collect$$$$00000000) refers (Special) to entry8b.o(.ARM.Collect$$$$0000000A) for _main_cpp_init
    entry.o(.ARM.Collect$$$$00000000) refers (Special) to entry9a.o(.ARM.Collect$$$$0000000B) for _main_init
    entry.o(.ARM.Collect$$$$00000000) refers (Special) to entry5.o(.ARM.Collect$$$$00000004) for _main_scatterload
    entry.o(.ARM.Collect$$$$00000000) refers (Special) to entry2.o(.ARM.Collect$$$$00000001) for _main_stk
    ldiv.o(.text) refers to uldiv.o(.text) for __aeabi_uldivmod
    printfb.o(i.__0fprintf$bare) refers to printfb.o(i._printf_core) for _printf_core
    printfb.o(i.__0fprintf$bare) refers to fputc.o(i.fputc) for fputc
    printfb.o(i.__0printf$bare) refers to printfb.o(i._printf_core) for _printf_core
    printfb.o(i.__0printf$bare) refers to fputc.o(i.fputc) for fputc
    printfb.o(i.__0printf$bare) refers to stdout.o(.data) for __stdout
    printfb.o(i.__0snprintf$bare) refers to printfb.o(i._printf_core) for _printf_core
    printfb.o(i.__0snprintf$bare) refers to printfb.o(i._snputc) for _snputc
    printfb.o(i.__0sprintf$bare) refers to printfb.o(i._printf_core) for _printf_core
    printfb.o(i.__0sprintf$bare) refers to printfb.o(i._sputc) for _sputc
    printfb.o(i.__0vfprintf$bare) refers to printfb.o(i._printf_core) for _printf_core
    printfb.o(i.__0vfprintf$bare) refers to fputc.o(i.fputc) for fputc
    printfb.o(i.__0vprintf$bare) refers to printfb.o(i._printf_core) for _printf_core
    printfb.o(i.__0vprintf$bare) refers to fputc.o(i.fputc) for fputc
    printfb.o(i.__0vprintf$bare) refers to stdout.o(.data) for __stdout
    printfb.o(i.__0vsnprintf$bare) refers to printfb.o(i._printf_core) for _printf_core
    printfb.o(i.__0vsnprintf$bare) refers to printfb.o(i._snputc) for _snputc
    printfb.o(i.__0vsprintf$bare) refers to printfb.o(i._printf_core) for _printf_core
    printfb.o(i.__0vsprintf$bare) refers to printfb.o(i._sputc) for _sputc
    printf0.o(i.__0fprintf$0) refers to printf0.o(i._printf_core) for _printf_core
    printf0.o(i.__0fprintf$0) refers to fputc.o(i.fputc) for fputc
    printf0.o(i.__0printf$0) refers to printf0.o(i._printf_core) for _printf_core
    printf0.o(i.__0printf$0) refers to fputc.o(i.fputc) for fputc
    printf0.o(i.__0printf$0) refers to stdout.o(.data) for __stdout
    printf0.o(i.__0snprintf$0) refers to printf0.o(i._printf_core) for _printf_core
    printf0.o(i.__0snprintf$0) refers to printf0.o(i._snputc) for _snputc
    printf0.o(i.__0sprintf$0) refers to printf0.o(i._printf_core) for _printf_core
    printf0.o(i.__0sprintf$0) refers to printf0.o(i._sputc) for _sputc
    printf0.o(i.__0vfprintf$0) refers to printf0.o(i._printf_core) for _printf_core
    printf0.o(i.__0vfprintf$0) refers to fputc.o(i.fputc) for fputc
    printf0.o(i.__0vprintf$0) refers to printf0.o(i._printf_core) for _printf_core
    printf0.o(i.__0vprintf$0) refers to fputc.o(i.fputc) for fputc
    printf0.o(i.__0vprintf$0) refers to stdout.o(.data) for __stdout
    printf0.o(i.__0vsnprintf$0) refers to printf0.o(i._printf_core) for _printf_core
    printf0.o(i.__0vsnprintf$0) refers to printf0.o(i._snputc) for _snputc
    printf0.o(i.__0vsprintf$0) refers to printf0.o(i._printf_core) for _printf_core
    printf0.o(i.__0vsprintf$0) refers to printf0.o(i._sputc) for _sputc
    printf1.o(i.__0fprintf$1) refers to printf1.o(i._printf_core) for _printf_core
    printf1.o(i.__0fprintf$1) refers to fputc.o(i.fputc) for fputc
    printf1.o(i.__0printf$1) refers to printf1.o(i._printf_core) for _printf_core
    printf1.o(i.__0printf$1) refers to fputc.o(i.fputc) for fputc
    printf1.o(i.__0printf$1) refers to stdout.o(.data) for __stdout
    printf1.o(i.__0snprintf$1) refers to printf1.o(i._printf_core) for _printf_core
    printf1.o(i.__0snprintf$1) refers to printf1.o(i._snputc) for _snputc
    printf1.o(i.__0sprintf$1) refers to printf1.o(i._printf_core) for _printf_core
    printf1.o(i.__0sprintf$1) refers to printf1.o(i._sputc) for _sputc
    printf1.o(i.__0vfprintf$1) refers to printf1.o(i._printf_core) for _printf_core
    printf1.o(i.__0vfprintf$1) refers to fputc.o(i.fputc) for fputc
    printf1.o(i.__0vprintf$1) refers to printf1.o(i._printf_core) for _printf_core
    printf1.o(i.__0vprintf$1) refers to fputc.o(i.fputc) for fputc
    printf1.o(i.__0vprintf$1) refers to stdout.o(.data) for __stdout
    printf1.o(i.__0vsnprintf$1) refers to printf1.o(i._printf_core) for _printf_core
    printf1.o(i.__0vsnprintf$1) refers to printf1.o(i._snputc) for _snputc
    printf1.o(i.__0vsprintf$1) refers to printf1.o(i._printf_core) for _printf_core
    printf1.o(i.__0vsprintf$1) refers to printf1.o(i._sputc) for _sputc
    printf1.o(i._printf_core) refers to uidiv.o(.text) for __aeabi_uidivmod
    printf2.o(i.__0fprintf$2) refers to printf2.o(i._printf_core) for _printf_core
    printf2.o(i.__0fprintf$2) refers to fputc.o(i.fputc) for fputc
    printf2.o(i.__0printf$2) refers to printf2.o(i._printf_core) for _printf_core
    printf2.o(i.__0printf$2) refers to fputc.o(i.fputc) for fputc
    printf2.o(i.__0printf$2) refers to stdout.o(.data) for __stdout
    printf2.o(i.__0snprintf$2) refers to printf2.o(i._printf_core) for _printf_core
    printf2.o(i.__0snprintf$2) refers to printf2.o(i._snputc) for _snputc
    printf2.o(i.__0sprintf$2) refers to printf2.o(i._printf_core) for _printf_core
    printf2.o(i.__0sprintf$2) refers to printf2.o(i._sputc) for _sputc
    printf2.o(i.__0vfprintf$2) refers to printf2.o(i._printf_core) for _printf_core
    printf2.o(i.__0vfprintf$2) refers to fputc.o(i.fputc) for fputc
    printf2.o(i.__0vprintf$2) refers to printf2.o(i._printf_core) for _printf_core
    printf2.o(i.__0vprintf$2) refers to fputc.o(i.fputc) for fputc
    printf2.o(i.__0vprintf$2) refers to stdout.o(.data) for __stdout
    printf2.o(i.__0vsnprintf$2) refers to printf2.o(i._printf_core) for _printf_core
    printf2.o(i.__0vsnprintf$2) refers to printf2.o(i._snputc) for _snputc
    printf2.o(i.__0vsprintf$2) refers to printf2.o(i._printf_core) for _printf_core
    printf2.o(i.__0vsprintf$2) refers to printf2.o(i._sputc) for _sputc
    printf3.o(i.__0fprintf$3) refers to printf3.o(i._printf_core) for _printf_core
    printf3.o(i.__0fprintf$3) refers to fputc.o(i.fputc) for fputc
    printf3.o(i.__0printf$3) refers to printf3.o(i._printf_core) for _printf_core
    printf3.o(i.__0printf$3) refers to fputc.o(i.fputc) for fputc
    printf3.o(i.__0printf$3) refers to stdout.o(.data) for __stdout
    printf3.o(i.__0snprintf$3) refers to printf3.o(i._printf_core) for _printf_core
    printf3.o(i.__0snprintf$3) refers to printf3.o(i._snputc) for _snputc
    printf3.o(i.__0sprintf$3) refers to printf3.o(i._printf_core) for _printf_core
    printf3.o(i.__0sprintf$3) refers to printf3.o(i._sputc) for _sputc
    printf3.o(i.__0vfprintf$3) refers to printf3.o(i._printf_core) for _printf_core
    printf3.o(i.__0vfprintf$3) refers to fputc.o(i.fputc) for fputc
    printf3.o(i.__0vprintf$3) refers to printf3.o(i._printf_core) for _printf_core
    printf3.o(i.__0vprintf$3) refers to fputc.o(i.fputc) for fputc
    printf3.o(i.__0vprintf$3) refers to stdout.o(.data) for __stdout
    printf3.o(i.__0vsnprintf$3) refers to printf3.o(i._printf_core) for _printf_core
    printf3.o(i.__0vsnprintf$3) refers to printf3.o(i._snputc) for _snputc
    printf3.o(i.__0vsprintf$3) refers to printf3.o(i._printf_core) for _printf_core
    printf3.o(i.__0vsprintf$3) refers to printf3.o(i._sputc) for _sputc
    printf3.o(i._printf_core) refers to uidiv.o(.text) for __aeabi_uidivmod
    printf4.o(i.__0fprintf$4) refers to printf4.o(i._printf_core) for _printf_core
    printf4.o(i.__0fprintf$4) refers to fputc.o(i.fputc) for fputc
    printf4.o(i.__0printf$4) refers to printf4.o(i._printf_core) for _printf_core
    printf4.o(i.__0printf$4) refers to fputc.o(i.fputc) for fputc
    printf4.o(i.__0printf$4) refers to stdout.o(.data) for __stdout
    printf4.o(i.__0snprintf$4) refers to printf4.o(i._printf_core) for _printf_core
    printf4.o(i.__0snprintf$4) refers to printf4.o(i._snputc) for _snputc
    printf4.o(i.__0sprintf$4) refers to printf4.o(i._printf_core) for _printf_core
    printf4.o(i.__0sprintf$4) refers to printf4.o(i._sputc) for _sputc
    printf4.o(i.__0vfprintf$4) refers to printf4.o(i._printf_core) for _printf_core
    printf4.o(i.__0vfprintf$4) refers to fputc.o(i.fputc) for fputc
    printf4.o(i.__0vprintf$4) refers to printf4.o(i._printf_core) for _printf_core
    printf4.o(i.__0vprintf$4) refers to fputc.o(i.fputc) for fputc
    printf4.o(i.__0vprintf$4) refers to stdout.o(.data) for __stdout
    printf4.o(i.__0vsnprintf$4) refers to printf4.o(i._printf_core) for _printf_core
    printf4.o(i.__0vsnprintf$4) refers to printf4.o(i._snputc) for _snputc
    printf4.o(i.__0vsprintf$4) refers to printf4.o(i._printf_core) for _printf_core
    printf4.o(i.__0vsprintf$4) refers to printf4.o(i._sputc) for _sputc
    printf4.o(i._printf_core) refers to uldiv.o(.text) for __aeabi_uldivmod
    printf5.o(i.__0fprintf$5) refers to printf5.o(i._printf_core) for _printf_core
    printf5.o(i.__0fprintf$5) refers to fputc.o(i.fputc) for fputc
    printf5.o(i.__0printf$5) refers to printf5.o(i._printf_core) for _printf_core
    printf5.o(i.__0printf$5) refers to fputc.o(i.fputc) for fputc
    printf5.o(i.__0printf$5) refers to stdout.o(.data) for __stdout
    printf5.o(i.__0snprintf$5) refers to printf5.o(i._printf_core) for _printf_core
    printf5.o(i.__0snprintf$5) refers to printf5.o(i._snputc) for _snputc
    printf5.o(i.__0sprintf$5) refers to printf5.o(i._printf_core) for _printf_core
    printf5.o(i.__0sprintf$5) refers to printf5.o(i._sputc) for _sputc
    printf5.o(i.__0vfprintf$5) refers to printf5.o(i._printf_core) for _printf_core
    printf5.o(i.__0vfprintf$5) refers to fputc.o(i.fputc) for fputc
    printf5.o(i.__0vprintf$5) refers to printf5.o(i._printf_core) for _printf_core
    printf5.o(i.__0vprintf$5) refers to fputc.o(i.fputc) for fputc
    printf5.o(i.__0vprintf$5) refers to stdout.o(.data) for __stdout
    printf5.o(i.__0vsnprintf$5) refers to printf5.o(i._printf_core) for _printf_core
    printf5.o(i.__0vsnprintf$5) refers to printf5.o(i._snputc) for _snputc
    printf5.o(i.__0vsprintf$5) refers to printf5.o(i._printf_core) for _printf_core
    printf5.o(i.__0vsprintf$5) refers to printf5.o(i._sputc) for _sputc
    printf5.o(i._printf_core) refers to uldiv.o(.text) for __aeabi_uldivmod
    printf6.o(i.__0fprintf$6) refers to printf6.o(i._printf_core) for _printf_core
    printf6.o(i.__0fprintf$6) refers to fputc.o(i.fputc) for fputc
    printf6.o(i.__0printf$6) refers to printf6.o(i._printf_core) for _printf_core
    printf6.o(i.__0printf$6) refers to fputc.o(i.fputc) for fputc
    printf6.o(i.__0printf$6) refers to stdout.o(.data) for __stdout
    printf6.o(i.__0snprintf$6) refers to printf6.o(i._printf_core) for _printf_core
    printf6.o(i.__0snprintf$6) refers to printf6.o(i._snputc) for _snputc
    printf6.o(i.__0sprintf$6) refers to printf6.o(i._printf_core) for _printf_core
    printf6.o(i.__0sprintf$6) refers to printf6.o(i._sputc) for _sputc
    printf6.o(i.__0vfprintf$6) refers to printf6.o(i._printf_core) for _printf_core
    printf6.o(i.__0vfprintf$6) refers to fputc.o(i.fputc) for fputc
    printf6.o(i.__0vprintf$6) refers to printf6.o(i._printf_core) for _printf_core
    printf6.o(i.__0vprintf$6) refers to fputc.o(i.fputc) for fputc
    printf6.o(i.__0vprintf$6) refers to stdout.o(.data) for __stdout
    printf6.o(i.__0vsnprintf$6) refers to printf6.o(i._printf_core) for _printf_core
    printf6.o(i.__0vsnprintf$6) refers to printf6.o(i._snputc) for _snputc
    printf6.o(i.__0vsprintf$6) refers to printf6.o(i._printf_core) for _printf_core
    printf6.o(i.__0vsprintf$6) refers to printf6.o(i._sputc) for _sputc
    printf6.o(i._printf_core) refers to printf6.o(i._printf_pre_padding) for _printf_pre_padding
    printf6.o(i._printf_core) refers to uidiv.o(.text) for __aeabi_uidivmod
    printf6.o(i._printf_core) refers to printf6.o(i._printf_post_padding) for _printf_post_padding
    printf7.o(i.__0fprintf$7) refers to printf7.o(i._printf_core) for _printf_core
    printf7.o(i.__0fprintf$7) refers to fputc.o(i.fputc) for fputc
    printf7.o(i.__0printf$7) refers to printf7.o(i._printf_core) for _printf_core
    printf7.o(i.__0printf$7) refers to fputc.o(i.fputc) for fputc
    printf7.o(i.__0printf$7) refers to stdout.o(.data) for __stdout
    printf7.o(i.__0snprintf$7) refers to printf7.o(i._printf_core) for _printf_core
    printf7.o(i.__0snprintf$7) refers to printf7.o(i._snputc) for _snputc
    printf7.o(i.__0sprintf$7) refers to printf7.o(i._printf_core) for _printf_core
    printf7.o(i.__0sprintf$7) refers to printf7.o(i._sputc) for _sputc
    printf7.o(i.__0vfprintf$7) refers to printf7.o(i._printf_core) for _printf_core
    printf7.o(i.__0vfprintf$7) refers to fputc.o(i.fputc) for fputc
    printf7.o(i.__0vprintf$7) refers to printf7.o(i._printf_core) for _printf_core
    printf7.o(i.__0vprintf$7) refers to fputc.o(i.fputc) for fputc
    printf7.o(i.__0vprintf$7) refers to stdout.o(.data) for __stdout
    printf7.o(i.__0vsnprintf$7) refers to printf7.o(i._printf_core) for _printf_core
    printf7.o(i.__0vsnprintf$7) refers to printf7.o(i._snputc) for _snputc
    printf7.o(i.__0vsprintf$7) refers to printf7.o(i._printf_core) for _printf_core
    printf7.o(i.__0vsprintf$7) refers to printf7.o(i._sputc) for _sputc
    printf7.o(i._printf_core) refers to printf7.o(i._printf_pre_padding) for _printf_pre_padding
    printf7.o(i._printf_core) refers to uldiv.o(.text) for __aeabi_uldivmod
    printf7.o(i._printf_core) refers to printf7.o(i._printf_post_padding) for _printf_post_padding
    printf8.o(i.__0fprintf$8) refers to printf8.o(i._printf_core) for _printf_core
    printf8.o(i.__0fprintf$8) refers to fputc.o(i.fputc) for fputc
    printf8.o(i.__0printf$8) refers to printf8.o(i._printf_core) for _printf_core
    printf8.o(i.__0printf$8) refers to fputc.o(i.fputc) for fputc
    printf8.o(i.__0printf$8) refers to stdout.o(.data) for __stdout
    printf8.o(i.__0snprintf$8) refers to printf8.o(i._printf_core) for _printf_core
    printf8.o(i.__0snprintf$8) refers to printf8.o(i._snputc) for _snputc
    printf8.o(i.__0sprintf$8) refers to printf8.o(i._printf_core) for _printf_core
    printf8.o(i.__0sprintf$8) refers to printf8.o(i._sputc) for _sputc
    printf8.o(i.__0vfprintf$8) refers to printf8.o(i._printf_core) for _printf_core
    printf8.o(i.__0vfprintf$8) refers to fputc.o(i.fputc) for fputc
    printf8.o(i.__0vprintf$8) refers to printf8.o(i._printf_core) for _printf_core
    printf8.o(i.__0vprintf$8) refers to fputc.o(i.fputc) for fputc
    printf8.o(i.__0vprintf$8) refers to stdout.o(.data) for __stdout
    printf8.o(i.__0vsnprintf$8) refers to printf8.o(i._printf_core) for _printf_core
    printf8.o(i.__0vsnprintf$8) refers to printf8.o(i._snputc) for _snputc
    printf8.o(i.__0vsprintf$8) refers to printf8.o(i._printf_core) for _printf_core
    printf8.o(i.__0vsprintf$8) refers to printf8.o(i._sputc) for _sputc
    printf8.o(i._printf_core) refers to printf8.o(i._printf_pre_padding) for _printf_pre_padding
    printf8.o(i._printf_core) refers to uldiv.o(.text) for __aeabi_uldivmod
    printf8.o(i._printf_core) refers to printf8.o(i._printf_post_padding) for _printf_post_padding
    printfa.o(i.__0fprintf) refers (Special) to iusefp.o(.text) for __I$use$fp
    printfa.o(i.__0fprintf) refers to printfa.o(i._printf_core) for _printf_core
    printfa.o(i.__0fprintf) refers to fputc.o(i.fputc) for fputc
    printfa.o(i.__0printf) refers (Special) to iusefp.o(.text) for __I$use$fp
    printfa.o(i.__0printf) refers to printfa.o(i._printf_core) for _printf_core
    printfa.o(i.__0printf) refers to fputc.o(i.fputc) for fputc
    printfa.o(i.__0printf) refers to stdout.o(.data) for __stdout
    printfa.o(i.__0snprintf) refers (Special) to iusefp.o(.text) for __I$use$fp
    printfa.o(i.__0snprintf) refers to printfa.o(i._printf_core) for _printf_core
    printfa.o(i.__0snprintf) refers to printfa.o(i._snputc) for _snputc
    printfa.o(i.__0sprintf) refers (Special) to iusefp.o(.text) for __I$use$fp
    printfa.o(i.__0sprintf) refers to printfa.o(i._printf_core) for _printf_core
    printfa.o(i.__0sprintf) refers to printfa.o(i._sputc) for _sputc
    printfa.o(i.__0vfprintf) refers (Special) to iusefp.o(.text) for __I$use$fp
    printfa.o(i.__0vfprintf) refers to printfa.o(i._printf_core) for _printf_core
    printfa.o(i.__0vfprintf) refers to fputc.o(i.fputc) for fputc
    printfa.o(i.__0vprintf) refers (Special) to iusefp.o(.text) for __I$use$fp
    printfa.o(i.__0vprintf) refers to printfa.o(i._printf_core) for _printf_core
    printfa.o(i.__0vprintf) refers to fputc.o(i.fputc) for fputc
    printfa.o(i.__0vprintf) refers to stdout.o(.data) for __stdout
    printfa.o(i.__0vsnprintf) refers (Special) to iusefp.o(.text) for __I$use$fp
    printfa.o(i.__0vsnprintf) refers to printfa.o(i._printf_core) for _printf_core
    printfa.o(i.__0vsnprintf) refers to printfa.o(i._snputc) for _snputc
    printfa.o(i.__0vsprintf) refers (Special) to iusefp.o(.text) for __I$use$fp
    printfa.o(i.__0vsprintf) refers to printfa.o(i._printf_core) for _printf_core
    printfa.o(i.__0vsprintf) refers to printfa.o(i._sputc) for _sputc
    printfa.o(i._fp_digits) refers (Special) to iusefp.o(.text) for __I$use$fp
    printfa.o(i._fp_digits) refers to dmul.o(.text) for __aeabi_dmul
    printfa.o(i._fp_digits) refers to ddiv.o(.text) for __aeabi_ddiv
    printfa.o(i._fp_digits) refers to cdrcmple.o(.text) for __aeabi_cdrcmple
    printfa.o(i._fp_digits) refers to dadd.o(.text) for __aeabi_dadd
    printfa.o(i._fp_digits) refers to dfixul.o(.text) for __aeabi_d2ulz
    printfa.o(i._fp_digits) refers to uldiv.o(.text) for __aeabi_uldivmod
    printfa.o(i._printf_core) refers (Special) to iusefp.o(.text) for __I$use$fp
    printfa.o(i._printf_core) refers to printfa.o(i._printf_pre_padding) for _printf_pre_padding
    printfa.o(i._printf_core) refers to uldiv.o(.text) for __aeabi_uldivmod
    printfa.o(i._printf_core) refers to printfa.o(i._printf_post_padding) for _printf_post_padding
    printfa.o(i._printf_core) refers to printfa.o(i._fp_digits) for _fp_digits
    printfa.o(i._printf_core) refers to uidiv.o(.text) for __aeabi_uidivmod
    printfa.o(i._printf_post_padding) refers (Special) to iusefp.o(.text) for __I$use$fp
    printfa.o(i._printf_pre_padding) refers (Special) to iusefp.o(.text) for __I$use$fp
    printfa.o(i._snputc) refers (Special) to iusefp.o(.text) for __I$use$fp
    printfa.o(i._sputc) refers (Special) to iusefp.o(.text) for __I$use$fp
    dadd.o(.text) refers (Special) to iusefp.o(.text) for __I$use$fp
    dadd.o(.text) refers to llshl.o(.text) for __aeabi_llsl
    dadd.o(.text) refers to llsshr.o(.text) for __aeabi_lasr
    dadd.o(.text) refers to depilogue.o(.text) for _double_epilogue
    dmul.o(.text) refers (Special) to iusefp.o(.text) for __I$use$fp
    dmul.o(.text) refers to depilogue.o(.text) for _double_epilogue
    ddiv.o(.text) refers (Special) to iusefp.o(.text) for __I$use$fp
    ddiv.o(.text) refers to depilogue.o(.text) for _double_round
    ffltl.o(.text) refers (Special) to iusefp.o(.text) for __I$use$fp
    ffltl.o(.text) refers to fepilogue.o(.text) for _float_epilogue
    dflti.o(.text) refers (Special) to iusefp.o(.text) for __I$use$fp
    dflti.o(.text) refers to depilogue.o(.text) for _double_epilogue
    dfltui.o(.text) refers (Special) to iusefp.o(.text) for __I$use$fp
    dfltui.o(.text) refers to depilogue.o(.text) for _double_epilogue
    dfltl.o(.text) refers (Special) to iusefp.o(.text) for __I$use$fp
    dfltl.o(.text) refers to depilogue.o(.text) for _double_epilogue
    ffixl.o(.text) refers (Special) to iusefp.o(.text) for __I$use$fp
    ffixl.o(.text) refers to llshl.o(.text) for __aeabi_llsl
    dfixi.o(.text) refers (Special) to iusefp.o(.text) for __I$use$fp
    dfixi.o(.text) refers to llushr.o(.text) for __aeabi_llsr
    dfixl.o(.text) refers (Special) to iusefp.o(.text) for __I$use$fp
    dfixl.o(.text) refers to llushr.o(.text) for __aeabi_llsr
    dfixl.o(.text) refers to llshl.o(.text) for __aeabi_llsl
    f2d.o(.text) refers (Special) to iusefp.o(.text) for __I$use$fp
    d2f.o(.text) refers (Special) to iusefp.o(.text) for __I$use$fp
    d2f.o(.text) refers to fepilogue.o(.text) for _float_round
    cos_i.o(i.__kernel_cos) refers (Special) to iusefp.o(.text) for __I$use$fp
    cos_i.o(i.__kernel_cos) refers to dfixi.o(.text) for __aeabi_d2iz
    cos_i.o(i.__kernel_cos) refers to dmul.o(.text) for __aeabi_dmul
    cos_i.o(i.__kernel_cos) refers to poly.o(i.__kernel_poly) for __kernel_poly
    cos_i.o(i.__kernel_cos) refers to dadd.o(.text) for __aeabi_dsub
    cos_i.o(i.__kernel_cos) refers to cos_i.o(.constdata) for .constdata
    cos_i.o(.constdata) refers (Special) to iusefp.o(.text) for __I$use$fp
    dunder.o(i.__mathlib_dbl_divzero) refers to ddiv.o(.text) for __aeabi_ddiv
    dunder.o(i.__mathlib_dbl_infnan) refers to dadd.o(.text) for __aeabi_dadd
    dunder.o(i.__mathlib_dbl_infnan2) refers to dadd.o(.text) for __aeabi_dadd
    dunder.o(i.__mathlib_dbl_invalid) refers to ddiv.o(.text) for __aeabi_ddiv
    dunder.o(i.__mathlib_dbl_overflow) refers to dmul.o(.text) for __aeabi_dmul
    dunder.o(i.__mathlib_dbl_posinfnan) refers to dmul.o(.text) for __aeabi_dmul
    dunder.o(i.__mathlib_dbl_underflow) refers to dmul.o(.text) for __aeabi_dmul
    fabs.o(i.__hardfp_fabs) refers (Special) to iusefp.o(.text) for __I$use$fp
    fabs.o(i.__softfp_fabs) refers (Special) to iusefp.o(.text) for __I$use$fp
    fabs.o(i.fabs) refers (Special) to iusefp.o(.text) for __I$use$fp
    fpclassify.o(i.__ARM_fpclassify) refers (Special) to iusefp.o(.text) for __I$use$fp
    log.o(i.__hardfp_log) refers (Special) to iusefp.o(.text) for __I$use$fp
    log.o(i.__hardfp_log) refers to dunder.o(i.__mathlib_dbl_infnan) for __mathlib_dbl_infnan
    log.o(i.__hardfp_log) refers to errno.o(i.__set_errno) for __set_errno
    log.o(i.__hardfp_log) refers to dunder.o(i.__mathlib_dbl_invalid) for __mathlib_dbl_invalid
    log.o(i.__hardfp_log) refers to dunder.o(i.__mathlib_dbl_divzero) for __mathlib_dbl_divzero
    log.o(i.__hardfp_log) refers to dmul.o(.text) for __aeabi_dmul
    log.o(i.__hardfp_log) refers to dadd.o(.text) for __aeabi_dsub
    log.o(i.__hardfp_log) refers to cdcmple.o(.text) for __aeabi_cdcmpeq
    log.o(i.__hardfp_log) refers to dflti.o(.text) for __aeabi_i2d
    log.o(i.__hardfp_log) refers to ddiv.o(.text) for __aeabi_ddiv
    log.o(i.__hardfp_log) refers to poly.o(i.__kernel_poly) for __kernel_poly
    log.o(i.__hardfp_log) refers to qnan.o(.constdata) for __mathlib_zero
    log.o(i.__hardfp_log) refers to log.o(.constdata) for .constdata
    log.o(i.__softfp_log) refers (Special) to iusefp.o(.text) for __I$use$fp
    log.o(i.__softfp_log) refers to log.o(i.__hardfp_log) for __hardfp_log
    log.o(i.log) refers (Special) to iusefp.o(.text) for __I$use$fp
    log.o(i.log) refers to log.o(i.__hardfp_log) for __hardfp_log
    log.o(.constdata) refers (Special) to iusefp.o(.text) for __I$use$fp
    log_x.o(i.____hardfp_log$lsc) refers (Special) to iusefp.o(.text) for __I$use$fp
    log_x.o(i.____hardfp_log$lsc) refers to dunder.o(i.__mathlib_dbl_infnan) for __mathlib_dbl_infnan
    log_x.o(i.____hardfp_log$lsc) refers to errno.o(i.__set_errno) for __set_errno
    log_x.o(i.____hardfp_log$lsc) refers to dmul.o(.text) for __aeabi_dmul
    log_x.o(i.____hardfp_log$lsc) refers to dadd.o(.text) for __aeabi_dsub
    log_x.o(i.____hardfp_log$lsc) refers to cdcmple.o(.text) for __aeabi_cdcmpeq
    log_x.o(i.____hardfp_log$lsc) refers to dflti.o(.text) for __aeabi_i2d
    log_x.o(i.____hardfp_log$lsc) refers to ddiv.o(.text) for __aeabi_ddiv
    log_x.o(i.____hardfp_log$lsc) refers to poly.o(i.__kernel_poly) for __kernel_poly
    log_x.o(i.____hardfp_log$lsc) refers to qnan.o(.constdata) for __mathlib_zero
    log_x.o(i.____hardfp_log$lsc) refers to log_x.o(.constdata) for .constdata
    log_x.o(i.____softfp_log$lsc) refers (Special) to iusefp.o(.text) for __I$use$fp
    log_x.o(i.____softfp_log$lsc) refers to log_x.o(i.____hardfp_log$lsc) for ____hardfp_log$lsc
    log_x.o(i.__log$lsc) refers (Special) to iusefp.o(.text) for __I$use$fp
    log_x.o(i.__log$lsc) refers to log_x.o(i.____hardfp_log$lsc) for ____hardfp_log$lsc
    log_x.o(.constdata) refers (Special) to iusefp.o(.text) for __I$use$fp
    poly.o(i.__kernel_poly) refers (Special) to iusefp.o(.text) for __I$use$fp
    poly.o(i.__kernel_poly) refers to dmul.o(.text) for __aeabi_dmul
    poly.o(i.__kernel_poly) refers to dadd.o(.text) for __aeabi_dadd
    qnan.o(.constdata) refers (Special) to iusefp.o(.text) for __I$use$fp
    rred.o(i.__ieee754_rem_pio2) refers (Special) to iusefp.o(.text) for __I$use$fp
    rred.o(i.__ieee754_rem_pio2) refers to dadd.o(.text) for __aeabi_dsub
    rred.o(i.__ieee754_rem_pio2) refers to fabs.o(i.fabs) for fabs
    rred.o(i.__ieee754_rem_pio2) refers to dmul.o(.text) for __aeabi_dmul
    rred.o(i.__ieee754_rem_pio2) refers to dfixi.o(.text) for __aeabi_d2iz
    rred.o(i.__ieee754_rem_pio2) refers to dflti.o(.text) for __aeabi_i2d
    rred.o(i.__ieee754_rem_pio2) refers to dfltui.o(.text) for __aeabi_ui2d
    rred.o(i.__ieee754_rem_pio2) refers to rred.o(.constdata) for .constdata
    rred.o(i.__use_accurate_range_reduction) refers (Special) to iusefp.o(.text) for __I$use$fp
    rred.o(.constdata) refers (Special) to iusefp.o(.text) for __I$use$fp
    sin_i.o(i.__kernel_sin) refers (Special) to iusefp.o(.text) for __I$use$fp
    sin_i.o(i.__kernel_sin) refers to fpclassify.o(i.__ARM_fpclassify) for __ARM_fpclassify
    sin_i.o(i.__kernel_sin) refers to dunder.o(i.__mathlib_dbl_underflow) for __mathlib_dbl_underflow
    sin_i.o(i.__kernel_sin) refers to dmul.o(.text) for __aeabi_dmul
    sin_i.o(i.__kernel_sin) refers to poly.o(i.__kernel_poly) for __kernel_poly
    sin_i.o(i.__kernel_sin) refers to dadd.o(.text) for __aeabi_dsub
    sin_i.o(i.__kernel_sin) refers to sin_i.o(.constdata) for .constdata
    sin_i.o(.constdata) refers (Special) to iusefp.o(.text) for __I$use$fp
    sin_i_x.o(i.____kernel_sin$lsc) refers (Special) to iusefp.o(.text) for __I$use$fp
    sin_i_x.o(i.____kernel_sin$lsc) refers to dmul.o(.text) for __aeabi_dmul
    sin_i_x.o(i.____kernel_sin$lsc) refers to poly.o(i.__kernel_poly) for __kernel_poly
    sin_i_x.o(i.____kernel_sin$lsc) refers to dadd.o(.text) for __aeabi_dsub
    sin_i_x.o(i.____kernel_sin$lsc) refers to sin_i_x.o(.constdata) for .constdata
    sin_i_x.o(.constdata) refers (Special) to iusefp.o(.text) for __I$use$fp
    sqrt.o(i.__hardfp_sqrt) refers (Special) to iusefp.o(.text) for __I$use$fp
    sqrt.o(i.__hardfp_sqrt) refers to dsqrt.o(.text) for _dsqrt
    sqrt.o(i.__hardfp_sqrt) refers to errno.o(i.__set_errno) for __set_errno
    sqrt.o(i.__softfp_sqrt) refers (Special) to iusefp.o(.text) for __I$use$fp
    sqrt.o(i.__softfp_sqrt) refers to dsqrt.o(.text) for _dsqrt
    sqrt.o(i.__softfp_sqrt) refers to errno.o(i.__set_errno) for __set_errno
    sqrt.o(i.sqrt) refers (Special) to iusefp.o(.text) for __I$use$fp
    sqrt.o(i.sqrt) refers to dsqrt.o(.text) for _dsqrt
    sqrt.o(i.sqrt) refers to errno.o(i.__set_errno) for __set_errno
    sqrt_x.o(i.____hardfp_sqrt$lsc) refers (Special) to iusefp.o(.text) for __I$use$fp
    sqrt_x.o(i.____hardfp_sqrt$lsc) refers to cdcmple.o(.text) for __aeabi_cdcmple
    sqrt_x.o(i.____hardfp_sqrt$lsc) refers to errno.o(i.__set_errno) for __set_errno
    sqrt_x.o(i.____hardfp_sqrt$lsc) refers to dsqrt.o(.text) for _dsqrt
    sqrt_x.o(i.____softfp_sqrt$lsc) refers (Special) to iusefp.o(.text) for __I$use$fp
    sqrt_x.o(i.____softfp_sqrt$lsc) refers to cdcmple.o(.text) for __aeabi_cdcmple
    sqrt_x.o(i.____softfp_sqrt$lsc) refers to errno.o(i.__set_errno) for __set_errno
    sqrt_x.o(i.____softfp_sqrt$lsc) refers to dsqrt.o(.text) for _dsqrt
    sqrt_x.o(i.__sqrt$lsc) refers (Special) to iusefp.o(.text) for __I$use$fp
    sqrt_x.o(i.__sqrt$lsc) refers to cdcmple.o(.text) for __aeabi_cdcmple
    sqrt_x.o(i.__sqrt$lsc) refers to errno.o(i.__set_errno) for __set_errno
    sqrt_x.o(i.__sqrt$lsc) refers to dsqrt.o(.text) for _dsqrt
    entry2.o(.ARM.Collect$$$$00000001) refers to entry2.o(.ARM.Collect$$$$00002712) for __lit__00000000
    entry2.o(.ARM.Collect$$$$00002712) refers to startup_stm32f4xx.o(STACK) for __initial_sp
    entry2.o(__vectab_stack_and_reset_area) refers to startup_stm32f4xx.o(STACK) for __initial_sp
    entry2.o(__vectab_stack_and_reset_area) refers to entry.o(.ARM.Collect$$$$00000000) for __main
    entry5.o(.ARM.Collect$$$$00000004) refers to init.o(.text) for __scatterload
    entry9a.o(.ARM.Collect$$$$0000000B) refers to main.o(i.main) for main
    entry9b.o(.ARM.Collect$$$$0000000C) refers to main.o(i.main) for main
    fputc.o(i.fputc) refers (Special) to iusesemip.o(.text) for __I$use$semihosting$fputc
    fputc.o(i.fputc) refers (Special) to semi.o(.text) for __semihosting_library_function
    uldiv.o(.text) refers to llushr.o(.text) for __aeabi_llsr
    uldiv.o(.text) refers to llshl.o(.text) for __aeabi_llsl
    errno.o(i.__aeabi_errno_addr) refers to errno.o(.data) for .data
    errno.o(i.__read_errno) refers to errno.o(.data) for .data
    errno.o(i.__set_errno) refers to errno.o(.data) for .data
    strtod.o(.text) refers to scanf_fp.o(.text) for _scanf_real
    strtod.o(.text) refers to _sgetc.o(.text) for _sgetc
    strtod.o(.text) refers to isspace_c.o(.text) for isspace
    depilogue.o(.text) refers to llshl.o(.text) for __aeabi_llsl
    depilogue.o(.text) refers to llushr.o(.text) for __aeabi_llsr
    dfixul.o(.text) refers to llushr.o(.text) for __aeabi_llsr
    dfixul.o(.text) refers to llshl.o(.text) for __aeabi_llsl
    init.o(.text) refers to entry5.o(.ARM.Collect$$$$00000004) for __main_after_scatterload
    isspace_c.o(.text) refers to ctype_c.o(.text) for __ctype_lookup
    scanf_fp.o(.text) refers (Special) to iusefp.o(.text) for __I$use$fp
    scanf_fp.o(.text) refers to dfltul.o(.text) for __aeabi_ul2d
    scanf_fp.o(.text) refers to dmul.o(.text) for __aeabi_dmul
    scanf_fp.o(.text) refers to ddiv.o(.text) for __aeabi_ddiv
    scanf_fp.o(.text) refers to scanf_fp.o(i._is_digit) for _is_digit
    scanf_fp.o(.text) refers to d2f.o(.text) for __aeabi_d2f
    dsqrt.o(.text) refers to llushr.o(.text) for __aeabi_llsr
    dsqrt.o(.text) refers to depilogue.o(.text) for _double_round
    ctype_c.o(.text) refers to ctype_c.o(.constdata) for .constdata
    dfltul.o(.text) refers to depilogue.o(.text) for _double_epilogue
    scanf_fp.o(i._is_digit) refers (Special) to iusefp.o(.text) for __I$use$fp


==============================================================================

Removing Unused input sections from the image.

    Removing stm32f4xx_it.o(.emb_text), (8 bytes).
    Removing main.o(.emb_text), (8 bytes).
    Removing txh.o(.emb_text), (8 bytes).
    Removing system_stm32f4xx.o(.emb_text), (8 bytes).
    Removing system_stm32f4xx.o(i.SystemCoreClockUpdate), (192 bytes).
    Removing system_stm32f4xx.o(.data), (20 bytes).
    Removing startup_stm32f4xx.o(HEAP), (0 bytes).
    Removing misc.o(.emb_text), (8 bytes).
    Removing misc.o(i.NVIC_PriorityGroupConfig), (20 bytes).
    Removing misc.o(i.NVIC_SystemLPConfig), (32 bytes).
    Removing stm32f4xx_adc.o(.emb_text), (8 bytes).
    Removing stm32f4xx_adc.o(i.ADC_AnalogWatchdogCmd), (20 bytes).
    Removing stm32f4xx_adc.o(i.ADC_AnalogWatchdogSingleChannelConfig), (16 bytes).
    Removing stm32f4xx_adc.o(i.ADC_AnalogWatchdogThresholdsConfig), (6 bytes).
    Removing stm32f4xx_adc.o(i.ADC_AutoInjectedConvCmd), (22 bytes).
    Removing stm32f4xx_adc.o(i.ADC_ClearFlag), (6 bytes).
    Removing stm32f4xx_adc.o(i.ADC_ClearITPendingBit), (10 bytes).
    Removing stm32f4xx_adc.o(i.ADC_Cmd), (22 bytes).
    Removing stm32f4xx_adc.o(i.ADC_CommonInit), (48 bytes).
    Removing stm32f4xx_adc.o(i.ADC_CommonStructInit), (12 bytes).
    Removing stm32f4xx_adc.o(i.ADC_ContinuousModeCmd), (22 bytes).
    Removing stm32f4xx_adc.o(i.ADC_DMACmd), (22 bytes).
    Removing stm32f4xx_adc.o(i.ADC_DMARequestAfterLastTransferCmd), (22 bytes).
    Removing stm32f4xx_adc.o(i.ADC_DeInit), (22 bytes).
    Removing stm32f4xx_adc.o(i.ADC_DiscModeChannelCountConfig), (24 bytes).
    Removing stm32f4xx_adc.o(i.ADC_DiscModeCmd), (22 bytes).
    Removing stm32f4xx_adc.o(i.ADC_EOCOnEachRegularChannelCmd), (22 bytes).
    Removing stm32f4xx_adc.o(i.ADC_ExternalTrigInjectedConvConfig), (16 bytes).
    Removing stm32f4xx_adc.o(i.ADC_ExternalTrigInjectedConvEdgeConfig), (16 bytes).
    Removing stm32f4xx_adc.o(i.ADC_GetConversionValue), (8 bytes).
    Removing stm32f4xx_adc.o(i.ADC_GetFlagStatus), (18 bytes).
    Removing stm32f4xx_adc.o(i.ADC_GetITStatus), (38 bytes).
    Removing stm32f4xx_adc.o(i.ADC_GetInjectedConversionValue), (28 bytes).
    Removing stm32f4xx_adc.o(i.ADC_GetMultiModeConversionValue), (12 bytes).
    Removing stm32f4xx_adc.o(i.ADC_GetSoftwareStartConvStatus), (20 bytes).
    Removing stm32f4xx_adc.o(i.ADC_GetSoftwareStartInjectedConvCmdStatus), (20 bytes).
    Removing stm32f4xx_adc.o(i.ADC_ITConfig), (32 bytes).
    Removing stm32f4xx_adc.o(i.ADC_Init), (84 bytes).
    Removing stm32f4xx_adc.o(i.ADC_InjectedChannelConfig), (130 bytes).
    Removing stm32f4xx_adc.o(i.ADC_InjectedDiscModeCmd), (22 bytes).
    Removing stm32f4xx_adc.o(i.ADC_InjectedSequencerLengthConfig), (24 bytes).
    Removing stm32f4xx_adc.o(i.ADC_MultiModeDMARequestAfterLastTransferCmd), (44 bytes).
    Removing stm32f4xx_adc.o(i.ADC_RegularChannelConfig), (184 bytes).
    Removing stm32f4xx_adc.o(i.ADC_SetInjectedOffset), (20 bytes).
    Removing stm32f4xx_adc.o(i.ADC_SoftwareStartConv), (10 bytes).
    Removing stm32f4xx_adc.o(i.ADC_SoftwareStartInjectedConv), (10 bytes).
    Removing stm32f4xx_adc.o(i.ADC_StructInit), (20 bytes).
    Removing stm32f4xx_adc.o(i.ADC_TempSensorVrefintCmd), (44 bytes).
    Removing stm32f4xx_adc.o(i.ADC_VBATCmd), (44 bytes).
    Removing stm32f4xx_crc.o(.emb_text), (8 bytes).
    Removing stm32f4xx_crc.o(i.CRC_CalcBlockCRC), (36 bytes).
    Removing stm32f4xx_crc.o(i.CRC_CalcCRC), (16 bytes).
    Removing stm32f4xx_crc.o(i.CRC_GetCRC), (12 bytes).
    Removing stm32f4xx_crc.o(i.CRC_GetIDRegister), (12 bytes).
    Removing stm32f4xx_crc.o(i.CRC_ResetDR), (12 bytes).
    Removing stm32f4xx_crc.o(i.CRC_SetIDRegister), (12 bytes).
    Removing stm32f4xx_dma.o(.emb_text), (8 bytes).
    Removing stm32f4xx_dma.o(i.DMA_ClearITPendingBit), (52 bytes).
    Removing stm32f4xx_dma.o(i.DMA_DoubleBufferModeCmd), (22 bytes).
    Removing stm32f4xx_dma.o(i.DMA_DoubleBufferModeConfig), (24 bytes).
    Removing stm32f4xx_dma.o(i.DMA_FlowControllerConfig), (22 bytes).
    Removing stm32f4xx_dma.o(i.DMA_GetCmdStatus), (20 bytes).
    Removing stm32f4xx_dma.o(i.DMA_GetCurrDataCounter), (8 bytes).
    Removing stm32f4xx_dma.o(i.DMA_GetCurrentMemoryTarget), (20 bytes).
    Removing stm32f4xx_dma.o(i.DMA_GetFIFOStatus), (12 bytes).
    Removing stm32f4xx_dma.o(i.DMA_GetFlagStatus), (68 bytes).
    Removing stm32f4xx_dma.o(i.DMA_GetITStatus), (100 bytes).
    Removing stm32f4xx_dma.o(i.DMA_MemoryTargetConfig), (10 bytes).
    Removing stm32f4xx_dma.o(i.DMA_PeriphIncOffsetSizeConfig), (22 bytes).
    Removing stm32f4xx_dma.o(i.DMA_SetCurrDataCounter), (4 bytes).
    Removing stm32f4xx_dma.o(i.DMA_StructInit), (34 bytes).
    Removing stm32f4xx_exti.o(.emb_text), (8 bytes).
    Removing stm32f4xx_exti.o(i.EXTI_ClearFlag), (12 bytes).
    Removing stm32f4xx_exti.o(i.EXTI_DeInit), (36 bytes).
    Removing stm32f4xx_exti.o(i.EXTI_GenerateSWInterrupt), (16 bytes).
    Removing stm32f4xx_exti.o(i.EXTI_GetFlagStatus), (24 bytes).
    Removing stm32f4xx_exti.o(i.EXTI_StructInit), (16 bytes).
    Removing stm32f4xx_flash.o(.emb_text), (8 bytes).
    Removing stm32f4xx_flash.o(i.FLASH_ClearFlag), (12 bytes).
    Removing stm32f4xx_flash.o(i.FLASH_DataCacheCmd), (36 bytes).
    Removing stm32f4xx_flash.o(i.FLASH_DataCacheReset), (20 bytes).
    Removing stm32f4xx_flash.o(i.FLASH_EraseAllSectors), (108 bytes).
    Removing stm32f4xx_flash.o(i.FLASH_EraseSector), (136 bytes).
    Removing stm32f4xx_flash.o(i.FLASH_GetFlagStatus), (24 bytes).
    Removing stm32f4xx_flash.o(i.FLASH_GetStatus), (72 bytes).
    Removing stm32f4xx_flash.o(i.FLASH_ITConfig), (32 bytes).
    Removing stm32f4xx_flash.o(i.FLASH_InstructionCacheCmd), (36 bytes).
    Removing stm32f4xx_flash.o(i.FLASH_InstructionCacheReset), (20 bytes).
    Removing stm32f4xx_flash.o(i.FLASH_Lock), (20 bytes).
    Removing stm32f4xx_flash.o(i.FLASH_OB_BORConfig), (28 bytes).
    Removing stm32f4xx_flash.o(i.FLASH_OB_GetBOR), (16 bytes).
    Removing stm32f4xx_flash.o(i.FLASH_OB_GetRDP), (24 bytes).
    Removing stm32f4xx_flash.o(i.FLASH_OB_GetUser), (16 bytes).
    Removing stm32f4xx_flash.o(i.FLASH_OB_GetWRP), (12 bytes).
    Removing stm32f4xx_flash.o(i.FLASH_OB_Launch), (32 bytes).
    Removing stm32f4xx_flash.o(i.FLASH_OB_Lock), (20 bytes).
    Removing stm32f4xx_flash.o(i.FLASH_OB_RDPConfig), (28 bytes).
    Removing stm32f4xx_flash.o(i.FLASH_OB_Unlock), (36 bytes).
    Removing stm32f4xx_flash.o(i.FLASH_OB_UserConfig), (48 bytes).
    Removing stm32f4xx_flash.o(i.FLASH_OB_WRPConfig), (52 bytes).
    Removing stm32f4xx_flash.o(i.FLASH_PrefetchBufferCmd), (36 bytes).
    Removing stm32f4xx_flash.o(i.FLASH_ProgramByte), (76 bytes).
    Removing stm32f4xx_flash.o(i.FLASH_ProgramDoubleWord), (84 bytes).
    Removing stm32f4xx_flash.o(i.FLASH_ProgramHalfWord), (80 bytes).
    Removing stm32f4xx_flash.o(i.FLASH_ProgramWord), (80 bytes).
    Removing stm32f4xx_flash.o(i.FLASH_SetLatency), (12 bytes).
    Removing stm32f4xx_flash.o(i.FLASH_Unlock), (36 bytes).
    Removing stm32f4xx_flash.o(i.FLASH_WaitForLastOperation), (34 bytes).
    Removing stm32f4xx_gpio.o(.emb_text), (8 bytes).
    Removing stm32f4xx_gpio.o(i.GPIO_PinLockConfig), (34 bytes).
    Removing stm32f4xx_gpio.o(i.GPIO_ReadInputData), (8 bytes).
    Removing stm32f4xx_gpio.o(i.GPIO_ReadOutputData), (8 bytes).
    Removing stm32f4xx_gpio.o(i.GPIO_ReadOutputDataBit), (18 bytes).
    Removing stm32f4xx_gpio.o(i.GPIO_StructInit), (18 bytes).
    Removing stm32f4xx_gpio.o(i.GPIO_ToggleBits), (8 bytes).
    Removing stm32f4xx_gpio.o(i.GPIO_Write), (4 bytes).
    Removing stm32f4xx_gpio.o(i.GPIO_WriteBit), (10 bytes).
    Removing stm32f4xx_rcc.o(.emb_text), (8 bytes).
    Removing stm32f4xx_rcc.o(i.RCC_AHB1PeriphClockLPModeCmd), (32 bytes).
    Removing stm32f4xx_rcc.o(i.RCC_AHB2PeriphClockLPModeCmd), (32 bytes).
    Removing stm32f4xx_rcc.o(i.RCC_AHB2PeriphResetCmd), (32 bytes).
    Removing stm32f4xx_rcc.o(i.RCC_AHB3PeriphClockCmd), (32 bytes).
    Removing stm32f4xx_rcc.o(i.RCC_AHB3PeriphClockLPModeCmd), (32 bytes).
    Removing stm32f4xx_rcc.o(i.RCC_AHB3PeriphResetCmd), (32 bytes).
    Removing stm32f4xx_rcc.o(i.RCC_APB1PeriphClockLPModeCmd), (32 bytes).
    Removing stm32f4xx_rcc.o(i.RCC_APB2PeriphClockLPModeCmd), (32 bytes).
    Removing stm32f4xx_rcc.o(i.RCC_AdjustHSICalibrationValue), (24 bytes).
    Removing stm32f4xx_rcc.o(i.RCC_BackupResetCmd), (12 bytes).
    Removing stm32f4xx_rcc.o(i.RCC_ClearFlag), (20 bytes).
    Removing stm32f4xx_rcc.o(i.RCC_ClearITPendingBit), (12 bytes).
    Removing stm32f4xx_rcc.o(i.RCC_ClockSecuritySystemCmd), (12 bytes).
    Removing stm32f4xx_rcc.o(i.RCC_DeInit), (72 bytes).
    Removing stm32f4xx_rcc.o(i.RCC_GetFlagStatus), (64 bytes).
    Removing stm32f4xx_rcc.o(i.RCC_GetITStatus), (24 bytes).
    Removing stm32f4xx_rcc.o(i.RCC_GetSYSCLKSource), (16 bytes).
    Removing stm32f4xx_rcc.o(i.RCC_HCLKConfig), (24 bytes).
    Removing stm32f4xx_rcc.o(i.RCC_HSEConfig), (16 bytes).
    Removing stm32f4xx_rcc.o(i.RCC_HSICmd), (12 bytes).
    Removing stm32f4xx_rcc.o(i.RCC_I2SCLKConfig), (12 bytes).
    Removing stm32f4xx_rcc.o(i.RCC_ITConfig), (32 bytes).
    Removing stm32f4xx_rcc.o(i.RCC_LSEConfig), (44 bytes).
    Removing stm32f4xx_rcc.o(i.RCC_LSICmd), (12 bytes).
    Removing stm32f4xx_rcc.o(i.RCC_MCO1Config), (28 bytes).
    Removing stm32f4xx_rcc.o(i.RCC_MCO2Config), (28 bytes).
    Removing stm32f4xx_rcc.o(i.RCC_PCLK1Config), (24 bytes).
    Removing stm32f4xx_rcc.o(i.RCC_PCLK2Config), (24 bytes).
    Removing stm32f4xx_rcc.o(i.RCC_PLLCmd), (12 bytes).
    Removing stm32f4xx_rcc.o(i.RCC_PLLConfig), (36 bytes).
    Removing stm32f4xx_rcc.o(i.RCC_PLLI2SCmd), (12 bytes).
    Removing stm32f4xx_rcc.o(i.RCC_PLLI2SConfig), (16 bytes).
    Removing stm32f4xx_rcc.o(i.RCC_RTCCLKCmd), (12 bytes).
    Removing stm32f4xx_rcc.o(i.RCC_RTCCLKConfig), (60 bytes).
    Removing stm32f4xx_rcc.o(i.RCC_SYSCLKConfig), (24 bytes).
    Removing stm32f4xx_rcc.o(i.RCC_WaitForHSEStartUp), (56 bytes).
    Removing stm32f4xx_spi.o(.emb_text), (8 bytes).
    Removing stm32f4xx_spi.o(i.I2S_Cmd), (24 bytes).
    Removing stm32f4xx_spi.o(i.I2S_FullDuplexConfig), (80 bytes).
    Removing stm32f4xx_spi.o(i.I2S_Init), (360 bytes).
    Removing stm32f4xx_spi.o(i.I2S_StructInit), (20 bytes).
    Removing stm32f4xx_spi.o(i.SPI_BiDirectionalLineConfig), (28 bytes).
    Removing stm32f4xx_spi.o(i.SPI_CalculateCRC), (24 bytes).
    Removing stm32f4xx_spi.o(i.SPI_DataSizeConfig), (18 bytes).
    Removing stm32f4xx_spi.o(i.SPI_GetCRC), (16 bytes).
    Removing stm32f4xx_spi.o(i.SPI_GetCRCPolynomial), (6 bytes).
    Removing stm32f4xx_spi.o(i.SPI_I2S_ClearFlag), (6 bytes).
    Removing stm32f4xx_spi.o(i.SPI_I2S_ClearITPendingBit), (20 bytes).
    Removing stm32f4xx_spi.o(i.SPI_I2S_DMACmd), (18 bytes).
    Removing stm32f4xx_spi.o(i.SPI_I2S_GetITStatus), (52 bytes).
    Removing stm32f4xx_spi.o(i.SPI_I2S_ITConfig), (32 bytes).
    Removing stm32f4xx_spi.o(i.SPI_NSSInternalSoftwareConfig), (30 bytes).
    Removing stm32f4xx_spi.o(i.SPI_SSOutputCmd), (24 bytes).
    Removing stm32f4xx_spi.o(i.SPI_StructInit), (24 bytes).
    Removing stm32f4xx_spi.o(i.SPI_TIModeCmd), (24 bytes).
    Removing stm32f4xx_spi.o(i.SPI_TransmitCRC), (10 bytes).
    Removing stm32f4xx_syscfg.o(.emb_text), (8 bytes).
    Removing stm32f4xx_syscfg.o(i.SYSCFG_CompensationCellCmd), (12 bytes).
    Removing stm32f4xx_syscfg.o(i.SYSCFG_DeInit), (22 bytes).
    Removing stm32f4xx_syscfg.o(i.SYSCFG_ETH_MediaInterfaceConfig), (12 bytes).
    Removing stm32f4xx_syscfg.o(i.SYSCFG_GetCompensationCellStatus), (24 bytes).
    Removing stm32f4xx_syscfg.o(i.SYSCFG_MemoryRemapConfig), (12 bytes).
    Removing stm32f4xx_tim.o(.emb_text), (8 bytes).
    Removing stm32f4xx_tim.o(i.TI1_Config), (58 bytes).
    Removing stm32f4xx_tim.o(i.TI2_Config), (80 bytes).
    Removing stm32f4xx_tim.o(i.TI3_Config), (72 bytes).
    Removing stm32f4xx_tim.o(i.TI4_Config), (80 bytes).
    Removing stm32f4xx_tim.o(i.TIM_ARRPreloadConfig), (24 bytes).
    Removing stm32f4xx_tim.o(i.TIM_BDTRConfig), (32 bytes).
    Removing stm32f4xx_tim.o(i.TIM_BDTRStructInit), (18 bytes).
    Removing stm32f4xx_tim.o(i.TIM_CCPreloadControl), (24 bytes).
    Removing stm32f4xx_tim.o(i.TIM_CCxCmd), (30 bytes).
    Removing stm32f4xx_tim.o(i.TIM_CCxNCmd), (30 bytes).
    Removing stm32f4xx_tim.o(i.TIM_ClearITPendingBit), (6 bytes).
    Removing stm32f4xx_tim.o(i.TIM_ClearOC1Ref), (18 bytes).
    Removing stm32f4xx_tim.o(i.TIM_ClearOC2Ref), (24 bytes).
    Removing stm32f4xx_tim.o(i.TIM_ClearOC3Ref), (18 bytes).
    Removing stm32f4xx_tim.o(i.TIM_ClearOC4Ref), (24 bytes).
    Removing stm32f4xx_tim.o(i.TIM_CounterModeConfig), (18 bytes).
    Removing stm32f4xx_tim.o(i.TIM_CtrlPWMOutputs), (30 bytes).
    Removing stm32f4xx_tim.o(i.TIM_DMACmd), (18 bytes).
    Removing stm32f4xx_tim.o(i.TIM_DMAConfig), (10 bytes).
    Removing stm32f4xx_tim.o(i.TIM_ETRClockMode1Config), (54 bytes).
    Removing stm32f4xx_tim.o(i.TIM_ETRClockMode2Config), (32 bytes).
    Removing stm32f4xx_tim.o(i.TIM_ETRConfig), (28 bytes).
    Removing stm32f4xx_tim.o(i.TIM_EncoderInterfaceConfig), (66 bytes).
    Removing stm32f4xx_tim.o(i.TIM_ForcedOC1Config), (18 bytes).
    Removing stm32f4xx_tim.o(i.TIM_ForcedOC2Config), (26 bytes).
    Removing stm32f4xx_tim.o(i.TIM_ForcedOC3Config), (18 bytes).
    Removing stm32f4xx_tim.o(i.TIM_ForcedOC4Config), (26 bytes).
    Removing stm32f4xx_tim.o(i.TIM_GenerateEvent), (4 bytes).
    Removing stm32f4xx_tim.o(i.TIM_GetCapture1), (6 bytes).
    Removing stm32f4xx_tim.o(i.TIM_GetCapture2), (6 bytes).
    Removing stm32f4xx_tim.o(i.TIM_GetCapture3), (6 bytes).
    Removing stm32f4xx_tim.o(i.TIM_GetCapture4), (6 bytes).
    Removing stm32f4xx_tim.o(i.TIM_GetCounter), (6 bytes).
    Removing stm32f4xx_tim.o(i.TIM_GetFlagStatus), (18 bytes).
    Removing stm32f4xx_tim.o(i.TIM_GetPrescaler), (6 bytes).
    Removing stm32f4xx_tim.o(i.TIM_ICInit), (110 bytes).
    Removing stm32f4xx_tim.o(i.TIM_ICStructInit), (18 bytes).
    Removing stm32f4xx_tim.o(i.TIM_ITRxExternalClockConfig), (24 bytes).
    Removing stm32f4xx_tim.o(i.TIM_InternalClockConfig), (12 bytes).
    Removing stm32f4xx_tim.o(i.TIM_OC1FastConfig), (18 bytes).
    Removing stm32f4xx_tim.o(i.TIM_OC1Init), (124 bytes).
    Removing stm32f4xx_tim.o(i.TIM_OC1NPolarityConfig), (18 bytes).
    Removing stm32f4xx_tim.o(i.TIM_OC1PolarityConfig), (18 bytes).
    Removing stm32f4xx_tim.o(i.TIM_OC1PreloadConfig), (18 bytes).
    Removing stm32f4xx_tim.o(i.TIM_OC2FastConfig), (26 bytes).
    Removing stm32f4xx_tim.o(i.TIM_OC2Init), (164 bytes).
    Removing stm32f4xx_tim.o(i.TIM_OC2NPolarityConfig), (26 bytes).
    Removing stm32f4xx_tim.o(i.TIM_OC2PolarityConfig), (26 bytes).
    Removing stm32f4xx_tim.o(i.TIM_OC2PreloadConfig), (26 bytes).
    Removing stm32f4xx_tim.o(i.TIM_OC3FastConfig), (18 bytes).
    Removing stm32f4xx_tim.o(i.TIM_OC3Init), (160 bytes).
    Removing stm32f4xx_tim.o(i.TIM_OC3NPolarityConfig), (26 bytes).
    Removing stm32f4xx_tim.o(i.TIM_OC3PolarityConfig), (26 bytes).
    Removing stm32f4xx_tim.o(i.TIM_OC3PreloadConfig), (18 bytes).
    Removing stm32f4xx_tim.o(i.TIM_OC4FastConfig), (26 bytes).
    Removing stm32f4xx_tim.o(i.TIM_OC4Init), (120 bytes).
    Removing stm32f4xx_tim.o(i.TIM_OC4PolarityConfig), (26 bytes).
    Removing stm32f4xx_tim.o(i.TIM_OC4PreloadConfig), (26 bytes).
    Removing stm32f4xx_tim.o(i.TIM_OCStructInit), (20 bytes).
    Removing stm32f4xx_tim.o(i.TIM_PWMIConfig), (124 bytes).
    Removing stm32f4xx_tim.o(i.TIM_PrescalerConfig), (6 bytes).
    Removing stm32f4xx_tim.o(i.TIM_RemapConfig), (6 bytes).
    Removing stm32f4xx_tim.o(i.TIM_SelectCCDMA), (24 bytes).
    Removing stm32f4xx_tim.o(i.TIM_SelectCOM), (24 bytes).
    Removing stm32f4xx_tim.o(i.TIM_SelectHallSensor), (24 bytes).
    Removing stm32f4xx_tim.o(i.TIM_SelectInputTrigger), (18 bytes).
    Removing stm32f4xx_tim.o(i.TIM_SelectMasterSlaveMode), (18 bytes).
    Removing stm32f4xx_tim.o(i.TIM_SelectOCxM), (86 bytes).
    Removing stm32f4xx_tim.o(i.TIM_SelectOnePulseMode), (18 bytes).
    Removing stm32f4xx_tim.o(i.TIM_SelectOutputTrigger), (18 bytes).
    Removing stm32f4xx_tim.o(i.TIM_SelectSlaveMode), (18 bytes).
    Removing stm32f4xx_tim.o(i.TIM_SetAutoreload), (4 bytes).
    Removing stm32f4xx_tim.o(i.TIM_SetClockDivision), (18 bytes).
    Removing stm32f4xx_tim.o(i.TIM_SetCompare1), (4 bytes).
    Removing stm32f4xx_tim.o(i.TIM_SetCompare2), (4 bytes).
    Removing stm32f4xx_tim.o(i.TIM_SetCompare3), (4 bytes).
    Removing stm32f4xx_tim.o(i.TIM_SetCompare4), (4 bytes).
    Removing stm32f4xx_tim.o(i.TIM_SetCounter), (4 bytes).
    Removing stm32f4xx_tim.o(i.TIM_SetIC1Prescaler), (18 bytes).
    Removing stm32f4xx_tim.o(i.TIM_SetIC2Prescaler), (26 bytes).
    Removing stm32f4xx_tim.o(i.TIM_SetIC3Prescaler), (18 bytes).
    Removing stm32f4xx_tim.o(i.TIM_SetIC4Prescaler), (26 bytes).
    Removing stm32f4xx_tim.o(i.TIM_TIxExternalClockConfig), (62 bytes).
    Removing stm32f4xx_tim.o(i.TIM_TimeBaseStructInit), (18 bytes).
    Removing stm32f4xx_tim.o(i.TIM_UpdateDisableConfig), (24 bytes).
    Removing stm32f4xx_tim.o(i.TIM_UpdateRequestConfig), (24 bytes).
    Removing stm32f4xx_usart.o(.emb_text), (8 bytes).
    Removing stm32f4xx_usart.o(i.USART_ClearITPendingBit), (30 bytes).
    Removing stm32f4xx_usart.o(i.USART_ClockInit), (32 bytes).
    Removing stm32f4xx_usart.o(i.USART_ClockStructInit), (12 bytes).
    Removing stm32f4xx_usart.o(i.USART_HalfDuplexCmd), (24 bytes).
    Removing stm32f4xx_usart.o(i.USART_IrDACmd), (24 bytes).
    Removing stm32f4xx_usart.o(i.USART_IrDAConfig), (18 bytes).
    Removing stm32f4xx_usart.o(i.USART_LINBreakDetectLengthConfig), (18 bytes).
    Removing stm32f4xx_usart.o(i.USART_LINCmd), (24 bytes).
    Removing stm32f4xx_usart.o(i.USART_OneBitMethodCmd), (24 bytes).
    Removing stm32f4xx_usart.o(i.USART_OverSampling8Cmd), (22 bytes).
    Removing stm32f4xx_usart.o(i.USART_ReceiveData), (10 bytes).
    Removing stm32f4xx_usart.o(i.USART_ReceiverWakeUpCmd), (24 bytes).
    Removing stm32f4xx_usart.o(i.USART_SendBreak), (10 bytes).
    Removing stm32f4xx_usart.o(i.USART_SendData), (8 bytes).
    Removing stm32f4xx_usart.o(i.USART_SetAddress), (18 bytes).
    Removing stm32f4xx_usart.o(i.USART_SetGuardTime), (16 bytes).
    Removing stm32f4xx_usart.o(i.USART_SetPrescaler), (16 bytes).
    Removing stm32f4xx_usart.o(i.USART_SmartCardCmd), (24 bytes).
    Removing stm32f4xx_usart.o(i.USART_SmartCardNACKCmd), (24 bytes).
    Removing stm32f4xx_usart.o(i.USART_StructInit), (24 bytes).
    Removing stm32f4xx_usart.o(i.USART_WakeUpConfig), (18 bytes).
    Removing stm32f4xx_rng.o(.emb_text), (8 bytes).
    Removing stm32f4xx_rng.o(i.RNG_ClearFlag), (16 bytes).
    Removing stm32f4xx_rng.o(i.RNG_ClearITPendingBit), (16 bytes).
    Removing stm32f4xx_rng.o(i.RNG_DeInit), (20 bytes).
    Removing stm32f4xx_rng.o(i.RNG_GetFlagStatus), (24 bytes).
    Removing stm32f4xx_rng.o(i.RNG_GetITStatus), (24 bytes).
    Removing stm32f4xx_rng.o(i.RNG_ITConfig), (36 bytes).
    Removing stm32f4xx_wwdg.o(.emb_text), (8 bytes).
    Removing stm32f4xx_wwdg.o(i.WWDG_ClearFlag), (12 bytes).
    Removing stm32f4xx_wwdg.o(i.WWDG_DeInit), (22 bytes).
    Removing stm32f4xx_wwdg.o(i.WWDG_Enable), (16 bytes).
    Removing stm32f4xx_wwdg.o(i.WWDG_EnableIT), (12 bytes).
    Removing stm32f4xx_wwdg.o(i.WWDG_GetFlagStatus), (20 bytes).
    Removing stm32f4xx_wwdg.o(i.WWDG_SetCounter), (16 bytes).
    Removing stm32f4xx_wwdg.o(i.WWDG_SetPrescaler), (24 bytes).
    Removing stm32f4xx_wwdg.o(i.WWDG_SetWindowValue), (40 bytes).
    Removing stm32f4xx_iwdg.o(.emb_text), (8 bytes).
    Removing stm32f4xx_iwdg.o(i.IWDG_Enable), (16 bytes).
    Removing stm32f4xx_iwdg.o(i.IWDG_GetFlagStatus), (24 bytes).
    Removing stm32f4xx_iwdg.o(i.IWDG_SetPrescaler), (12 bytes).
    Removing stm32f4xx_iwdg.o(i.IWDG_SetReload), (12 bytes).
    Removing stm32f4xx_iwdg.o(i.IWDG_WriteAccessCmd), (12 bytes).
    Removing time_count.o(.emb_text), (8 bytes).
    Removing time_count.o(i.delay), (22 bytes).
    Removing fram.o(.emb_text), (8 bytes).
    Removing fram.o(i.PCBEncryption), (104 bytes).
    Removing pluse_input.o(.emb_text), (8 bytes).
    Removing md_connect.o(.emb_text), (8 bytes).
    Removing md_connect.o(i.TrueCharBuffSize), (20 bytes).
    Removing pos_connect.o(.emb_text), (8 bytes).
    Removing pos_connect.o(i.DeQueue), (46 bytes).
    Removing pos_connect.o(i.EnQueue), (112 bytes).
    Removing pos_connect.o(i.FToHA), (92 bytes).
    Removing pos_connect.o(i.FindCharFStr), (44 bytes).
    Removing pos_connect.o(i.FindMessage), (42 bytes).
    Removing pos_connect.o(i.InitQueue), (8 bytes).
    Removing pos_connect.o(i.POS_Connect_u64ToBCD), (116 bytes).
    Removing pos_connect.o(i.POS_Network_APN_Set), (404 bytes).
    Removing pos_connect.o(i.POS_WIFIReconnect), (424 bytes).
    Removing ds1307.o(.emb_text), (8 bytes).
    Removing at45db.o(.emb_text), (8 bytes).
    Removing at45db.o(i.AT45DB_Data_Init), (272 bytes).
    Removing at45db.o(i.ExChangeByte), (14 bytes).
    Removing at45db.o(i.NotByte), (18 bytes).
    Removing pluse_putout.o(.emb_text), (8 bytes).
    Removing pluse_putout.o(i.Pluse_PutoutTast), (2 bytes).
    Removing analog.o(.emb_text), (8 bytes).
    Removing analog.o(i.Pressure_ADCDMA_IRQHandler), (32 bytes).
    Removing analog.o(i.Pressure_ADC_Configuration), (152 bytes).
    Removing analog.o(i.Pressure_DMA_Configuration), (128 bytes).
    Removing analog.o(i.Pressure_IO_Configuration), (40 bytes).
    Removing analog.o(i.Pressure_Init), (64 bytes).
    Removing analog.o(i.Pressure_NVIC_Configuration), (32 bytes).
    Removing analog.o(i.PrssureTask), (160 bytes).
    Removing analog.o(.bss), (40 bytes).
    Removing analog.o(.data), (13 bytes).
    Removing file_sys.o(.emb_text), (8 bytes).
    Removing file_sys.o(i.CH376DirCreate), (38 bytes).
    Removing file_sys.o(i.CH376DirInfoRead), (12 bytes).
    Removing file_sys.o(i.CH376DirInfoSave), (10 bytes).
    Removing file_sys.o(i.CH376DiskCapacity), (42 bytes).
    Removing file_sys.o(i.CH376DiskMount), (10 bytes).
    Removing file_sys.o(i.CH376DiskQuery), (144 bytes).
    Removing file_sys.o(i.CH376DiskReqSense), (26 bytes).
    Removing file_sys.o(i.CH376EndDirInfo), (12 bytes).
    Removing file_sys.o(i.CH376FileCreatePath), (56 bytes).
    Removing file_sys.o(i.CH376FileErase), (70 bytes).
    Removing file_sys.o(i.CH376FileOpenDir), (100 bytes).
    Removing file_sys.o(i.CH376FileOpenPath), (14 bytes).
    Removing file_sys.o(i.CH376GetDiskStatus), (10 bytes).
    Removing file_sys.o(i.CH376SecLocate), (60 bytes).
    Removing file_sys.o(i.CH376SeparatePath), (46 bytes).
    Removing file_sys.o(i.CH376WriteHostBlock), (56 bytes).
    Removing file_sys.o(i.CH376WriteOfsBlock), (64 bytes).
    Removing file_sys.o(i.CH376WriteVar8), (40 bytes).
    Removing file_sys.o(i.Spi376InByte), (28 bytes).
    Removing log.o(.emb_text), (8 bytes).
    Removing oled.o(.emb_text), (8 bytes).
    Removing oled.o(i.OLED_ColorTurn), (28 bytes).
    Removing oled.o(i.OLED_DisPlay_Off), (28 bytes).
    Removing oled.o(i.OLED_DisPlay_On), (28 bytes).
    Removing oled.o(i.OLED_DisplayTurn), (44 bytes).
    Removing oled.o(i.OLED_DrawArc), (424 bytes).
    Removing oled.o(i.OLED_DrawCircle), (168 bytes).
    Removing surface.o(.emb_text), (8 bytes).
    Removing printf.o(.emb_text), (8 bytes).
    Removing printf.o(i.LFnRow), (20 bytes).
    Removing printf.o(i.printCR), (10 bytes).
    Removing printf.o(i.printChinese), (18 bytes).
    Removing printf.o(i.printLF), (10 bytes).
    Removing printf.o(i.print_init), (16 bytes).
    Removing printf.o(i.setLeftSpace), (20 bytes).
    Removing printf.o(i.setPageLen), (20 bytes).
    Removing printf.o(i.setRightSpace), (20 bytes).
    Removing printf.o(i.setRowSpace), (20 bytes).
    Removing printf.o(i.setWordSpace), (20 bytes).
    Removing multiplex_port.o(.emb_text), (8 bytes).
    Removing multiplex_port.o(i.BigToLittle), (12 bytes).
    Removing multiplex_port.o(i.Multiplex_Port_TXDataCheck), (34 bytes).
    Removing multiplex_port.o(i.StringToHex), (132 bytes).
    Removing delay.o(.emb_text), (8 bytes).
    Removing dneg.o(.text), (6 bytes).
    Removing dfixul.o(.text), (48 bytes).

392 unused section(s) (total 13431 bytes) removed from the image.

==============================================================================

Image Symbol Table

    Local Symbols

    Symbol Name                              Value     Ov Type        Size  Object(Section)

    ../clib/../cmprslib/zerorunl2.c          0x00000000   Number         0  __dczerorl2.o ABSOLUTE
    ../clib/microlib/ctype/ctype.c           0x00000000   Number         0  isspace_c.o ABSOLUTE
    ../clib/microlib/ctype/ctype.c           0x00000000   Number         0  ctype_c.o ABSOLUTE
    ../clib/microlib/division.c              0x00000000   Number         0  uldiv.o ABSOLUTE
    ../clib/microlib/division.c              0x00000000   Number         0  ldiv.o ABSOLUTE
    ../clib/microlib/division.c              0x00000000   Number         0  uidiv.o ABSOLUTE
    ../clib/microlib/errno.c                 0x00000000   Number         0  errno.o ABSOLUTE
    ../clib/microlib/init/entry.s            0x00000000   Number         0  entry9a.o ABSOLUTE
    ../clib/microlib/init/entry.s            0x00000000   Number         0  entry8b.o ABSOLUTE
    ../clib/microlib/init/entry.s            0x00000000   Number         0  entry8a.o ABSOLUTE
    ../clib/microlib/init/entry.s            0x00000000   Number         0  entry10b.o ABSOLUTE
    ../clib/microlib/init/entry.s            0x00000000   Number         0  entry7b.o ABSOLUTE
    ../clib/microlib/init/entry.s            0x00000000   Number         0  entry7a.o ABSOLUTE
    ../clib/microlib/init/entry.s            0x00000000   Number         0  entry9b.o ABSOLUTE
    ../clib/microlib/init/entry.s            0x00000000   Number         0  entry.o ABSOLUTE
    ../clib/microlib/init/entry.s            0x00000000   Number         0  entry5.o ABSOLUTE
    ../clib/microlib/init/entry.s            0x00000000   Number         0  entry11a.o ABSOLUTE
    ../clib/microlib/init/entry.s            0x00000000   Number         0  entry11b.o ABSOLUTE
    ../clib/microlib/init/entry.s            0x00000000   Number         0  entry2.o ABSOLUTE
    ../clib/microlib/init/entry.s            0x00000000   Number         0  entry12a.o ABSOLUTE
    ../clib/microlib/init/entry.s            0x00000000   Number         0  entry12b.o ABSOLUTE
    ../clib/microlib/init/entry.s            0x00000000   Number         0  entry10a.o ABSOLUTE
    ../clib/microlib/longlong.c              0x00000000   Number         0  llsshr.o ABSOLUTE
    ../clib/microlib/longlong.c              0x00000000   Number         0  llshl.o ABSOLUTE
    ../clib/microlib/longlong.c              0x00000000   Number         0  llushr.o ABSOLUTE
    ../clib/microlib/printf/printf.c         0x00000000   Number         0  printfa.o ABSOLUTE
    ../clib/microlib/printf/printf.c         0x00000000   Number         0  printf8.o ABSOLUTE
    ../clib/microlib/printf/printf.c         0x00000000   Number         0  printf7.o ABSOLUTE
    ../clib/microlib/printf/printf.c         0x00000000   Number         0  printf5.o ABSOLUTE
    ../clib/microlib/printf/printf.c         0x00000000   Number         0  printf4.o ABSOLUTE
    ../clib/microlib/printf/printf.c         0x00000000   Number         0  printf6.o ABSOLUTE
    ../clib/microlib/printf/printf.c         0x00000000   Number         0  printf0.o ABSOLUTE
    ../clib/microlib/printf/printf.c         0x00000000   Number         0  printfb.o ABSOLUTE
    ../clib/microlib/printf/printf.c         0x00000000   Number         0  printf3.o ABSOLUTE
    ../clib/microlib/printf/printf.c         0x00000000   Number         0  printf2.o ABSOLUTE
    ../clib/microlib/printf/printf.c         0x00000000   Number         0  printf1.o ABSOLUTE
    ../clib/microlib/printf/stubs.s          0x00000000   Number         0  stubs.o ABSOLUTE
    ../clib/microlib/stdio/fputc.c           0x00000000   Number         0  fputc.o ABSOLUTE
    ../clib/microlib/stdio/semi.s            0x00000000   Number         0  semi.o ABSOLUTE
    ../clib/microlib/stdio/streams.c         0x00000000   Number         0  stdout.o ABSOLUTE
    ../clib/microlib/string/memcpy.c         0x00000000   Number         0  memcpyb.o ABSOLUTE
    ../clib/microlib/string/memcpy.c         0x00000000   Number         0  memcpya.o ABSOLUTE
    ../clib/microlib/string/strcat.c         0x00000000   Number         0  strcat.o ABSOLUTE
    ../clib/microlib/string/strlen.c         0x00000000   Number         0  strlen.o ABSOLUTE
    ../clib/microlib/string/strncmp.c        0x00000000   Number         0  strncmp.o ABSOLUTE
    ../clib/microlib/stubs.s                 0x00000000   Number         0  iusesemip.o ABSOLUTE
    ../clib/microlib/stubs.s                 0x00000000   Number         0  iusefp.o ABSOLUTE
    ../clib/scanf.c                          0x00000000   Number         0  scanf_fp.o ABSOLUTE
    ../clib/scanf.c                          0x00000000   Number         0  _sgetc.o ABSOLUTE
    ../clib/scanf.c                          0x00000000   Number         0  strtod.o ABSOLUTE
    ../fplib/microlib/d2f.c                  0x00000000   Number         0  d2f.o ABSOLUTE
    ../fplib/microlib/f2d.c                  0x00000000   Number         0  f2d.o ABSOLUTE
    ../fplib/microlib/fpadd.c                0x00000000   Number         0  dadd.o ABSOLUTE
    ../fplib/microlib/fpdiv.c                0x00000000   Number         0  ddiv.o ABSOLUTE
    ../fplib/microlib/fpepilogue.c           0x00000000   Number         0  depilogue.o ABSOLUTE
    ../fplib/microlib/fpepilogue.c           0x00000000   Number         0  fepilogue.o ABSOLUTE
    ../fplib/microlib/fpfix.c                0x00000000   Number         0  dfixi.o ABSOLUTE
    ../fplib/microlib/fpfix.c                0x00000000   Number         0  dfixul.o ABSOLUTE
    ../fplib/microlib/fpfix.c                0x00000000   Number         0  ffixl.o ABSOLUTE
    ../fplib/microlib/fpfix.c                0x00000000   Number         0  dfixl.o ABSOLUTE
    ../fplib/microlib/fpflt.c                0x00000000   Number         0  ffltl.o ABSOLUTE
    ../fplib/microlib/fpflt.c                0x00000000   Number         0  dfltul.o ABSOLUTE
    ../fplib/microlib/fpflt.c                0x00000000   Number         0  dflti.o ABSOLUTE
    ../fplib/microlib/fpflt.c                0x00000000   Number         0  dfltl.o ABSOLUTE
    ../fplib/microlib/fpflt.c                0x00000000   Number         0  dfltui.o ABSOLUTE
    ../fplib/microlib/fpmul.c                0x00000000   Number         0  dmul.o ABSOLUTE
    ../fplib/microlib/fpneg.c                0x00000000   Number         0  dneg.o ABSOLUTE
    ../fplib/microlib/fpscalb.c              0x00000000   Number         0  dscalb.o ABSOLUTE
    ../fplib/microlib/fpsqrt.c               0x00000000   Number         0  dsqrt.o ABSOLUTE
    ../mathlib/atof.c                        0x00000000   Number         0  atof.o ABSOLUTE
    ../mathlib/cos.c                         0x00000000   Number         0  cos.o ABSOLUTE
    ../mathlib/cos.c                         0x00000000   Number         0  cos_x.o ABSOLUTE
    ../mathlib/cos_i.c                       0x00000000   Number         0  cos_i.o ABSOLUTE
    ../mathlib/dunder.c                      0x00000000   Number         0  dunder.o ABSOLUTE
    ../mathlib/fabs.c                        0x00000000   Number         0  fabs.o ABSOLUTE
    ../mathlib/fpclassify.c                  0x00000000   Number         0  fpclassify.o ABSOLUTE
    ../mathlib/log.c                         0x00000000   Number         0  log_x.o ABSOLUTE
    ../mathlib/log.c                         0x00000000   Number         0  log.o ABSOLUTE
    ../mathlib/log10.c                       0x00000000   Number         0  log10_x.o ABSOLUTE
    ../mathlib/log10.c                       0x00000000   Number         0  log10.o ABSOLUTE
    ../mathlib/poly.c                        0x00000000   Number         0  poly.o ABSOLUTE
    ../mathlib/pow.c                         0x00000000   Number         0  pow_x.o ABSOLUTE
    ../mathlib/pow.c                         0x00000000   Number         0  pow.o ABSOLUTE
    ../mathlib/qnan.c                        0x00000000   Number         0  qnan.o ABSOLUTE
    ../mathlib/rred.c                        0x00000000   Number         0  rred.o ABSOLUTE
    ../mathlib/sin.c                         0x00000000   Number         0  sin.o ABSOLUTE
    ../mathlib/sin.c                         0x00000000   Number         0  sin_x.o ABSOLUTE
    ../mathlib/sin_i.c                       0x00000000   Number         0  sin_i_x.o ABSOLUTE
    ../mathlib/sin_i.c                       0x00000000   Number         0  sin_i.o ABSOLUTE
    ../mathlib/sqrt.c                        0x00000000   Number         0  sqrt_x.o ABSOLUTE
    ../mathlib/sqrt.c                        0x00000000   Number         0  sqrt.o ABSOLUTE
    ..\Libraries\STM32F4xx_StdPeriph_Driver\src\misc.c 0x00000000   Number         0  misc.o ABSOLUTE
    ..\Libraries\STM32F4xx_StdPeriph_Driver\src\stm32f4xx_adc.c 0x00000000   Number         0  stm32f4xx_adc.o ABSOLUTE
    ..\Libraries\STM32F4xx_StdPeriph_Driver\src\stm32f4xx_crc.c 0x00000000   Number         0  stm32f4xx_crc.o ABSOLUTE
    ..\Libraries\STM32F4xx_StdPeriph_Driver\src\stm32f4xx_dma.c 0x00000000   Number         0  stm32f4xx_dma.o ABSOLUTE
    ..\Libraries\STM32F4xx_StdPeriph_Driver\src\stm32f4xx_exti.c 0x00000000   Number         0  stm32f4xx_exti.o ABSOLUTE
    ..\Libraries\STM32F4xx_StdPeriph_Driver\src\stm32f4xx_flash.c 0x00000000   Number         0  stm32f4xx_flash.o ABSOLUTE
    ..\Libraries\STM32F4xx_StdPeriph_Driver\src\stm32f4xx_gpio.c 0x00000000   Number         0  stm32f4xx_gpio.o ABSOLUTE
    ..\Libraries\STM32F4xx_StdPeriph_Driver\src\stm32f4xx_iwdg.c 0x00000000   Number         0  stm32f4xx_iwdg.o ABSOLUTE
    ..\Libraries\STM32F4xx_StdPeriph_Driver\src\stm32f4xx_rcc.c 0x00000000   Number         0  stm32f4xx_rcc.o ABSOLUTE
    ..\Libraries\STM32F4xx_StdPeriph_Driver\src\stm32f4xx_rng.c 0x00000000   Number         0  stm32f4xx_rng.o ABSOLUTE
    ..\Libraries\STM32F4xx_StdPeriph_Driver\src\stm32f4xx_spi.c 0x00000000   Number         0  stm32f4xx_spi.o ABSOLUTE
    ..\Libraries\STM32F4xx_StdPeriph_Driver\src\stm32f4xx_syscfg.c 0x00000000   Number         0  stm32f4xx_syscfg.o ABSOLUTE
    ..\Libraries\STM32F4xx_StdPeriph_Driver\src\stm32f4xx_tim.c 0x00000000   Number         0  stm32f4xx_tim.o ABSOLUTE
    ..\Libraries\STM32F4xx_StdPeriph_Driver\src\stm32f4xx_usart.c 0x00000000   Number         0  stm32f4xx_usart.o ABSOLUTE
    ..\Libraries\STM32F4xx_StdPeriph_Driver\src\stm32f4xx_wwdg.c 0x00000000   Number         0  stm32f4xx_wwdg.o ABSOLUTE
    ..\System\startup_stm32f4xx.s            0x00000000   Number         0  startup_stm32f4xx.o ABSOLUTE
    ..\User\AT45DB\at45db.c                  0x00000000   Number         0  at45db.o ABSOLUTE
    ..\User\Analog\Analog.c                  0x00000000   Number         0  analog.o ABSOLUTE
    ..\User\CH376_Driver\FILE_SYS.c          0x00000000   Number         0  file_sys.o ABSOLUTE
    ..\User\DS1307\DS1307.c                  0x00000000   Number         0  ds1307.o ABSOLUTE
    ..\User\Delay\delay.c                    0x00000000   Number         0  delay.o ABSOLUTE
    ..\User\FRam\FRam.c                      0x00000000   Number         0  fram.o ABSOLUTE
    ..\User\Log\Log.c                        0x00000000   Number         0  log.o ABSOLUTE
    ..\User\MD_Connect\MD_Connect.c          0x00000000   Number         0  md_connect.o ABSOLUTE
    ..\User\Multiplex_Port\Multiplex_Port.c  0x00000000   Number         0  multiplex_port.o ABSOLUTE
    ..\User\OLED\oled.c                      0x00000000   Number         0  oled.o ABSOLUTE
    ..\User\POS_Connect\POS_Connect.c        0x00000000   Number         0  pos_connect.o ABSOLUTE
    ..\User\Printf\Printf.c                  0x00000000   Number         0  printf.o ABSOLUTE
    ..\User\Pulse_InPut\Pluse_InPut.c        0x00000000   Number         0  pluse_input.o ABSOLUTE
    ..\User\Pulse_PutOut\Pluse_Putout.c      0x00000000   Number         0  pluse_putout.o ABSOLUTE
    ..\User\Surface\Surface.c                0x00000000   Number         0  surface.o ABSOLUTE
    ..\User\TXH\TXH.c                        0x00000000   Number         0  txh.o ABSOLUTE
    ..\User\Timer\time_count.c               0x00000000   Number         0  time_count.o ABSOLUTE
    ..\User\main.c                           0x00000000   Number         0  main.o ABSOLUTE
    ..\User\stm32f4xx_it.c                   0x00000000   Number         0  stm32f4xx_it.o ABSOLUTE
    ..\User\system_stm32f4xx.c               0x00000000   Number         0  system_stm32f4xx.o ABSOLUTE
    ..\\Libraries\\STM32F4xx_StdPeriph_Driver\\src\\misc.c 0x00000000   Number         0  misc.o ABSOLUTE
    ..\\Libraries\\STM32F4xx_StdPeriph_Driver\\src\\stm32f4xx_adc.c 0x00000000   Number         0  stm32f4xx_adc.o ABSOLUTE
    ..\\Libraries\\STM32F4xx_StdPeriph_Driver\\src\\stm32f4xx_crc.c 0x00000000   Number         0  stm32f4xx_crc.o ABSOLUTE
    ..\\Libraries\\STM32F4xx_StdPeriph_Driver\\src\\stm32f4xx_dma.c 0x00000000   Number         0  stm32f4xx_dma.o ABSOLUTE
    ..\\Libraries\\STM32F4xx_StdPeriph_Driver\\src\\stm32f4xx_exti.c 0x00000000   Number         0  stm32f4xx_exti.o ABSOLUTE
    ..\\Libraries\\STM32F4xx_StdPeriph_Driver\\src\\stm32f4xx_flash.c 0x00000000   Number         0  stm32f4xx_flash.o ABSOLUTE
    ..\\Libraries\\STM32F4xx_StdPeriph_Driver\\src\\stm32f4xx_gpio.c 0x00000000   Number         0  stm32f4xx_gpio.o ABSOLUTE
    ..\\Libraries\\STM32F4xx_StdPeriph_Driver\\src\\stm32f4xx_iwdg.c 0x00000000   Number         0  stm32f4xx_iwdg.o ABSOLUTE
    ..\\Libraries\\STM32F4xx_StdPeriph_Driver\\src\\stm32f4xx_rcc.c 0x00000000   Number         0  stm32f4xx_rcc.o ABSOLUTE
    ..\\Libraries\\STM32F4xx_StdPeriph_Driver\\src\\stm32f4xx_rng.c 0x00000000   Number         0  stm32f4xx_rng.o ABSOLUTE
    ..\\Libraries\\STM32F4xx_StdPeriph_Driver\\src\\stm32f4xx_spi.c 0x00000000   Number         0  stm32f4xx_spi.o ABSOLUTE
    ..\\Libraries\\STM32F4xx_StdPeriph_Driver\\src\\stm32f4xx_syscfg.c 0x00000000   Number         0  stm32f4xx_syscfg.o ABSOLUTE
    ..\\Libraries\\STM32F4xx_StdPeriph_Driver\\src\\stm32f4xx_tim.c 0x00000000   Number         0  stm32f4xx_tim.o ABSOLUTE
    ..\\Libraries\\STM32F4xx_StdPeriph_Driver\\src\\stm32f4xx_usart.c 0x00000000   Number         0  stm32f4xx_usart.o ABSOLUTE
    ..\\Libraries\\STM32F4xx_StdPeriph_Driver\\src\\stm32f4xx_wwdg.c 0x00000000   Number         0  stm32f4xx_wwdg.o ABSOLUTE
    ..\\User\\AT45DB\\at45db.c               0x00000000   Number         0  at45db.o ABSOLUTE
    ..\\User\\Analog\\Analog.c               0x00000000   Number         0  analog.o ABSOLUTE
    ..\\User\\CH376_Driver\\FILE_SYS.c       0x00000000   Number         0  file_sys.o ABSOLUTE
    ..\\User\\DS1307\\DS1307.c               0x00000000   Number         0  ds1307.o ABSOLUTE
    ..\\User\\Delay\\delay.c                 0x00000000   Number         0  delay.o ABSOLUTE
    ..\\User\\FRam\\FRam.c                   0x00000000   Number         0  fram.o ABSOLUTE
    ..\\User\\Log\\Log.c                     0x00000000   Number         0  log.o ABSOLUTE
    ..\\User\\MD_Connect\\MD_Connect.c       0x00000000   Number         0  md_connect.o ABSOLUTE
    ..\\User\\Multiplex_Port\\Multiplex_Port.c 0x00000000   Number         0  multiplex_port.o ABSOLUTE
    ..\\User\\OLED\\oled.c                   0x00000000   Number         0  oled.o ABSOLUTE
    ..\\User\\POS_Connect\\POS_Connect.c     0x00000000   Number         0  pos_connect.o ABSOLUTE
    ..\\User\\Printf\\Printf.c               0x00000000   Number         0  printf.o ABSOLUTE
    ..\\User\\Pulse_InPut\\Pluse_InPut.c     0x00000000   Number         0  pluse_input.o ABSOLUTE
    ..\\User\\Pulse_PutOut\\Pluse_Putout.c   0x00000000   Number         0  pluse_putout.o ABSOLUTE
    ..\\User\\Surface\\Surface.c             0x00000000   Number         0  surface.o ABSOLUTE
    ..\\User\\TXH\\TXH.c                     0x00000000   Number         0  txh.o ABSOLUTE
    ..\\User\\Timer\\time_count.c            0x00000000   Number         0  time_count.o ABSOLUTE
    ..\\User\\main.c                         0x00000000   Number         0  main.o ABSOLUTE
    ..\\User\\stm32f4xx_it.c                 0x00000000   Number         0  stm32f4xx_it.o ABSOLUTE
    ..\\User\\system_stm32f4xx.c             0x00000000   Number         0  system_stm32f4xx.o ABSOLUTE
    cdcmple.s                                0x00000000   Number         0  cdcmple.o ABSOLUTE
    cdrcmple.s                               0x00000000   Number         0  cdrcmple.o ABSOLUTE
    dc.s                                     0x00000000   Number         0  dc.o ABSOLUTE
    handlers.s                               0x00000000   Number         0  handlers.o ABSOLUTE
    init.s                                   0x00000000   Number         0  init.o ABSOLUTE
    RESET                                    0x08008000   Section      392  startup_stm32f4xx.o(RESET)
    .ARM.Collect$$$$00000000                 0x08008188   Section        0  entry.o(.ARM.Collect$$$$00000000)
    .ARM.Collect$$$$00000001                 0x08008188   Section        4  entry2.o(.ARM.Collect$$$$00000001)
    .ARM.Collect$$$$00000004                 0x0800818c   Section        4  entry5.o(.ARM.Collect$$$$00000004)
    .ARM.Collect$$$$00000008                 0x08008190   Section        0  entry7b.o(.ARM.Collect$$$$00000008)
    .ARM.Collect$$$$0000000A                 0x08008190   Section        0  entry8b.o(.ARM.Collect$$$$0000000A)
    .ARM.Collect$$$$0000000B                 0x08008190   Section        8  entry9a.o(.ARM.Collect$$$$0000000B)
    .ARM.Collect$$$$0000000E                 0x08008198   Section        4  entry12b.o(.ARM.Collect$$$$0000000E)
    .ARM.Collect$$$$0000000F                 0x0800819c   Section        0  entry10a.o(.ARM.Collect$$$$0000000F)
    .ARM.Collect$$$$00000011                 0x0800819c   Section        0  entry11a.o(.ARM.Collect$$$$00000011)
    .ARM.Collect$$$$00002712                 0x0800819c   Section        4  entry2.o(.ARM.Collect$$$$00002712)
    __lit__00000000                          0x0800819c   Data           4  entry2.o(.ARM.Collect$$$$00002712)
    .text                                    0x080081a0   Section       36  startup_stm32f4xx.o(.text)
    $v0                                      0x080081a0   Number         0  startup_stm32f4xx.o(.text)
    .text                                    0x080081c4   Section        0  ldiv.o(.text)
    .text                                    0x08008226   Section        0  llsshr.o(.text)
    .text                                    0x0800824a   Section        0  memcpya.o(.text)
    .text                                    0x0800826e   Section        0  strcat.o(.text)
    .text                                    0x08008286   Section        0  strlen.o(.text)
    .text                                    0x08008294   Section        0  strncmp.o(.text)
    .text                                    0x080082b2   Section        0  dadd.o(.text)
    .text                                    0x08008400   Section        0  dmul.o(.text)
    .text                                    0x080084e4   Section        0  ddiv.o(.text)
    .text                                    0x080085c2   Section        0  ffltl.o(.text)
    .text                                    0x080085ee   Section        0  dflti.o(.text)
    .text                                    0x08008610   Section        0  dfltui.o(.text)
    .text                                    0x0800862a   Section        0  dfltl.o(.text)
    .text                                    0x08008652   Section        0  ffixl.o(.text)
    .text                                    0x08008694   Section        0  dfixi.o(.text)
    .text                                    0x080086d2   Section        0  dfixl.o(.text)
    .text                                    0x0800871c   Section        0  f2d.o(.text)
    .text                                    0x08008742   Section        0  d2f.o(.text)
    .text                                    0x0800877a   Section        0  uldiv.o(.text)
    .text                                    0x080087dc   Section        0  llshl.o(.text)
    .text                                    0x080087fa   Section        0  llushr.o(.text)
    .text                                    0x0800881c   Section        0  strtod.o(.text)
    _local_sscanf                            0x0800881d   Thumb Code    54  strtod.o(.text)
    .text                                    0x080088b8   Section        0  iusefp.o(.text)
    .text                                    0x080088b8   Section        0  fepilogue.o(.text)
    .text                                    0x08008926   Section        0  depilogue.o(.text)
    .text                                    0x080089e0   Section        0  dscalb.o(.text)
    .text                                    0x08008a10   Section       48  cdrcmple.o(.text)
    .text                                    0x08008a40   Section       36  init.o(.text)
    .text                                    0x08008a64   Section        0  isspace_c.o(.text)
    .text                                    0x08008a70   Section        0  scanf_fp.o(.text)
    _fp_value                                0x08008a71   Thumb Code   296  scanf_fp.o(.text)
    .text                                    0x08008dd0   Section        0  _sgetc.o(.text)
    .text                                    0x08008e10   Section        0  dsqrt.o(.text)
    .text                                    0x08008eb4   Section       48  cdcmple.o(.text)
    .text                                    0x08008ee4   Section        0  ctype_c.o(.text)
    .text                                    0x08008f0c   Section        0  dfltul.o(.text)
    .text                                    0x08008f24   Section        0  __dczerorl2.o(.text)
    i.AT45DBDataCheck                        0x08008f7a   Section        0  at45db.o(i.AT45DBDataCheck)
    i.AT45DBItemRead                         0x08008f98   Section        0  at45db.o(i.AT45DBItemRead)
    i.AT45DBItemWrite                        0x080090d0   Section        0  at45db.o(i.AT45DBItemWrite)
    i.AT45DB_Init                            0x080091b8   Section        0  at45db.o(i.AT45DB_Init)
    i.AT45DB_ReadPage                        0x08009208   Section        0  at45db.o(i.AT45DB_ReadPage)
    i.AT45DB_SendByte                        0x080092c8   Section        0  at45db.o(i.AT45DB_SendByte)
    i.AT45DB_SetPageByte                     0x08009300   Section        0  at45db.o(i.AT45DB_SetPageByte)
    i.AT45DB_WriteBuff                       0x0800938c   Section        0  at45db.o(i.AT45DB_WriteBuff)
    i.AT45DB_WritePage                       0x08009430   Section        0  at45db.o(i.AT45DB_WritePage)
    i.BCC_CheckSum                           0x080094d4   Section        0  md_connect.o(i.BCC_CheckSum)
    i.Bluesky_Decrypt                        0x080094ee   Section        0  md_connect.o(i.Bluesky_Decrypt)
    i.Bluesky_Encrypt                        0x08009502   Section        0  md_connect.o(i.Bluesky_Encrypt)
    i.CH376ByteLocate                        0x08009564   Section        0  file_sys.o(i.CH376ByteLocate)
    i.CH376ByteRead                          0x080095a0   Section        0  file_sys.o(i.CH376ByteRead)
    i.CH376ByteWrite                         0x08009604   Section        0  file_sys.o(i.CH376ByteWrite)
    i.CH376DiskConnect                       0x0800966c   Section        0  file_sys.o(i.CH376DiskConnect)
    i.CH376FileClose                         0x08009680   Section        0  file_sys.o(i.CH376FileClose)
    i.CH376FileCreate                        0x0800968e   Section        0  file_sys.o(i.CH376FileCreate)
    i.CH376FileOpen                          0x080096a2   Section        0  file_sys.o(i.CH376FileOpen)
    i.CH376GetFileSize                       0x080096c8   Section        0  file_sys.o(i.CH376GetFileSize)
    i.CH376GetIntStatus                      0x080096d4   Section        0  file_sys.o(i.CH376GetIntStatus)
    i.CH376Read32bitDat                      0x080096f4   Section        0  file_sys.o(i.CH376Read32bitDat)
    i.CH376ReadBlock                         0x08009730   Section        0  file_sys.o(i.CH376ReadBlock)
    i.CH376ReadVar32                         0x08009768   Section        0  file_sys.o(i.CH376ReadVar32)
    i.CH376ReadVar8                          0x08009780   Section        0  file_sys.o(i.CH376ReadVar8)
    i.CH376SendCmdDatWaitInt                 0x080097a8   Section        0  file_sys.o(i.CH376SendCmdDatWaitInt)
    i.CH376SendCmdWaitInt                    0x080097d0   Section        0  file_sys.o(i.CH376SendCmdWaitInt)
    i.CH376SetFileName                       0x080097f0   Section        0  file_sys.o(i.CH376SetFileName)
    i.CH376WriteReqBlock                     0x08009898   Section        0  file_sys.o(i.CH376WriteReqBlock)
    i.CH376WriteVar32                        0x080098d0   Section        0  file_sys.o(i.CH376WriteVar32)
    i.CRC_Check                              0x08009910   Section        0  pos_connect.o(i.CRC_Check)
    i.CheckSum                               0x08009948   Section        0  md_connect.o(i.CheckSum)
    i.CheckSum8                              0x0800998e   Section        0  md_connect.o(i.CheckSum8)
    i.DMA1_Stream3_IRQHandler                0x080099aa   Section        0  stm32f4xx_it.o(i.DMA1_Stream3_IRQHandler)
    i.DMA1_Stream4_IRQHandler                0x080099b2   Section        0  stm32f4xx_it.o(i.DMA1_Stream4_IRQHandler)
    i.DMA1_Stream6_IRQHandler                0x080099ba   Section        0  stm32f4xx_it.o(i.DMA1_Stream6_IRQHandler)
    i.DMA1_Stream7_IRQHandler                0x080099c2   Section        0  stm32f4xx_it.o(i.DMA1_Stream7_IRQHandler)
    i.DMA2_Stream6_IRQHandler                0x080099ca   Section        0  stm32f4xx_it.o(i.DMA2_Stream6_IRQHandler)
    i.DMA2_Stream7_IRQHandler                0x080099d2   Section        0  stm32f4xx_it.o(i.DMA2_Stream7_IRQHandler)
    i.DMA_ClearFlag                          0x080099dc   Section        0  stm32f4xx_dma.o(i.DMA_ClearFlag)
    i.DMA_Cmd                                0x08009a10   Section        0  stm32f4xx_dma.o(i.DMA_Cmd)
    i.DMA_DeInit                             0x08009a28   Section        0  stm32f4xx_dma.o(i.DMA_DeInit)
    i.DMA_ITConfig                           0x08009b80   Section        0  stm32f4xx_dma.o(i.DMA_ITConfig)
    i.DMA_Init                               0x08009bbc   Section        0  stm32f4xx_dma.o(i.DMA_Init)
    i.DS1307_Init                            0x08009c14   Section        0  ds1307.o(i.DS1307_Init)
    i.DS1307_Read                            0x08009cac   Section        0  ds1307.o(i.DS1307_Read)
    i.DS1307_Write                           0x08009d34   Section        0  ds1307.o(i.DS1307_Write)
    i.DartCRC16                              0x08009db0   Section        0  pos_connect.o(i.DartCRC16)
    i.Decode_Data                            0x08009de8   Section        0  pos_connect.o(i.Decode_Data)
    i.EXTI0_IRQHandler                       0x08009e18   Section        0  stm32f4xx_it.o(i.EXTI0_IRQHandler)
    i.EXTI15_10_IRQHandler                   0x08009e20   Section        0  stm32f4xx_it.o(i.EXTI15_10_IRQHandler)
    i.EXTI1_IRQHandler                       0x08009e28   Section        0  stm32f4xx_it.o(i.EXTI1_IRQHandler)
    i.EXTI_ClearITPendingBit                 0x08009e30   Section        0  stm32f4xx_exti.o(i.EXTI_ClearITPendingBit)
    i.EXTI_GetITStatus                       0x08009e3c   Section        0  stm32f4xx_exti.o(i.EXTI_GetITStatus)
    i.EXTI_Init                              0x08009e64   Section        0  stm32f4xx_exti.o(i.EXTI_Init)
    i.Encrypt_Data                           0x08009ef8   Section        0  pos_connect.o(i.Encrypt_Data)
    i.FMItemRead                             0x08009f28   Section        0  fram.o(i.FMItemRead)
    i.FMItemWrite                            0x0800a0ac   Section        0  fram.o(i.FMItemWrite)
    i.FM_Data_Init                           0x0800a1f8   Section        0  fram.o(i.FM_Data_Init)
    i.FM_IO_Configuration                    0x0800a350   Section        0  fram.o(i.FM_IO_Configuration)
    i.FM_Init                                0x0800a3d0   Section        0  fram.o(i.FM_Init)
    i.FM_ReadData                            0x0800a4bc   Section        0  fram.o(i.FM_ReadData)
    i.FM_SPI1_SendByte                       0x0800a528   Section        0  fram.o(i.FM_SPI1_SendByte)
    i.FM_SPI_Configuration                   0x0800a560   Section        0  fram.o(i.FM_SPI_Configuration)
    i.FM_WriteData                           0x0800a5c0   Section        0  fram.o(i.FM_WriteData)
    i.FRamDataCheck                          0x0800a648   Section        0  fram.o(i.FRamDataCheck)
    i.FindKey                                0x0800a664   Section        0  surface.o(i.FindKey)
    i.FindSysconfigFile                      0x0800a738   Section        0  log.o(i.FindSysconfigFile)
    i.GPIO_DeInit                            0x0800a988   Section        0  stm32f4xx_gpio.o(i.GPIO_DeInit)
    i.GPIO_Init                              0x0800aa88   Section        0  stm32f4xx_gpio.o(i.GPIO_Init)
    i.GPIO_PinAFConfig                       0x0800ab18   Section        0  stm32f4xx_gpio.o(i.GPIO_PinAFConfig)
    i.GPIO_ReadInputDataBit                  0x0800ab5e   Section        0  stm32f4xx_gpio.o(i.GPIO_ReadInputDataBit)
    i.GPIO_ResetBits                         0x0800ab70   Section        0  stm32f4xx_gpio.o(i.GPIO_ResetBits)
    i.GPIO_SetBits                           0x0800ab74   Section        0  stm32f4xx_gpio.o(i.GPIO_SetBits)
    i.GetKeyNum                              0x0800ab78   Section        0  surface.o(i.GetKeyNum)
    i.HardFault_Handler                      0x0800ab88   Section        0  stm32f4xx_it.o(i.HardFault_Handler)
    i.IWDG_ReloadCounter                     0x0800abcc   Section        0  stm32f4xx_iwdg.o(i.IWDG_ReloadCounter)
    i.InteiHEXCheck                          0x0800abdc   Section        0  md_connect.o(i.InteiHEXCheck)
    i.Log_Init                               0x0800abfc   Section        0  log.o(i.Log_Init)
    i.Log_Task                               0x0800ac0c   Section        0  log.o(i.Log_Task)
    i.MD_ConnectRXTask                       0x0800ae74   Section        0  md_connect.o(i.MD_ConnectRXTask)
    i.MD_ConnectTXTask                       0x0801f1cc   Section        0  md_connect.o(i.MD_ConnectTXTask)
    i.MD_Connect_BCDTou64                    0x08027e90   Section        0  md_connect.o(i.MD_Connect_BCDTou64)
    i.MD_Connect_DMARX1_IRQHandler           0x08027f30   Section        0  md_connect.o(i.MD_Connect_DMARX1_IRQHandler)
    i.MD_Connect_DMARX2_IRQHandler           0x08027f84   Section        0  md_connect.o(i.MD_Connect_DMARX2_IRQHandler)
    i.MD_Connect_DMARX3_IRQHandler           0x08027fc8   Section        0  md_connect.o(i.MD_Connect_DMARX3_IRQHandler)
    i.MD_Connect_DMARX4_IRQHandler           0x0802800c   Section        0  md_connect.o(i.MD_Connect_DMARX4_IRQHandler)
    i.MD_Connect_DMATX1_IRQHandler           0x08028054   Section        0  md_connect.o(i.MD_Connect_DMATX1_IRQHandler)
    i.MD_Connect_DMATX2_IRQHandler           0x080280b4   Section        0  md_connect.o(i.MD_Connect_DMATX2_IRQHandler)
    i.MD_Connect_DMATX3_IRQHandler           0x08028114   Section        0  md_connect.o(i.MD_Connect_DMATX3_IRQHandler)
    i.MD_Connect_DMATX4_IRQHandler           0x08028178   Section        0  md_connect.o(i.MD_Connect_DMATX4_IRQHandler)
    i.MD_Connect_DMA_Configuration           0x080281dc   Section        0  md_connect.o(i.MD_Connect_DMA_Configuration)
    i.MD_Connect_IO_Configuration            0x0802851c   Section        0  md_connect.o(i.MD_Connect_IO_Configuration)
    i.MD_Connect_Init                        0x08028664   Section        0  md_connect.o(i.MD_Connect_Init)
    i.MD_Connect_NVIC_Configuration          0x080286c4   Section        0  md_connect.o(i.MD_Connect_NVIC_Configuration)
    i.MD_Connect_TXDataCheck                 0x080287b0   Section        0  md_connect.o(i.MD_Connect_TXDataCheck)
    i.MD_Connect_USART_Configuration         0x080287d4   Section        0  md_connect.o(i.MD_Connect_USART_Configuration)
    i.MD_Connect_u64ToBCD                    0x080289f8   Section        0  md_connect.o(i.MD_Connect_u64ToBCD)
    i.MD_Port_Init                           0x08028a6c   Section        0  md_connect.o(i.MD_Port_Init)
    i.MD_Port_LORASet                        0x080294ec   Section        0  md_connect.o(i.MD_Port_LORASet)
    i.Multiplex_PortRXTask                   0x08029860   Section        0  multiplex_port.o(i.Multiplex_PortRXTask)
    i.Multiplex_PortTXTask                   0x0802a034   Section        0  multiplex_port.o(i.Multiplex_PortTXTask)
    i.Multiplex_Port_Choose                  0x0802a830   Section        0  multiplex_port.o(i.Multiplex_Port_Choose)
    i.Multiplex_Port_DMARX_IRQHandler        0x0802a8a4   Section        0  multiplex_port.o(i.Multiplex_Port_DMARX_IRQHandler)
    i.Multiplex_Port_DMATX_IRQHandler        0x0802a8f4   Section        0  multiplex_port.o(i.Multiplex_Port_DMATX_IRQHandler)
    i.Multiplex_Port_DMA_Configuration       0x0802a960   Section        0  multiplex_port.o(i.Multiplex_Port_DMA_Configuration)
    i.Multiplex_Port_IO_Configuration        0x0802aa24   Section        0  multiplex_port.o(i.Multiplex_Port_IO_Configuration)
    i.Multiplex_Port_Init                    0x0802aaa8   Section        0  multiplex_port.o(i.Multiplex_Port_Init)
    i.Multiplex_Port_NVIC_Configuration      0x0802ac54   Section        0  multiplex_port.o(i.Multiplex_Port_NVIC_Configuration)
    i.Multiplex_Port_USART_Configuration     0x0802ac94   Section        0  multiplex_port.o(i.Multiplex_Port_USART_Configuration)
    i.NVIC_Init                              0x0802ad20   Section        0  misc.o(i.NVIC_Init)
    i.NVIC_SetVectorTable                    0x0802ad98   Section        0  misc.o(i.NVIC_SetVectorTable)
    i.OLED_Clear                             0x0802adac   Section        0  oled.o(i.OLED_Clear)
    i.OLED_DrawLine                          0x0802add4   Section        0  oled.o(i.OLED_DrawLine)
    i.OLED_DrawPoint                         0x0802ae80   Section        0  oled.o(i.OLED_DrawPoint)
    i.OLED_Init                              0x0802aef8   Section        0  oled.o(i.OLED_Init)
    i.OLED_Pow                               0x0802b06c   Section        0  oled.o(i.OLED_Pow)
    i.OLED_ProgressBar                       0x0802b082   Section        0  oled.o(i.OLED_ProgressBar)
    i.OLED_Refresh                           0x0802b124   Section        0  oled.o(i.OLED_Refresh)
    i.OLED_SPI2_SendByte                     0x0802b174   Section        0  oled.o(i.OLED_SPI2_SendByte)
    i.OLED_ShowChar                          0x0802b1ac   Section        0  oled.o(i.OLED_ShowChar)
    i.OLED_ShowNum                           0x0802b2e8   Section        0  oled.o(i.OLED_ShowNum)
    i.OLED_ShowPicture                       0x0802b42c   Section        0  oled.o(i.OLED_ShowPicture)
    i.OLED_ShowString                        0x0802b502   Section        0  oled.o(i.OLED_ShowString)
    i.OLED_WR_Byte                           0x0802b554   Section        0  oled.o(i.OLED_WR_Byte)
    i.PCBEncryption_Check                    0x0802b5ac   Section        0  fram.o(i.PCBEncryption_Check)
    i.POS_ConnectRXTask                      0x0802b65c   Section        0  pos_connect.o(i.POS_ConnectRXTask)
    i.POS_ConnectTXTask                      0x080301a4   Section        0  pos_connect.o(i.POS_ConnectTXTask)
    i.POS_Connect_DMARX_IRQHandler           0x0803237c   Section        0  pos_connect.o(i.POS_Connect_DMARX_IRQHandler)
    i.POS_Connect_DMATX_IRQHandler           0x080323f4   Section        0  pos_connect.o(i.POS_Connect_DMATX_IRQHandler)
    i.POS_Connect_DMA_Configuration          0x08032414   Section        0  pos_connect.o(i.POS_Connect_DMA_Configuration)
    i.POS_Connect_IO_Configuration           0x080324d4   Section        0  pos_connect.o(i.POS_Connect_IO_Configuration)
    i.POS_Connect_Init                       0x08032540   Section        0  pos_connect.o(i.POS_Connect_Init)
    i.POS_Connect_NVIC_Configuration         0x080327f4   Section        0  pos_connect.o(i.POS_Connect_NVIC_Configuration)
    i.POS_Connect_USART_Configuration        0x08032834   Section        0  pos_connect.o(i.POS_Connect_USART_Configuration)
    i.Pluse_InPut_EXTI_Configuration         0x08032890   Section        0  pluse_input.o(i.Pluse_InPut_EXTI_Configuration)
    i.Pluse_InPut_IO_Configuration           0x080328f4   Section        0  pluse_input.o(i.Pluse_InPut_IO_Configuration)
    i.Pluse_InPut_IRQHandler                 0x080329e0   Section        0  pluse_input.o(i.Pluse_InPut_IRQHandler)
    i.Pluse_InPut_Init                       0x08032a5c   Section        0  pluse_input.o(i.Pluse_InPut_Init)
    i.Pluse_InPut_NVIC_Configuration         0x08032b1c   Section        0  pluse_input.o(i.Pluse_InPut_NVIC_Configuration)
    i.Pluse_Putout_IO_Configuration          0x08032b58   Section        0  pluse_putout.o(i.Pluse_Putout_IO_Configuration)
    i.Pluse_Putout_Init                      0x08032bf0   Section        0  pluse_putout.o(i.Pluse_Putout_Init)
    i.Price_DataCheck                        0x08032bf8   Section        0  multiplex_port.o(i.Price_DataCheck)
    i.Print_Num                              0x08032c14   Section        0  printf.o(i.Print_Num)
    i.Query376Interrupt                      0x08032d80   Section        0  file_sys.o(i.Query376Interrupt)
    i.RCC_AHB1PeriphClockCmd                 0x08032d98   Section        0  stm32f4xx_rcc.o(i.RCC_AHB1PeriphClockCmd)
    i.RCC_AHB1PeriphResetCmd                 0x08032db8   Section        0  stm32f4xx_rcc.o(i.RCC_AHB1PeriphResetCmd)
    i.RCC_AHB2PeriphClockCmd                 0x08032dd8   Section        0  stm32f4xx_rcc.o(i.RCC_AHB2PeriphClockCmd)
    i.RCC_APB1PeriphClockCmd                 0x08032df8   Section        0  stm32f4xx_rcc.o(i.RCC_APB1PeriphClockCmd)
    i.RCC_APB1PeriphResetCmd                 0x08032e18   Section        0  stm32f4xx_rcc.o(i.RCC_APB1PeriphResetCmd)
    i.RCC_APB2PeriphClockCmd                 0x08032e38   Section        0  stm32f4xx_rcc.o(i.RCC_APB2PeriphClockCmd)
    i.RCC_APB2PeriphResetCmd                 0x08032e58   Section        0  stm32f4xx_rcc.o(i.RCC_APB2PeriphResetCmd)
    i.RCC_GetClocksFreq                      0x08032e78   Section        0  stm32f4xx_rcc.o(i.RCC_GetClocksFreq)
    i.RNG_Cmd                                0x08032f60   Section        0  stm32f4xx_rng.o(i.RNG_Cmd)
    i.RNG_GetRandomNumber                    0x08032f84   Section        0  stm32f4xx_rng.o(i.RNG_GetRandomNumber)
    i.ReadDFStatus                           0x08032f90   Section        0  at45db.o(i.ReadDFStatus)
    i.ReadDriverID                           0x08032fcc   Section        0  at45db.o(i.ReadDriverID)
    i.SPI2_Init                              0x0803305c   Section        0  file_sys.o(i.SPI2_Init)
    i.SPI2_ReadWriteByte                     0x08033144   Section        0  file_sys.o(i.SPI2_ReadWriteByte)
    i.SPI_Cmd                                0x0803317c   Section        0  stm32f4xx_spi.o(i.SPI_Cmd)
    i.SPI_I2S_DeInit                         0x08033194   Section        0  stm32f4xx_spi.o(i.SPI_I2S_DeInit)
    i.SPI_I2S_GetFlagStatus                  0x080331ec   Section        0  stm32f4xx_spi.o(i.SPI_I2S_GetFlagStatus)
    i.SPI_I2S_ReceiveData                    0x080331fe   Section        0  stm32f4xx_spi.o(i.SPI_I2S_ReceiveData)
    i.SPI_I2S_SendData                       0x08033204   Section        0  stm32f4xx_spi.o(i.SPI_I2S_SendData)
    i.SPI_Init                               0x08033208   Section        0  stm32f4xx_spi.o(i.SPI_Init)
    i.SUMCRC                                 0x08033244   Section        0  pos_connect.o(i.SUMCRC)
    i.SYSCFG_EXTILineConfig                  0x08033260   Section        0  stm32f4xx_syscfg.o(i.SYSCFG_EXTILineConfig)
    i.SYSTimer_IRQHandler                    0x080332a0   Section        0  time_count.o(i.SYSTimer_IRQHandler)
    i.SetSysClock                            0x08033378   Section        0  system_stm32f4xx.o(i.SetSysClock)
    SetSysClock                              0x08033379   Thumb Code   216  system_stm32f4xx.o(i.SetSysClock)
    i.Spi376OutByte                          0x08033460   Section        0  file_sys.o(i.Spi376OutByte)
    i.StrToFloat                             0x0803346c   Section        0  md_connect.o(i.StrToFloat)
    i.StrToInt                               0x080334f0   Section        0  md_connect.o(i.StrToInt)
    i.Sureface_Wait_TimeUpData               0x0803353c   Section        0  surface.o(i.Sureface_Wait_TimeUpData)
    i.SurfaceJump                            0x080336d8   Section        0  surface.o(i.SurfaceJump)
    i.SurfaceTast                            0x080336e8   Section        0  surface.o(i.SurfaceTast)
    i.Surface_Copy_16                        0x08035ddc   Section        0  surface.o(i.Surface_Copy_16)
    i.Surface_Init                           0x08035e20   Section        0  surface.o(i.Surface_Init)
    i.SysTick_CLKSourceConfig                0x08035e4c   Section        0  misc.o(i.SysTick_CLKSourceConfig)
    i.SystemInit                             0x08035e74   Section        0  system_stm32f4xx.o(i.SystemInit)
    i.TIM2_IRQHandler                        0x08035edc   Section        0  stm32f4xx_it.o(i.TIM2_IRQHandler)
    i.TIM_ClearFlag                          0x08035ee4   Section        0  stm32f4xx_tim.o(i.TIM_ClearFlag)
    i.TIM_Cmd                                0x08035eea   Section        0  stm32f4xx_tim.o(i.TIM_Cmd)
    i.TIM_DeInit                             0x08035f04   Section        0  stm32f4xx_tim.o(i.TIM_DeInit)
    i.TIM_GetITStatus                        0x08036094   Section        0  stm32f4xx_tim.o(i.TIM_GetITStatus)
    i.TIM_ITConfig                           0x080360b6   Section        0  stm32f4xx_tim.o(i.TIM_ITConfig)
    i.TIM_TimeBaseInit                       0x080360c8   Section        0  stm32f4xx_tim.o(i.TIM_TimeBaseInit)
    i.TXH_Init                               0x0803614c   Section        0  txh.o(i.TXH_Init)
    i.TXH_Task                               0x0803620c   Section        0  txh.o(i.TXH_Task)
    i.Timer_Init                             0x08036ad0   Section        0  time_count.o(i.Timer_Init)
    i.Timer_NVIC_Configuration               0x08036e00   Section        0  time_count.o(i.Timer_NVIC_Configuration)
    i.UART4_IRQHandler                       0x08036e22   Section        0  stm32f4xx_it.o(i.UART4_IRQHandler)
    i.UART5_IRQHandler                       0x08036e2a   Section        0  stm32f4xx_it.o(i.UART5_IRQHandler)
    i.USART1_IRQHandler                      0x08036e32   Section        0  stm32f4xx_it.o(i.USART1_IRQHandler)
    i.USART2_IRQHandler                      0x08036e3a   Section        0  stm32f4xx_it.o(i.USART2_IRQHandler)
    i.USART3_IRQHandler                      0x08036e42   Section        0  stm32f4xx_it.o(i.USART3_IRQHandler)
    i.USART6_IRQHandler                      0x08036e4a   Section        0  stm32f4xx_it.o(i.USART6_IRQHandler)
    i.USART_ClearFlag                        0x08036e52   Section        0  stm32f4xx_usart.o(i.USART_ClearFlag)
    i.USART_Cmd                              0x08036e64   Section        0  stm32f4xx_usart.o(i.USART_Cmd)
    i.USART_DMACmd                           0x08036e7c   Section        0  stm32f4xx_usart.o(i.USART_DMACmd)
    i.USART_DeInit                           0x08036e90   Section        0  stm32f4xx_usart.o(i.USART_DeInit)
    i.USART_GetFlagStatus                    0x08036f44   Section        0  stm32f4xx_usart.o(i.USART_GetFlagStatus)
    i.USART_GetITStatus                      0x08036f5e   Section        0  stm32f4xx_usart.o(i.USART_GetITStatus)
    i.USART_ITConfig                         0x08036fb2   Section        0  stm32f4xx_usart.o(i.USART_ITConfig)
    i.USART_Init                             0x08036ffc   Section        0  stm32f4xx_usart.o(i.USART_Init)
    i.Wait376Interrupt                       0x080370d0   Section        0  file_sys.o(i.Wait376Interrupt)
    i.__0sprintf$8                           0x080370f4   Section        0  printf8.o(i.__0sprintf$8)
    i.__ARM_fpclassify                       0x0803711c   Section        0  fpclassify.o(i.__ARM_fpclassify)
    i.__hardfp_atof                          0x08037150   Section        0  atof.o(i.__hardfp_atof)
    i.__hardfp_log                           0x08037188   Section        0  log.o(i.__hardfp_log)
    i.__hardfp_log10                         0x08037550   Section        0  log10.o(i.__hardfp_log10)
    i.__hardfp_pow                           0x08037680   Section        0  pow.o(i.__hardfp_pow)
    i.__kernel_poly                          0x080382d0   Section        0  poly.o(i.__kernel_poly)
    i.__mathlib_dbl_divzero                  0x080383c8   Section        0  dunder.o(i.__mathlib_dbl_divzero)
    i.__mathlib_dbl_infnan                   0x080383f8   Section        0  dunder.o(i.__mathlib_dbl_infnan)
    i.__mathlib_dbl_infnan2                  0x0803840c   Section        0  dunder.o(i.__mathlib_dbl_infnan2)
    i.__mathlib_dbl_invalid                  0x08038420   Section        0  dunder.o(i.__mathlib_dbl_invalid)
    i.__mathlib_dbl_overflow                 0x08038440   Section        0  dunder.o(i.__mathlib_dbl_overflow)
    i.__mathlib_dbl_underflow                0x08038460   Section        0  dunder.o(i.__mathlib_dbl_underflow)
    i.__read_errno                           0x08038480   Section        0  errno.o(i.__read_errno)
    i.__scatterload_copy                     0x0803848c   Section       14  handlers.o(i.__scatterload_copy)
    i.__scatterload_null                     0x0803849a   Section        2  handlers.o(i.__scatterload_null)
    i.__scatterload_zeroinit                 0x0803849c   Section       14  handlers.o(i.__scatterload_zeroinit)
    i.__set_PRIMASK                          0x080384aa   Section        0  fram.o(i.__set_PRIMASK)
    __set_PRIMASK                            0x080384ab   Thumb Code     6  fram.o(i.__set_PRIMASK)
    i.__set_PRIMASK                          0x080384b0   Section        0  at45db.o(i.__set_PRIMASK)
    __set_PRIMASK                            0x080384b1   Thumb Code     6  at45db.o(i.__set_PRIMASK)
    i.__set_errno                            0x080384b8   Section        0  errno.o(i.__set_errno)
    i._is_digit                              0x080384c4   Section        0  scanf_fp.o(i._is_digit)
    i._printf_core                           0x080384d4   Section        0  printf8.o(i._printf_core)
    _printf_core                             0x080384d5   Thumb Code   984  printf8.o(i._printf_core)
    i._printf_post_padding                   0x080388d8   Section        0  printf8.o(i._printf_post_padding)
    _printf_post_padding                     0x080388d9   Thumb Code    36  printf8.o(i._printf_post_padding)
    i._printf_pre_padding                    0x080388fc   Section        0  printf8.o(i._printf_pre_padding)
    _printf_pre_padding                      0x080388fd   Thumb Code    46  printf8.o(i._printf_pre_padding)
    i._sputc                                 0x0803892a   Section        0  printf8.o(i._sputc)
    _sputc                                   0x0803892b   Thumb Code    10  printf8.o(i._sputc)
    i.delay_init                             0x08038934   Section        0  delay.o(i.delay_init)
    i.delay_ms                               0x08038940   Section        0  delay.o(i.delay_ms)
    i.delay_us                               0x08038984   Section        0  delay.o(i.delay_us)
    i.do_crc                                 0x080389c8   Section        0  md_connect.o(i.do_crc)
    i.fabs                                   0x080389f0   Section        0  fabs.o(i.fabs)
    i.iic_ack                                0x08038a08   Section        0  ds1307.o(i.iic_ack)
    i.iic_noack                              0x08038a48   Section        0  ds1307.o(i.iic_noack)
    i.iic_readbyte                           0x08038a88   Section        0  ds1307.o(i.iic_readbyte)
    i.iic_sendbyte                           0x08038ae8   Section        0  ds1307.o(i.iic_sendbyte)
    i.iic_start                              0x08038b50   Section        0  ds1307.o(i.iic_start)
    i.iic_stop                               0x08038b84   Section        0  ds1307.o(i.iic_stop)
    i.iic_wait4ack                           0x08038bb8   Section        0  ds1307.o(i.iic_wait4ack)
    i.log                                    0x08038c14   Section        0  log.o(i.log)
    i.mInitCH376Host                         0x08038c24   Section        0  file_sys.o(i.mInitCH376Host)
    i.main                                   0x08038c90   Section        0  main.o(i.main)
    i.mystrstr                               0x08038cfc   Section        0  multiplex_port.o(i.mystrstr)
    i.sqrt                                   0x08038d40   Section        0  sqrt.o(i.sqrt)
    i.xReadCH376Data                         0x08038dae   Section        0  file_sys.o(i.xReadCH376Data)
    i.xWriteCH376Cmd                         0x08038dc4   Section        0  file_sys.o(i.xWriteCH376Cmd)
    i.xWriteCH376Data                        0x08038e04   Section        0  file_sys.o(i.xWriteCH376Data)
    .constdata                               0x08038e16   Section       11  txh.o(.constdata)
    .constdata                               0x08038e24   Section     3052  fram.o(.constdata)
    .constdata                               0x08039a10   Section      106  md_connect.o(.constdata)
    .constdata                               0x08039a7c   Section    20386  pos_connect.o(.constdata)
    .constdata                               0x0803ea20   Section      580  at45db.o(.constdata)
    .constdata                               0x0803ec64   Section     7696  oled.o(.constdata)
    .constdata                               0x08040a74   Section     1948  surface.o(.constdata)
    .constdata                               0x08041210   Section      136  pow.o(.constdata)
    bp                                       0x08041210   Data          16  pow.o(.constdata)
    dp_h                                     0x08041220   Data          16  pow.o(.constdata)
    dp_l                                     0x08041230   Data          16  pow.o(.constdata)
    L                                        0x08041240   Data          48  pow.o(.constdata)
    P                                        0x08041270   Data          40  pow.o(.constdata)
    .constdata                               0x08041298   Section       56  log.o(.constdata)
    Lg2                                      0x08041298   Data          24  log.o(.constdata)
    Lg                                       0x080412b0   Data          32  log.o(.constdata)
    .constdata                               0x080412d0   Section        8  qnan.o(.constdata)
    .constdata                               0x080412d8   Section       64  ctype_c.o(.constdata)
    .data                                    0x20000000   Section       16  stm32f4xx_rcc.o(.data)
    APBAHBPrescTable                         0x20000000   Data          16  stm32f4xx_rcc.o(.data)
    .data                                    0x20000010   Section        2  fram.o(.data)
    .data                                    0x20000012   Section      524  md_connect.o(.data)
    .data                                    0x20000220   Section     2059  pos_connect.o(.data)
    .data                                    0x20000a2c   Section        6  at45db.o(.data)
    .data                                    0x20000a38   Section      165  log.o(.data)
    .data                                    0x20000add   Section        5  surface.o(.data)
    .data                                    0x20000ae2   Section     2003  multiplex_port.o(.data)
    .data                                    0x200012b8   Section        4  errno.o(.data)
    _errno                                   0x200012b8   Data           4  errno.o(.data)
    .bss                                     0x200012bc   Section    28260  txh.o(.bss)
    .bss                                     0x20008120   Section     1208  fram.o(.bss)
    .bss                                     0x200085d8   Section     6488  md_connect.o(.bss)
    .bss                                     0x20009f30   Section     4000  pos_connect.o(.bss)
    .bss                                     0x2000aed0   Section      531  at45db.o(.bss)
    .bss                                     0x2000b0e3   Section     1152  oled.o(.bss)
    STACK                                    0x2000b568   Section    16384  startup_stm32f4xx.o(STACK)

    Global Symbols

    Symbol Name                              Value     Ov Type        Size  Object(Section)

    BuildAttributes$$THM_ISAv4$E$P$D$K$B$S$7EM$VFPi3$EXTD16$VFPS$VFMA$PE$A:L22UL41UL21$X:L11$S22US41US21$IEEE1$IW$USESV6$~STKCKD$USESV7$~SHL$OTIME$ROPI$IEEEX$EBA8$MICROLIB$REQ8$PRES8$EABIv2 0x00000000   Number         0  anon$$obj.o ABSOLUTE
    __ARM_use_no_argv                        0x00000000   Number         0  main.o ABSOLUTE
    _printf_a                                0x00000000   Number         0  stubs.o ABSOLUTE
    _printf_c                                0x00000000   Number         0  stubs.o ABSOLUTE
    _printf_charcount                        0x00000000   Number         0  stubs.o ABSOLUTE
    _printf_d                                0x00000000   Number         0  stubs.o ABSOLUTE
    _printf_e                                0x00000000   Number         0  stubs.o ABSOLUTE
    _printf_f                                0x00000000   Number         0  stubs.o ABSOLUTE
    _printf_flags                            0x00000000   Number         0  stubs.o ABSOLUTE
    _printf_fp_dec                           0x00000000   Number         0  stubs.o ABSOLUTE
    _printf_fp_hex                           0x00000000   Number         0  stubs.o ABSOLUTE
    _printf_g                                0x00000000   Number         0  stubs.o ABSOLUTE
    _printf_i                                0x00000000   Number         0  stubs.o ABSOLUTE
    _printf_int_dec                          0x00000000   Number         0  stubs.o ABSOLUTE
    _printf_l                                0x00000000   Number         0  stubs.o ABSOLUTE
    _printf_lc                               0x00000000   Number         0  stubs.o ABSOLUTE
    _printf_ll                               0x00000000   Number         0  stubs.o ABSOLUTE
    _printf_lld                              0x00000000   Number         0  stubs.o ABSOLUTE
    _printf_lli                              0x00000000   Number         0  stubs.o ABSOLUTE
    _printf_llo                              0x00000000   Number         0  stubs.o ABSOLUTE
    _printf_llu                              0x00000000   Number         0  stubs.o ABSOLUTE
    _printf_llx                              0x00000000   Number         0  stubs.o ABSOLUTE
    _printf_longlong_dec                     0x00000000   Number         0  stubs.o ABSOLUTE
    _printf_longlong_hex                     0x00000000   Number         0  stubs.o ABSOLUTE
    _printf_longlong_oct                     0x00000000   Number         0  stubs.o ABSOLUTE
    _printf_ls                               0x00000000   Number         0  stubs.o ABSOLUTE
    _printf_mbtowc                           0x00000000   Number         0  stubs.o ABSOLUTE
    _printf_n                                0x00000000   Number         0  stubs.o ABSOLUTE
    _printf_o                                0x00000000   Number         0  stubs.o ABSOLUTE
    _printf_p                                0x00000000   Number         0  stubs.o ABSOLUTE
    _printf_percent                          0x00000000   Number         0  stubs.o ABSOLUTE
    _printf_pre_padding                      0x00000000   Number         0  stubs.o ABSOLUTE
    _printf_return_value                     0x00000000   Number         0  stubs.o ABSOLUTE
    _printf_s                                0x00000000   Number         0  stubs.o ABSOLUTE
    _printf_sizespec                         0x00000000   Number         0  stubs.o ABSOLUTE
    _printf_str                              0x00000000   Number         0  stubs.o ABSOLUTE
    _printf_truncate_signed                  0x00000000   Number         0  stubs.o ABSOLUTE
    _printf_truncate_unsigned                0x00000000   Number         0  stubs.o ABSOLUTE
    _printf_u                                0x00000000   Number         0  stubs.o ABSOLUTE
    _printf_wc                               0x00000000   Number         0  stubs.o ABSOLUTE
    _printf_wctomb                           0x00000000   Number         0  stubs.o ABSOLUTE
    _printf_widthprec                        0x00000000   Number         0  stubs.o ABSOLUTE
    _printf_x                                0x00000000   Number         0  stubs.o ABSOLUTE
    __arm_fini_                               - Undefined Weak Reference
    __cpp_initialize__aeabi_                  - Undefined Weak Reference
    __cxa_finalize                            - Undefined Weak Reference
    _clock_init                               - Undefined Weak Reference
    _microlib_exit                            - Undefined Weak Reference
    __Vectors_Size                           0x00000188   Number         0  startup_stm32f4xx.o ABSOLUTE
    __Vectors                                0x08008000   Data           4  startup_stm32f4xx.o(RESET)
    __Vectors_End                            0x08008188   Data           0  startup_stm32f4xx.o(RESET)
    __main                                   0x08008189   Thumb Code     0  entry.o(.ARM.Collect$$$$00000000)
    _main_stk                                0x08008189   Thumb Code     0  entry2.o(.ARM.Collect$$$$00000001)
    _main_scatterload                        0x0800818d   Thumb Code     0  entry5.o(.ARM.Collect$$$$00000004)
    __main_after_scatterload                 0x08008191   Thumb Code     0  entry5.o(.ARM.Collect$$$$00000004)
    _main_clock                              0x08008191   Thumb Code     0  entry7b.o(.ARM.Collect$$$$00000008)
    _main_cpp_init                           0x08008191   Thumb Code     0  entry8b.o(.ARM.Collect$$$$0000000A)
    _main_init                               0x08008191   Thumb Code     0  entry9a.o(.ARM.Collect$$$$0000000B)
    __rt_lib_shutdown_fini                   0x08008199   Thumb Code     0  entry12b.o(.ARM.Collect$$$$0000000E)
    __rt_final_cpp                           0x0800819d   Thumb Code     0  entry10a.o(.ARM.Collect$$$$0000000F)
    __rt_final_exit                          0x0800819d   Thumb Code     0  entry11a.o(.ARM.Collect$$$$00000011)
    Reset_Handler                            0x080081a1   Thumb Code     8  startup_stm32f4xx.o(.text)
    NMI_Handler                              0x080081a9   Thumb Code     2  startup_stm32f4xx.o(.text)
    MemManage_Handler                        0x080081ad   Thumb Code     2  startup_stm32f4xx.o(.text)
    BusFault_Handler                         0x080081af   Thumb Code     2  startup_stm32f4xx.o(.text)
    UsageFault_Handler                       0x080081b1   Thumb Code     2  startup_stm32f4xx.o(.text)
    SVC_Handler                              0x080081b3   Thumb Code     2  startup_stm32f4xx.o(.text)
    DebugMon_Handler                         0x080081b5   Thumb Code     2  startup_stm32f4xx.o(.text)
    PendSV_Handler                           0x080081b7   Thumb Code     2  startup_stm32f4xx.o(.text)
    SysTick_Handler                          0x080081b9   Thumb Code     2  startup_stm32f4xx.o(.text)
    ADC_IRQHandler                           0x080081bb   Thumb Code     0  startup_stm32f4xx.o(.text)
    CAN1_RX0_IRQHandler                      0x080081bb   Thumb Code     0  startup_stm32f4xx.o(.text)
    CAN1_RX1_IRQHandler                      0x080081bb   Thumb Code     0  startup_stm32f4xx.o(.text)
    CAN1_SCE_IRQHandler                      0x080081bb   Thumb Code     0  startup_stm32f4xx.o(.text)
    CAN1_TX_IRQHandler                       0x080081bb   Thumb Code     0  startup_stm32f4xx.o(.text)
    CAN2_RX0_IRQHandler                      0x080081bb   Thumb Code     0  startup_stm32f4xx.o(.text)
    CAN2_RX1_IRQHandler                      0x080081bb   Thumb Code     0  startup_stm32f4xx.o(.text)
    CAN2_SCE_IRQHandler                      0x080081bb   Thumb Code     0  startup_stm32f4xx.o(.text)
    CAN2_TX_IRQHandler                       0x080081bb   Thumb Code     0  startup_stm32f4xx.o(.text)
    CRYP_IRQHandler                          0x080081bb   Thumb Code     0  startup_stm32f4xx.o(.text)
    DCMI_IRQHandler                          0x080081bb   Thumb Code     0  startup_stm32f4xx.o(.text)
    DMA1_Stream0_IRQHandler                  0x080081bb   Thumb Code     0  startup_stm32f4xx.o(.text)
    DMA1_Stream1_IRQHandler                  0x080081bb   Thumb Code     0  startup_stm32f4xx.o(.text)
    DMA1_Stream2_IRQHandler                  0x080081bb   Thumb Code     0  startup_stm32f4xx.o(.text)
    DMA1_Stream5_IRQHandler                  0x080081bb   Thumb Code     0  startup_stm32f4xx.o(.text)
    DMA2_Stream0_IRQHandler                  0x080081bb   Thumb Code     0  startup_stm32f4xx.o(.text)
    DMA2_Stream1_IRQHandler                  0x080081bb   Thumb Code     0  startup_stm32f4xx.o(.text)
    DMA2_Stream2_IRQHandler                  0x080081bb   Thumb Code     0  startup_stm32f4xx.o(.text)
    DMA2_Stream3_IRQHandler                  0x080081bb   Thumb Code     0  startup_stm32f4xx.o(.text)
    DMA2_Stream4_IRQHandler                  0x080081bb   Thumb Code     0  startup_stm32f4xx.o(.text)
    DMA2_Stream5_IRQHandler                  0x080081bb   Thumb Code     0  startup_stm32f4xx.o(.text)
    ETH_IRQHandler                           0x080081bb   Thumb Code     0  startup_stm32f4xx.o(.text)
    ETH_WKUP_IRQHandler                      0x080081bb   Thumb Code     0  startup_stm32f4xx.o(.text)
    EXTI2_IRQHandler                         0x080081bb   Thumb Code     0  startup_stm32f4xx.o(.text)
    EXTI3_IRQHandler                         0x080081bb   Thumb Code     0  startup_stm32f4xx.o(.text)
    EXTI4_IRQHandler                         0x080081bb   Thumb Code     0  startup_stm32f4xx.o(.text)
    EXTI9_5_IRQHandler                       0x080081bb   Thumb Code     0  startup_stm32f4xx.o(.text)
    FLASH_IRQHandler                         0x080081bb   Thumb Code     0  startup_stm32f4xx.o(.text)
    FPU_IRQHandler                           0x080081bb   Thumb Code     0  startup_stm32f4xx.o(.text)
    FSMC_IRQHandler                          0x080081bb   Thumb Code     0  startup_stm32f4xx.o(.text)
    HASH_RNG_IRQHandler                      0x080081bb   Thumb Code     0  startup_stm32f4xx.o(.text)
    I2C1_ER_IRQHandler                       0x080081bb   Thumb Code     0  startup_stm32f4xx.o(.text)
    I2C1_EV_IRQHandler                       0x080081bb   Thumb Code     0  startup_stm32f4xx.o(.text)
    I2C2_ER_IRQHandler                       0x080081bb   Thumb Code     0  startup_stm32f4xx.o(.text)
    I2C2_EV_IRQHandler                       0x080081bb   Thumb Code     0  startup_stm32f4xx.o(.text)
    I2C3_ER_IRQHandler                       0x080081bb   Thumb Code     0  startup_stm32f4xx.o(.text)
    I2C3_EV_IRQHandler                       0x080081bb   Thumb Code     0  startup_stm32f4xx.o(.text)
    OTG_FS_IRQHandler                        0x080081bb   Thumb Code     0  startup_stm32f4xx.o(.text)
    OTG_FS_WKUP_IRQHandler                   0x080081bb   Thumb Code     0  startup_stm32f4xx.o(.text)
    OTG_HS_EP1_IN_IRQHandler                 0x080081bb   Thumb Code     0  startup_stm32f4xx.o(.text)
    OTG_HS_EP1_OUT_IRQHandler                0x080081bb   Thumb Code     0  startup_stm32f4xx.o(.text)
    OTG_HS_IRQHandler                        0x080081bb   Thumb Code     0  startup_stm32f4xx.o(.text)
    OTG_HS_WKUP_IRQHandler                   0x080081bb   Thumb Code     0  startup_stm32f4xx.o(.text)
    PVD_IRQHandler                           0x080081bb   Thumb Code     0  startup_stm32f4xx.o(.text)
    RCC_IRQHandler                           0x080081bb   Thumb Code     0  startup_stm32f4xx.o(.text)
    RTC_Alarm_IRQHandler                     0x080081bb   Thumb Code     0  startup_stm32f4xx.o(.text)
    RTC_WKUP_IRQHandler                      0x080081bb   Thumb Code     0  startup_stm32f4xx.o(.text)
    SDIO_IRQHandler                          0x080081bb   Thumb Code     0  startup_stm32f4xx.o(.text)
    SPI1_IRQHandler                          0x080081bb   Thumb Code     0  startup_stm32f4xx.o(.text)
    SPI2_IRQHandler                          0x080081bb   Thumb Code     0  startup_stm32f4xx.o(.text)
    SPI3_IRQHandler                          0x080081bb   Thumb Code     0  startup_stm32f4xx.o(.text)
    TAMP_STAMP_IRQHandler                    0x080081bb   Thumb Code     0  startup_stm32f4xx.o(.text)
    TIM1_BRK_TIM9_IRQHandler                 0x080081bb   Thumb Code     0  startup_stm32f4xx.o(.text)
    TIM1_CC_IRQHandler                       0x080081bb   Thumb Code     0  startup_stm32f4xx.o(.text)
    TIM1_TRG_COM_TIM11_IRQHandler            0x080081bb   Thumb Code     0  startup_stm32f4xx.o(.text)
    TIM1_UP_TIM10_IRQHandler                 0x080081bb   Thumb Code     0  startup_stm32f4xx.o(.text)
    TIM3_IRQHandler                          0x080081bb   Thumb Code     0  startup_stm32f4xx.o(.text)
    TIM4_IRQHandler                          0x080081bb   Thumb Code     0  startup_stm32f4xx.o(.text)
    TIM5_IRQHandler                          0x080081bb   Thumb Code     0  startup_stm32f4xx.o(.text)
    TIM6_DAC_IRQHandler                      0x080081bb   Thumb Code     0  startup_stm32f4xx.o(.text)
    TIM7_IRQHandler                          0x080081bb   Thumb Code     0  startup_stm32f4xx.o(.text)
    TIM8_BRK_TIM12_IRQHandler                0x080081bb   Thumb Code     0  startup_stm32f4xx.o(.text)
    TIM8_CC_IRQHandler                       0x080081bb   Thumb Code     0  startup_stm32f4xx.o(.text)
    TIM8_TRG_COM_TIM14_IRQHandler            0x080081bb   Thumb Code     0  startup_stm32f4xx.o(.text)
    TIM8_UP_TIM13_IRQHandler                 0x080081bb   Thumb Code     0  startup_stm32f4xx.o(.text)
    WWDG_IRQHandler                          0x080081bb   Thumb Code     0  startup_stm32f4xx.o(.text)
    __aeabi_ldivmod                          0x080081c5   Thumb Code    98  ldiv.o(.text)
    __aeabi_lasr                             0x08008227   Thumb Code    36  llsshr.o(.text)
    _ll_sshift_r                             0x08008227   Thumb Code     0  llsshr.o(.text)
    __aeabi_memcpy                           0x0800824b   Thumb Code    36  memcpya.o(.text)
    __aeabi_memcpy4                          0x0800824b   Thumb Code     0  memcpya.o(.text)
    __aeabi_memcpy8                          0x0800824b   Thumb Code     0  memcpya.o(.text)
    strcat                                   0x0800826f   Thumb Code    24  strcat.o(.text)
    strlen                                   0x08008287   Thumb Code    14  strlen.o(.text)
    strncmp                                  0x08008295   Thumb Code    30  strncmp.o(.text)
    __aeabi_dadd                             0x080082b3   Thumb Code   322  dadd.o(.text)
    __aeabi_dsub                             0x080083f5   Thumb Code     6  dadd.o(.text)
    __aeabi_drsub                            0x080083fb   Thumb Code     6  dadd.o(.text)
    __aeabi_dmul                             0x08008401   Thumb Code   228  dmul.o(.text)
    __aeabi_ddiv                             0x080084e5   Thumb Code   222  ddiv.o(.text)
    __aeabi_l2f                              0x080085c3   Thumb Code    44  ffltl.o(.text)
    __aeabi_i2d                              0x080085ef   Thumb Code    34  dflti.o(.text)
    __aeabi_ui2d                             0x08008611   Thumb Code    26  dfltui.o(.text)
    __aeabi_l2d                              0x0800862b   Thumb Code    40  dfltl.o(.text)
    __aeabi_f2lz                             0x08008653   Thumb Code    66  ffixl.o(.text)
    __aeabi_d2iz                             0x08008695   Thumb Code    62  dfixi.o(.text)
    __aeabi_d2lz                             0x080086d3   Thumb Code    74  dfixl.o(.text)
    __aeabi_f2d                              0x0800871d   Thumb Code    38  f2d.o(.text)
    __aeabi_d2f                              0x08008743   Thumb Code    56  d2f.o(.text)
    __aeabi_uldivmod                         0x0800877b   Thumb Code    98  uldiv.o(.text)
    __aeabi_llsl                             0x080087dd   Thumb Code    30  llshl.o(.text)
    _ll_shift_l                              0x080087dd   Thumb Code     0  llshl.o(.text)
    __aeabi_llsr                             0x080087fb   Thumb Code    32  llushr.o(.text)
    _ll_ushift_r                             0x080087fb   Thumb Code     0  llushr.o(.text)
    __strtod_int                             0x08008853   Thumb Code    90  strtod.o(.text)
    __I$use$fp                               0x080088b9   Thumb Code     0  iusefp.o(.text)
    _float_round                             0x080088b9   Thumb Code    18  fepilogue.o(.text)
    _float_epilogue                          0x080088cb   Thumb Code    92  fepilogue.o(.text)
    _double_round                            0x08008927   Thumb Code    30  depilogue.o(.text)
    _double_epilogue                         0x08008945   Thumb Code   156  depilogue.o(.text)
    __ARM_scalbn                             0x080089e1   Thumb Code    46  dscalb.o(.text)
    scalbn                                   0x080089e1   Thumb Code     0  dscalb.o(.text)
    __aeabi_cdrcmple                         0x08008a11   Thumb Code    48  cdrcmple.o(.text)
    __scatterload                            0x08008a41   Thumb Code    28  init.o(.text)
    __scatterload_rt2                        0x08008a41   Thumb Code     0  init.o(.text)
    isspace                                  0x08008a65   Thumb Code    10  isspace_c.o(.text)
    _scanf_real                              0x08008b99   Thumb Code     0  scanf_fp.o(.text)
    _scanf_really_real                       0x08008b99   Thumb Code   556  scanf_fp.o(.text)
    _sgetc                                   0x08008dd1   Thumb Code    30  _sgetc.o(.text)
    _sbackspace                              0x08008def   Thumb Code    34  _sgetc.o(.text)
    _dsqrt                                   0x08008e11   Thumb Code   162  dsqrt.o(.text)
    __aeabi_cdcmpeq                          0x08008eb5   Thumb Code     0  cdcmple.o(.text)
    __aeabi_cdcmple                          0x08008eb5   Thumb Code    48  cdcmple.o(.text)
    __ctype_lookup                           0x08008ee5   Thumb Code    34  ctype_c.o(.text)
    __aeabi_ul2d                             0x08008f0d   Thumb Code    24  dfltul.o(.text)
    __decompress                             0x08008f25   Thumb Code     0  __dczerorl2.o(.text)
    __decompress1                            0x08008f25   Thumb Code    86  __dczerorl2.o(.text)
    AT45DBDataCheck                          0x08008f7b   Thumb Code    28  at45db.o(i.AT45DBDataCheck)
    AT45DBItemRead                           0x08008f99   Thumb Code   300  at45db.o(i.AT45DBItemRead)
    AT45DBItemWrite                          0x080090d1   Thumb Code   226  at45db.o(i.AT45DBItemWrite)
    AT45DB_Init                              0x080091b9   Thumb Code    70  at45db.o(i.AT45DB_Init)
    AT45DB_ReadPage                          0x08009209   Thumb Code   184  at45db.o(i.AT45DB_ReadPage)
    AT45DB_SendByte                          0x080092c9   Thumb Code    50  at45db.o(i.AT45DB_SendByte)
    AT45DB_SetPageByte                       0x08009301   Thumb Code   130  at45db.o(i.AT45DB_SetPageByte)
    AT45DB_WriteBuff                         0x0800938d   Thumb Code   154  at45db.o(i.AT45DB_WriteBuff)
    AT45DB_WritePage                         0x08009431   Thumb Code   154  at45db.o(i.AT45DB_WritePage)
    BCC_CheckSum                             0x080094d5   Thumb Code    26  md_connect.o(i.BCC_CheckSum)
    Bluesky_Decrypt                          0x080094ef   Thumb Code    20  md_connect.o(i.Bluesky_Decrypt)
    Bluesky_Encrypt                          0x08009503   Thumb Code    96  md_connect.o(i.Bluesky_Encrypt)
    CH376ByteLocate                          0x08009565   Thumb Code    54  file_sys.o(i.CH376ByteLocate)
    CH376ByteRead                            0x080095a1   Thumb Code    94  file_sys.o(i.CH376ByteRead)
    CH376ByteWrite                           0x08009605   Thumb Code   100  file_sys.o(i.CH376ByteWrite)
    CH376DiskConnect                         0x0800966d   Thumb Code    20  file_sys.o(i.CH376DiskConnect)
    CH376FileClose                           0x08009681   Thumb Code    14  file_sys.o(i.CH376FileClose)
    CH376FileCreate                          0x0800968f   Thumb Code    20  file_sys.o(i.CH376FileCreate)
    CH376FileOpen                            0x080096a3   Thumb Code    38  file_sys.o(i.CH376FileOpen)
    CH376GetFileSize                         0x080096c9   Thumb Code    10  file_sys.o(i.CH376GetFileSize)
    CH376GetIntStatus                        0x080096d5   Thumb Code    28  file_sys.o(i.CH376GetIntStatus)
    CH376Read32bitDat                        0x080096f5   Thumb Code    54  file_sys.o(i.CH376Read32bitDat)
    CH376ReadBlock                           0x08009731   Thumb Code    52  file_sys.o(i.CH376ReadBlock)
    CH376ReadVar32                           0x08009769   Thumb Code    22  file_sys.o(i.CH376ReadVar32)
    CH376ReadVar8                            0x08009781   Thumb Code    36  file_sys.o(i.CH376ReadVar8)
    CH376SendCmdDatWaitInt                   0x080097a9   Thumb Code    34  file_sys.o(i.CH376SendCmdDatWaitInt)
    CH376SendCmdWaitInt                      0x080097d1   Thumb Code    26  file_sys.o(i.CH376SendCmdWaitInt)
    CH376SetFileName                         0x080097f1   Thumb Code   162  file_sys.o(i.CH376SetFileName)
    CH376WriteReqBlock                       0x08009899   Thumb Code    52  file_sys.o(i.CH376WriteReqBlock)
    CH376WriteVar32                          0x080098d1   Thumb Code    58  file_sys.o(i.CH376WriteVar32)
    CRC_Check                                0x08009911   Thumb Code    48  pos_connect.o(i.CRC_Check)
    CheckSum                                 0x08009949   Thumb Code    70  md_connect.o(i.CheckSum)
    CheckSum8                                0x0800998f   Thumb Code    28  md_connect.o(i.CheckSum8)
    DMA1_Stream3_IRQHandler                  0x080099ab   Thumb Code     8  stm32f4xx_it.o(i.DMA1_Stream3_IRQHandler)
    DMA1_Stream4_IRQHandler                  0x080099b3   Thumb Code     8  stm32f4xx_it.o(i.DMA1_Stream4_IRQHandler)
    DMA1_Stream6_IRQHandler                  0x080099bb   Thumb Code     8  stm32f4xx_it.o(i.DMA1_Stream6_IRQHandler)
    DMA1_Stream7_IRQHandler                  0x080099c3   Thumb Code     8  stm32f4xx_it.o(i.DMA1_Stream7_IRQHandler)
    DMA2_Stream6_IRQHandler                  0x080099cb   Thumb Code     8  stm32f4xx_it.o(i.DMA2_Stream6_IRQHandler)
    DMA2_Stream7_IRQHandler                  0x080099d3   Thumb Code     8  stm32f4xx_it.o(i.DMA2_Stream7_IRQHandler)
    DMA_ClearFlag                            0x080099dd   Thumb Code    38  stm32f4xx_dma.o(i.DMA_ClearFlag)
    DMA_Cmd                                  0x08009a11   Thumb Code    22  stm32f4xx_dma.o(i.DMA_Cmd)
    DMA_DeInit                               0x08009a29   Thumb Code   324  stm32f4xx_dma.o(i.DMA_DeInit)
    DMA_ITConfig                             0x08009b81   Thumb Code    58  stm32f4xx_dma.o(i.DMA_ITConfig)
    DMA_Init                                 0x08009bbd   Thumb Code    82  stm32f4xx_dma.o(i.DMA_Init)
    DS1307_Init                              0x08009c15   Thumb Code   134  ds1307.o(i.DS1307_Init)
    DS1307_Read                              0x08009cad   Thumb Code   126  ds1307.o(i.DS1307_Read)
    DS1307_Write                             0x08009d35   Thumb Code   114  ds1307.o(i.DS1307_Write)
    DartCRC16                                0x08009db1   Thumb Code    48  pos_connect.o(i.DartCRC16)
    Decode_Data                              0x08009de9   Thumb Code    48  pos_connect.o(i.Decode_Data)
    EXTI0_IRQHandler                         0x08009e19   Thumb Code     8  stm32f4xx_it.o(i.EXTI0_IRQHandler)
    EXTI15_10_IRQHandler                     0x08009e21   Thumb Code     8  stm32f4xx_it.o(i.EXTI15_10_IRQHandler)
    EXTI1_IRQHandler                         0x08009e29   Thumb Code     8  stm32f4xx_it.o(i.EXTI1_IRQHandler)
    EXTI_ClearITPendingBit                   0x08009e31   Thumb Code     6  stm32f4xx_exti.o(i.EXTI_ClearITPendingBit)
    EXTI_GetITStatus                         0x08009e3d   Thumb Code    34  stm32f4xx_exti.o(i.EXTI_GetITStatus)
    EXTI_Init                                0x08009e65   Thumb Code   142  stm32f4xx_exti.o(i.EXTI_Init)
    Encrypt_Data                             0x08009ef9   Thumb Code    48  pos_connect.o(i.Encrypt_Data)
    FMItemRead                               0x08009f29   Thumb Code   378  fram.o(i.FMItemRead)
    FMItemWrite                              0x0800a0ad   Thumb Code   318  fram.o(i.FMItemWrite)
    FM_Data_Init                             0x0800a1f9   Thumb Code   326  fram.o(i.FM_Data_Init)
    FM_IO_Configuration                      0x0800a351   Thumb Code   124  fram.o(i.FM_IO_Configuration)
    FM_Init                                  0x0800a3d1   Thumb Code   216  fram.o(i.FM_Init)
    FM_ReadData                              0x0800a4bd   Thumb Code   102  fram.o(i.FM_ReadData)
    FM_SPI1_SendByte                         0x0800a529   Thumb Code    50  fram.o(i.FM_SPI1_SendByte)
    FM_SPI_Configuration                     0x0800a561   Thumb Code    90  fram.o(i.FM_SPI_Configuration)
    FM_WriteData                             0x0800a5c1   Thumb Code   130  fram.o(i.FM_WriteData)
    FRamDataCheck                            0x0800a649   Thumb Code    28  fram.o(i.FRamDataCheck)
    FindKey                                  0x0800a665   Thumb Code   180  surface.o(i.FindKey)
    FindSysconfigFile                        0x0800a739   Thumb Code   510  log.o(i.FindSysconfigFile)
    GPIO_DeInit                              0x0800a989   Thumb Code   220  stm32f4xx_gpio.o(i.GPIO_DeInit)
    GPIO_Init                                0x0800aa89   Thumb Code   144  stm32f4xx_gpio.o(i.GPIO_Init)
    GPIO_PinAFConfig                         0x0800ab19   Thumb Code    70  stm32f4xx_gpio.o(i.GPIO_PinAFConfig)
    GPIO_ReadInputDataBit                    0x0800ab5f   Thumb Code    18  stm32f4xx_gpio.o(i.GPIO_ReadInputDataBit)
    GPIO_ResetBits                           0x0800ab71   Thumb Code     4  stm32f4xx_gpio.o(i.GPIO_ResetBits)
    GPIO_SetBits                             0x0800ab75   Thumb Code     4  stm32f4xx_gpio.o(i.GPIO_SetBits)
    GetKeyNum                                0x0800ab79   Thumb Code    12  surface.o(i.GetKeyNum)
    HardFault_Handler                        0x0800ab89   Thumb Code    58  stm32f4xx_it.o(i.HardFault_Handler)
    IWDG_ReloadCounter                       0x0800abcd   Thumb Code    10  stm32f4xx_iwdg.o(i.IWDG_ReloadCounter)
    InteiHEXCheck                            0x0800abdd   Thumb Code    32  md_connect.o(i.InteiHEXCheck)
    Log_Init                                 0x0800abfd   Thumb Code    16  log.o(i.Log_Init)
    Log_Task                                 0x0800ac0d   Thumb Code   592  log.o(i.Log_Task)
    MD_ConnectRXTask                         0x0800ae75   Thumb Code 82732  md_connect.o(i.MD_ConnectRXTask)
    MD_ConnectTXTask                         0x0801f1cd   Thumb Code 36024  md_connect.o(i.MD_ConnectTXTask)
    MD_Connect_BCDTou64                      0x08027e91   Thumb Code   152  md_connect.o(i.MD_Connect_BCDTou64)
    MD_Connect_DMARX1_IRQHandler             0x08027f31   Thumb Code    66  md_connect.o(i.MD_Connect_DMARX1_IRQHandler)
    MD_Connect_DMARX2_IRQHandler             0x08027f85   Thumb Code    52  md_connect.o(i.MD_Connect_DMARX2_IRQHandler)
    MD_Connect_DMARX3_IRQHandler             0x08027fc9   Thumb Code    50  md_connect.o(i.MD_Connect_DMARX3_IRQHandler)
    MD_Connect_DMARX4_IRQHandler             0x0802800d   Thumb Code    54  md_connect.o(i.MD_Connect_DMARX4_IRQHandler)
    MD_Connect_DMATX1_IRQHandler             0x08028055   Thumb Code    72  md_connect.o(i.MD_Connect_DMATX1_IRQHandler)
    MD_Connect_DMATX2_IRQHandler             0x080280b5   Thumb Code    72  md_connect.o(i.MD_Connect_DMATX2_IRQHandler)
    MD_Connect_DMATX3_IRQHandler             0x08028115   Thumb Code    74  md_connect.o(i.MD_Connect_DMATX3_IRQHandler)
    MD_Connect_DMATX4_IRQHandler             0x08028179   Thumb Code    74  md_connect.o(i.MD_Connect_DMATX4_IRQHandler)
    MD_Connect_DMA_Configuration             0x080281dd   Thumb Code   780  md_connect.o(i.MD_Connect_DMA_Configuration)
    MD_Connect_IO_Configuration              0x0802851d   Thumb Code   310  md_connect.o(i.MD_Connect_IO_Configuration)
    MD_Connect_Init                          0x08028665   Thumb Code    84  md_connect.o(i.MD_Connect_Init)
    MD_Connect_NVIC_Configuration            0x080286c5   Thumb Code   236  md_connect.o(i.MD_Connect_NVIC_Configuration)
    MD_Connect_TXDataCheck                   0x080287b1   Thumb Code    34  md_connect.o(i.MD_Connect_TXDataCheck)
    MD_Connect_USART_Configuration           0x080287d5   Thumb Code   532  md_connect.o(i.MD_Connect_USART_Configuration)
    MD_Connect_u64ToBCD                      0x080289f9   Thumb Code   116  md_connect.o(i.MD_Connect_u64ToBCD)
    MD_Port_Init                             0x08028a6d   Thumb Code  2670  md_connect.o(i.MD_Port_Init)
    MD_Port_LORASet                          0x080294ed   Thumb Code   830  md_connect.o(i.MD_Port_LORASet)
    Multiplex_PortRXTask                     0x08029861   Thumb Code  1972  multiplex_port.o(i.Multiplex_PortRXTask)
    Multiplex_PortTXTask                     0x0802a035   Thumb Code  2014  multiplex_port.o(i.Multiplex_PortTXTask)
    Multiplex_Port_Choose                    0x0802a831   Thumb Code   112  multiplex_port.o(i.Multiplex_Port_Choose)
    Multiplex_Port_DMARX_IRQHandler          0x0802a8a5   Thumb Code    68  multiplex_port.o(i.Multiplex_Port_DMARX_IRQHandler)
    Multiplex_Port_DMATX_IRQHandler          0x0802a8f5   Thumb Code    84  multiplex_port.o(i.Multiplex_Port_DMATX_IRQHandler)
    Multiplex_Port_DMA_Configuration         0x0802a961   Thumb Code   178  multiplex_port.o(i.Multiplex_Port_DMA_Configuration)
    Multiplex_Port_IO_Configuration          0x0802aa25   Thumb Code   126  multiplex_port.o(i.Multiplex_Port_IO_Configuration)
    Multiplex_Port_Init                      0x0802aaa9   Thumb Code   416  multiplex_port.o(i.Multiplex_Port_Init)
    Multiplex_Port_NVIC_Configuration        0x0802ac55   Thumb Code    62  multiplex_port.o(i.Multiplex_Port_NVIC_Configuration)
    Multiplex_Port_USART_Configuration       0x0802ac95   Thumb Code   134  multiplex_port.o(i.Multiplex_Port_USART_Configuration)
    NVIC_Init                                0x0802ad21   Thumb Code   106  misc.o(i.NVIC_Init)
    NVIC_SetVectorTable                      0x0802ad99   Thumb Code    12  misc.o(i.NVIC_SetVectorTable)
    OLED_Clear                               0x0802adad   Thumb Code    36  oled.o(i.OLED_Clear)
    OLED_DrawLine                            0x0802add5   Thumb Code   172  oled.o(i.OLED_DrawLine)
    OLED_DrawPoint                           0x0802ae81   Thumb Code   114  oled.o(i.OLED_DrawPoint)
    OLED_Init                                0x0802aef9   Thumb Code   360  oled.o(i.OLED_Init)
    OLED_Pow                                 0x0802b06d   Thumb Code    22  oled.o(i.OLED_Pow)
    OLED_ProgressBar                         0x0802b083   Thumb Code   162  oled.o(i.OLED_ProgressBar)
    OLED_Refresh                             0x0802b125   Thumb Code    74  oled.o(i.OLED_Refresh)
    OLED_SPI2_SendByte                       0x0802b175   Thumb Code    50  oled.o(i.OLED_SPI2_SendByte)
    OLED_ShowChar                            0x0802b1ad   Thumb Code   300  oled.o(i.OLED_ShowChar)
    OLED_ShowNum                             0x0802b2e9   Thumb Code   314  oled.o(i.OLED_ShowNum)
    OLED_ShowPicture                         0x0802b42d   Thumb Code   214  oled.o(i.OLED_ShowPicture)
    OLED_ShowString                          0x0802b503   Thumb Code    80  oled.o(i.OLED_ShowString)
    OLED_WR_Byte                             0x0802b555   Thumb Code    78  oled.o(i.OLED_WR_Byte)
    PCBEncryption_Check                      0x0802b5ad   Thumb Code   164  fram.o(i.PCBEncryption_Check)
    POS_ConnectRXTask                        0x0802b65d   Thumb Code 19248  pos_connect.o(i.POS_ConnectRXTask)
    POS_ConnectTXTask                        0x080301a5   Thumb Code  8664  pos_connect.o(i.POS_ConnectTXTask)
    POS_Connect_DMARX_IRQHandler             0x0803237d   Thumb Code    98  pos_connect.o(i.POS_Connect_DMARX_IRQHandler)
    POS_Connect_DMATX_IRQHandler             0x080323f5   Thumb Code    22  pos_connect.o(i.POS_Connect_DMATX_IRQHandler)
    POS_Connect_DMA_Configuration            0x08032415   Thumb Code   174  pos_connect.o(i.POS_Connect_DMA_Configuration)
    POS_Connect_IO_Configuration             0x080324d5   Thumb Code   104  pos_connect.o(i.POS_Connect_IO_Configuration)
    POS_Connect_Init                         0x08032541   Thumb Code   604  pos_connect.o(i.POS_Connect_Init)
    POS_Connect_NVIC_Configuration           0x080327f5   Thumb Code    62  pos_connect.o(i.POS_Connect_NVIC_Configuration)
    POS_Connect_USART_Configuration          0x08032835   Thumb Code    86  pos_connect.o(i.POS_Connect_USART_Configuration)
    Pluse_InPut_EXTI_Configuration           0x08032891   Thumb Code   100  pluse_input.o(i.Pluse_InPut_EXTI_Configuration)
    Pluse_InPut_IO_Configuration             0x080328f5   Thumb Code   212  pluse_input.o(i.Pluse_InPut_IO_Configuration)
    Pluse_InPut_IRQHandler                   0x080329e1   Thumb Code   116  pluse_input.o(i.Pluse_InPut_IRQHandler)
    Pluse_InPut_Init                         0x08032a5d   Thumb Code   164  pluse_input.o(i.Pluse_InPut_Init)
    Pluse_InPut_NVIC_Configuration           0x08032b1d   Thumb Code    60  pluse_input.o(i.Pluse_InPut_NVIC_Configuration)
    Pluse_Putout_IO_Configuration            0x08032b59   Thumb Code   130  pluse_putout.o(i.Pluse_Putout_IO_Configuration)
    Pluse_Putout_Init                        0x08032bf1   Thumb Code     8  pluse_putout.o(i.Pluse_Putout_Init)
    Price_DataCheck                          0x08032bf9   Thumb Code    26  multiplex_port.o(i.Price_DataCheck)
    Print_Num                                0x08032c15   Thumb Code   358  printf.o(i.Print_Num)
    Query376Interrupt                        0x08032d81   Thumb Code    18  file_sys.o(i.Query376Interrupt)
    RCC_AHB1PeriphClockCmd                   0x08032d99   Thumb Code    26  stm32f4xx_rcc.o(i.RCC_AHB1PeriphClockCmd)
    RCC_AHB1PeriphResetCmd                   0x08032db9   Thumb Code    26  stm32f4xx_rcc.o(i.RCC_AHB1PeriphResetCmd)
    RCC_AHB2PeriphClockCmd                   0x08032dd9   Thumb Code    26  stm32f4xx_rcc.o(i.RCC_AHB2PeriphClockCmd)
    RCC_APB1PeriphClockCmd                   0x08032df9   Thumb Code    26  stm32f4xx_rcc.o(i.RCC_APB1PeriphClockCmd)
    RCC_APB1PeriphResetCmd                   0x08032e19   Thumb Code    26  stm32f4xx_rcc.o(i.RCC_APB1PeriphResetCmd)
    RCC_APB2PeriphClockCmd                   0x08032e39   Thumb Code    26  stm32f4xx_rcc.o(i.RCC_APB2PeriphClockCmd)
    RCC_APB2PeriphResetCmd                   0x08032e59   Thumb Code    26  stm32f4xx_rcc.o(i.RCC_APB2PeriphResetCmd)
    RCC_GetClocksFreq                        0x08032e79   Thumb Code   214  stm32f4xx_rcc.o(i.RCC_GetClocksFreq)
    RNG_Cmd                                  0x08032f61   Thumb Code    30  stm32f4xx_rng.o(i.RNG_Cmd)
    RNG_GetRandomNumber                      0x08032f85   Thumb Code     6  stm32f4xx_rng.o(i.RNG_GetRandomNumber)
    ReadDFStatus                             0x08032f91   Thumb Code    56  at45db.o(i.ReadDFStatus)
    ReadDriverID                             0x08032fcd   Thumb Code   130  at45db.o(i.ReadDriverID)
    SPI2_Init                                0x0803305d   Thumb Code   224  file_sys.o(i.SPI2_Init)
    SPI2_ReadWriteByte                       0x08033145   Thumb Code    50  file_sys.o(i.SPI2_ReadWriteByte)
    SPI_Cmd                                  0x0803317d   Thumb Code    24  stm32f4xx_spi.o(i.SPI_Cmd)
    SPI_I2S_DeInit                           0x08033195   Thumb Code    76  stm32f4xx_spi.o(i.SPI_I2S_DeInit)
    SPI_I2S_GetFlagStatus                    0x080331ed   Thumb Code    18  stm32f4xx_spi.o(i.SPI_I2S_GetFlagStatus)
    SPI_I2S_ReceiveData                      0x080331ff   Thumb Code     6  stm32f4xx_spi.o(i.SPI_I2S_ReceiveData)
    SPI_I2S_SendData                         0x08033205   Thumb Code     4  stm32f4xx_spi.o(i.SPI_I2S_SendData)
    SPI_Init                                 0x08033209   Thumb Code    60  stm32f4xx_spi.o(i.SPI_Init)
    SUMCRC                                   0x08033245   Thumb Code    28  pos_connect.o(i.SUMCRC)
    SYSCFG_EXTILineConfig                    0x08033261   Thumb Code    60  stm32f4xx_syscfg.o(i.SYSCFG_EXTILineConfig)
    SYSTimer_IRQHandler                      0x080332a1   Thumb Code   208  time_count.o(i.SYSTimer_IRQHandler)
    Spi376OutByte                            0x08033461   Thumb Code    12  file_sys.o(i.Spi376OutByte)
    StrToFloat                               0x0803346d   Thumb Code   128  md_connect.o(i.StrToFloat)
    StrToInt                                 0x080334f1   Thumb Code    76  md_connect.o(i.StrToInt)
    Sureface_Wait_TimeUpData                 0x0803353d   Thumb Code   402  surface.o(i.Sureface_Wait_TimeUpData)
    SurfaceJump                              0x080336d9   Thumb Code    12  surface.o(i.SurfaceJump)
    SurfaceTast                              0x080336e9   Thumb Code  9938  surface.o(i.SurfaceTast)
    Surface_Copy_16                          0x08035ddd   Thumb Code    68  surface.o(i.Surface_Copy_16)
    Surface_Init                             0x08035e21   Thumb Code    38  surface.o(i.Surface_Init)
    SysTick_CLKSourceConfig                  0x08035e4d   Thumb Code    40  misc.o(i.SysTick_CLKSourceConfig)
    SystemInit                               0x08035e75   Thumb Code    88  system_stm32f4xx.o(i.SystemInit)
    TIM2_IRQHandler                          0x08035edd   Thumb Code     8  stm32f4xx_it.o(i.TIM2_IRQHandler)
    TIM_ClearFlag                            0x08035ee5   Thumb Code     6  stm32f4xx_tim.o(i.TIM_ClearFlag)
    TIM_Cmd                                  0x08035eeb   Thumb Code    24  stm32f4xx_tim.o(i.TIM_Cmd)
    TIM_DeInit                               0x08035f05   Thumb Code   346  stm32f4xx_tim.o(i.TIM_DeInit)
    TIM_GetITStatus                          0x08036095   Thumb Code    34  stm32f4xx_tim.o(i.TIM_GetITStatus)
    TIM_ITConfig                             0x080360b7   Thumb Code    18  stm32f4xx_tim.o(i.TIM_ITConfig)
    TIM_TimeBaseInit                         0x080360c9   Thumb Code   104  stm32f4xx_tim.o(i.TIM_TimeBaseInit)
    TXH_Init                                 0x0803614d   Thumb Code   184  txh.o(i.TXH_Init)
    TXH_Task                                 0x0803620d   Thumb Code  2228  txh.o(i.TXH_Task)
    Timer_Init                               0x08036ad1   Thumb Code   788  time_count.o(i.Timer_Init)
    Timer_NVIC_Configuration                 0x08036e01   Thumb Code    34  time_count.o(i.Timer_NVIC_Configuration)
    UART4_IRQHandler                         0x08036e23   Thumb Code     8  stm32f4xx_it.o(i.UART4_IRQHandler)
    UART5_IRQHandler                         0x08036e2b   Thumb Code     8  stm32f4xx_it.o(i.UART5_IRQHandler)
    USART1_IRQHandler                        0x08036e33   Thumb Code     8  stm32f4xx_it.o(i.USART1_IRQHandler)
    USART2_IRQHandler                        0x08036e3b   Thumb Code     8  stm32f4xx_it.o(i.USART2_IRQHandler)
    USART3_IRQHandler                        0x08036e43   Thumb Code     8  stm32f4xx_it.o(i.USART3_IRQHandler)
    USART6_IRQHandler                        0x08036e4b   Thumb Code     8  stm32f4xx_it.o(i.USART6_IRQHandler)
    USART_ClearFlag                          0x08036e53   Thumb Code    18  stm32f4xx_usart.o(i.USART_ClearFlag)
    USART_Cmd                                0x08036e65   Thumb Code    24  stm32f4xx_usart.o(i.USART_Cmd)
    USART_DMACmd                             0x08036e7d   Thumb Code    18  stm32f4xx_usart.o(i.USART_DMACmd)
    USART_DeInit                             0x08036e91   Thumb Code   156  stm32f4xx_usart.o(i.USART_DeInit)
    USART_GetFlagStatus                      0x08036f45   Thumb Code    26  stm32f4xx_usart.o(i.USART_GetFlagStatus)
    USART_GetITStatus                        0x08036f5f   Thumb Code    84  stm32f4xx_usart.o(i.USART_GetITStatus)
    USART_ITConfig                           0x08036fb3   Thumb Code    74  stm32f4xx_usart.o(i.USART_ITConfig)
    USART_Init                               0x08036ffd   Thumb Code   204  stm32f4xx_usart.o(i.USART_Init)
    Wait376Interrupt                         0x080370d1   Thumb Code    30  file_sys.o(i.Wait376Interrupt)
    __0sprintf$8                             0x080370f5   Thumb Code    34  printf8.o(i.__0sprintf$8)
    __1sprintf$8                             0x080370f5   Thumb Code     0  printf8.o(i.__0sprintf$8)
    __2sprintf                               0x080370f5   Thumb Code     0  printf8.o(i.__0sprintf$8)
    __ARM_fpclassify                         0x0803711d   Thumb Code    48  fpclassify.o(i.__ARM_fpclassify)
    __hardfp_atof                            0x08037151   Thumb Code    44  atof.o(i.__hardfp_atof)
    __hardfp_log                             0x08037189   Thumb Code   872  log.o(i.__hardfp_log)
    __hardfp_log10                           0x08037551   Thumb Code   260  log10.o(i.__hardfp_log10)
    __hardfp_pow                             0x08037681   Thumb Code  3072  pow.o(i.__hardfp_pow)
    __kernel_poly                            0x080382d1   Thumb Code   248  poly.o(i.__kernel_poly)
    __mathlib_dbl_divzero                    0x080383c9   Thumb Code    28  dunder.o(i.__mathlib_dbl_divzero)
    __mathlib_dbl_infnan                     0x080383f9   Thumb Code    20  dunder.o(i.__mathlib_dbl_infnan)
    __mathlib_dbl_infnan2                    0x0803840d   Thumb Code    20  dunder.o(i.__mathlib_dbl_infnan2)
    __mathlib_dbl_invalid                    0x08038421   Thumb Code    24  dunder.o(i.__mathlib_dbl_invalid)
    __mathlib_dbl_overflow                   0x08038441   Thumb Code    24  dunder.o(i.__mathlib_dbl_overflow)
    __mathlib_dbl_underflow                  0x08038461   Thumb Code    24  dunder.o(i.__mathlib_dbl_underflow)
    __read_errno                             0x08038481   Thumb Code     6  errno.o(i.__read_errno)
    __scatterload_copy                       0x0803848d   Thumb Code    14  handlers.o(i.__scatterload_copy)
    __scatterload_null                       0x0803849b   Thumb Code     2  handlers.o(i.__scatterload_null)
    __scatterload_zeroinit                   0x0803849d   Thumb Code    14  handlers.o(i.__scatterload_zeroinit)
    __set_errno                              0x080384b9   Thumb Code     6  errno.o(i.__set_errno)
    _is_digit                                0x080384c5   Thumb Code    14  scanf_fp.o(i._is_digit)
    delay_init                               0x08038935   Thumb Code    12  delay.o(i.delay_init)
    delay_ms                                 0x08038941   Thumb Code    68  delay.o(i.delay_ms)
    delay_us                                 0x08038985   Thumb Code    66  delay.o(i.delay_us)
    do_crc                                   0x080389c9   Thumb Code    36  md_connect.o(i.do_crc)
    fabs                                     0x080389f1   Thumb Code    24  fabs.o(i.fabs)
    iic_ack                                  0x08038a09   Thumb Code    60  ds1307.o(i.iic_ack)
    iic_noack                                0x08038a49   Thumb Code    60  ds1307.o(i.iic_noack)
    iic_readbyte                             0x08038a89   Thumb Code    92  ds1307.o(i.iic_readbyte)
    iic_sendbyte                             0x08038ae9   Thumb Code    98  ds1307.o(i.iic_sendbyte)
    iic_start                                0x08038b51   Thumb Code    46  ds1307.o(i.iic_start)
    iic_stop                                 0x08038b85   Thumb Code    46  ds1307.o(i.iic_stop)
    iic_wait4ack                             0x08038bb9   Thumb Code    88  ds1307.o(i.iic_wait4ack)
    log                                      0x08038c15   Thumb Code    16  log.o(i.log)
    mInitCH376Host                           0x08038c25   Thumb Code    98  file_sys.o(i.mInitCH376Host)
    main                                     0x08038c91   Thumb Code    90  main.o(i.main)
    mystrstr                                 0x08038cfd   Thumb Code    68  multiplex_port.o(i.mystrstr)
    sqrt                                     0x08038d41   Thumb Code   110  sqrt.o(i.sqrt)
    xReadCH376Data                           0x08038daf   Thumb Code    20  file_sys.o(i.xReadCH376Data)
    xWriteCH376Cmd                           0x08038dc5   Thumb Code    54  file_sys.o(i.xWriteCH376Cmd)
    xWriteCH376Data                          0x08038e05   Thumb Code    18  file_sys.o(i.xWriteCH376Data)
    BoxVersion                               0x08038e16   Data          11  txh.o(.constdata)
    initFRam_Flag                            0x08038e24   Data           1  fram.o(.constdata)
    InitPrintInfo                            0x08038e25   Data         640  fram.o(.constdata)
    InitMD_Port_Data                         0x080390a8   Data         304  fram.o(.constdata)
    InitPOSData                              0x080391d8   Data         194  fram.o(.constdata)
    InitMD_Port_Num_Top                      0x0803929a   Data           1  fram.o(.constdata)
    InitROM_UpData                           0x0803929c   Data           4  fram.o(.constdata)
    InitPREXDATA_WaitUpNummber               0x080392a0   Data           4  fram.o(.constdata)
    InitPREXDATA_TTC                         0x080392a4   Data           4  fram.o(.constdata)
    initPrintLastRecord                      0x080392a8   Data          96  fram.o(.constdata)
    InitPOSNetSetState                       0x08039308   Data           2  fram.o(.constdata)
    InitMD_Multiplex_Port_Data               0x0803930c   Data         272  fram.o(.constdata)
    InitWhiteList                            0x0803941c   Data        1202  fram.o(.constdata)
    InitPREXDATA_Upload                      0x080398d0   Data           8  fram.o(.constdata)
    FDITab                                   0x080398d8   Data         312  fram.o(.constdata)
    MD_WifiWSSSID                            0x08039a10   Data          26  md_connect.o(.constdata)
    MD_WifiSOCKET                            0x08039a2a   Data          34  md_connect.o(.constdata)
    MD_WifiRSSI                              0x08039a4c   Data          12  md_connect.o(.constdata)
    MD_WifiRST                               0x08039a58   Data           9  md_connect.o(.constdata)
    MD_ATRec                                 0x08039a61   Data          11  md_connect.o(.constdata)
    MD_WMODE                                 0x08039a6c   Data          14  md_connect.o(.constdata)
    TsatURL                                  0x08039a7c   Data          40  pos_connect.o(.constdata)
    CMD_LinkMode                             0x08039aa4   Data          15  pos_connect.o(.constdata)
    CMD_UARTFL                               0x08039ab3   Data          17  pos_connect.o(.constdata)
    CMD_HEARTEN                              0x08039ac4   Data          17  pos_connect.o(.constdata)
    CMD_Save                                 0x08039ad5   Data           7  pos_connect.o(.constdata)
    CMD_ATRec                                0x08039adc   Data          11  pos_connect.o(.constdata)
    CMD_Model_Set                            0x08039ae7   Data           8  pos_connect.o(.constdata)
    CMD_Model_Set_1                          0x08039aef   Data           4  pos_connect.o(.constdata)
    CMD_Model_Set_2                          0x08039af3   Data           2  pos_connect.o(.constdata)
    CMD_Model_NET                            0x08039af5   Data          10  pos_connect.o(.constdata)
    CMD_ICCID                                0x08039aff   Data          12  pos_connect.o(.constdata)
    CMD_IMEI                                 0x08039b0b   Data          11  pos_connect.o(.constdata)
    CMD_CSQ                                  0x08039b16   Data          10  pos_connect.o(.constdata)
    NextStr                                  0x08039b20   Data           4  pos_connect.o(.constdata)
    WlanTsatURL                              0x08039b24   Data          42  pos_connect.o(.constdata)
    CMD_Reset                                0x08039b4e   Data           7  pos_connect.o(.constdata)
    CMD_DHCP                                 0x08039b55   Data          15  pos_connect.o(.constdata)
    CMD_GetIP                                0x08039b64   Data          10  pos_connect.o(.constdata)
    CMD_GetLinkState                         0x08039b6e   Data          14  pos_connect.o(.constdata)
    CMD_WifiWSSSID                           0x08039b7c   Data          29  pos_connect.o(.constdata)
    CMD_WifiWSSSID_WIFIStation               0x08039b99   Data          32  pos_connect.o(.constdata)
    CMD_WifiSOCKET                           0x08039bb9   Data          41  pos_connect.o(.constdata)
    CMD_WifiSOCKET_WIFIStation               0x08039be2   Data          36  pos_connect.o(.constdata)
    CMD_WifiRSSI                             0x08039c06   Data          12  pos_connect.o(.constdata)
    CMD_WifiRST                              0x08039c12   Data           9  pos_connect.o(.constdata)
    CMD_L510_AT                              0x08039c1b   Data           4  pos_connect.o(.constdata)
    CMD_L510_ATRec                           0x08039c1f   Data           7  pos_connect.o(.constdata)
    CMD_L510_IMEI                            0x08039c26   Data          10  pos_connect.o(.constdata)
    CMD_L510_ICPIN                           0x08039c30   Data          11  pos_connect.o(.constdata)
    CMD_L510_ICCID                           0x08039c3b   Data          11  pos_connect.o(.constdata)
    CMD_L510_RSSI                            0x08039c46   Data           9  pos_connect.o(.constdata)
    CMD_L510_Model_NET                       0x08039c4f   Data          15  pos_connect.o(.constdata)
    CMD_L510_APN                             0x08039c5e   Data          30  pos_connect.o(.constdata)
    CMD_L510_NETOPEN                         0x08039c7c   Data          13  pos_connect.o(.constdata)
    CMD_L510_SOCKET                          0x08039c89   Data          48  pos_connect.o(.constdata)
    CMD_L510_GetLinkState                    0x08039cb9   Data          17  pos_connect.o(.constdata)
    CMD_L510_RESET                           0x08039cca   Data          11  pos_connect.o(.constdata)
    CMD_L510_SetGPSMode                      0x08039cd5   Data          20  pos_connect.o(.constdata)
    CMD_L510_GetGPS                          0x08039ce9   Data          13  pos_connect.o(.constdata)
    Operators                                0x08039cf6   Data       19190  pos_connect.o(.constdata)
    auchCRCHi                                0x0803e7ec   Data         256  pos_connect.o(.constdata)
    auchCRCLo                                0x0803e8ec   Data         256  pos_connect.o(.constdata)
    initATDB45_Flag                          0x0803ea20   Data           1  at45db.o(.constdata)
    initPREXDATA                             0x0803ea21   Data          96  at45db.o(.constdata)
    AT45DBTab                                0x0803ea84   Data         480  at45db.o(.constdata)
    asc2_0806                                0x0803ec64   Data         552  oled.o(.constdata)
    asc2_1206                                0x0803ee8c   Data        1140  oled.o(.constdata)
    asc2_1608                                0x0803f300   Data        1520  oled.o(.constdata)
    asc2_2412                                0x0803f8f0   Data        3420  oled.o(.constdata)
    Hzk1                                     0x0804064c   Data         352  oled.o(.constdata)
    Hzk2                                     0x080407ac   Data          72  oled.o(.constdata)
    Hzk3                                     0x080407f4   Data         128  oled.o(.constdata)
    Hzk4                                     0x08040874   Data         512  oled.o(.constdata)
    BMP_Bluesky_Con_48                       0x08040a74   Data         288  surface.o(.constdata)
    BMP_Bluesky_Con_24                       0x08040b94   Data          72  surface.o(.constdata)
    BMP_Bluesky_Empty_8                      0x08040bdc   Data           8  surface.o(.constdata)
    BMP_Bluetooth_9                          0x08040be4   Data          18  surface.o(.constdata)
    BMP_GPS_9                                0x08040bf6   Data          18  surface.o(.constdata)
    BMP_GPS_None_9                           0x08040c08   Data          18  surface.o(.constdata)
    BMP_WIFI0_14x8                           0x08040c1a   Data          14  surface.o(.constdata)
    BMP_WIFI1_14x8                           0x08040c28   Data          14  surface.o(.constdata)
    BMP_WIFI2_14x8                           0x08040c36   Data          14  surface.o(.constdata)
    BMP_WIFI3_14x8                           0x08040c44   Data          14  surface.o(.constdata)
    BMP_WIFI4_14x8                           0x08040c52   Data          14  surface.o(.constdata)
    QueryMenu                                0x08040c60   Data         128  surface.o(.constdata)
    QueryNetworkInfo                         0x08040ce0   Data          64  surface.o(.constdata)
    PrintInfo                                0x08040d20   Data          64  surface.o(.constdata)
    QueryMDPortInfo                          0x08040d60   Data          64  surface.o(.constdata)
    QueryTestInfo                            0x08040da0   Data          64  surface.o(.constdata)
    QueryMDPortInfo_POSType                  0x08040de0   Data         208  surface.o(.constdata)
    YWY_Type_Info                            0x08040eb0   Data          48  surface.o(.constdata)
    QueryLORARSSI                            0x08040ee0   Data          64  surface.o(.constdata)
    QueryVeresion                            0x08040f20   Data          64  surface.o(.constdata)
    SetMenu                                  0x08040f60   Data         144  surface.o(.constdata)
    SetMDConnect                             0x08040ff0   Data          64  surface.o(.constdata)
    SetLORASlave                             0x08041030   Data          64  surface.o(.constdata)
    SetPortLogOutput                         0x08041070   Data          64  surface.o(.constdata)
    SetConnectMode                           0x080410b0   Data          64  surface.o(.constdata)
    SetNetworkSet                            0x080410f0   Data          64  surface.o(.constdata)
    ConnectMode_Info                         0x08041130   Data          80  surface.o(.constdata)
    Network_Type_Info                        0x08041180   Data          80  surface.o(.constdata)
    SetDataInit                              0x080411d0   Data          64  surface.o(.constdata)
    __mathlib_zero                           0x080412d0   Data           8  qnan.o(.constdata)
    __ctype_categories                       0x080412d8   Data          64  ctype_c.o(.constdata)
    Region$$Table$$Base                      0x08041318   Number         0  anon$$obj.o(Region$$Table)
    Region$$Table$$Limit                     0x08041338   Number         0  anon$$obj.o(Region$$Table)
    iiii                                     0x20000010   Data           2  fram.o(.data)
    MD_ConnectRX1Task_Flag                   0x20000012   Data           1  md_connect.o(.data)
    MD_ConnectRX2Task_Flag                   0x20000013   Data           1  md_connect.o(.data)
    MD_ConnectRX3Task_Flag                   0x20000014   Data           1  md_connect.o(.data)
    MD_ConnectRX4Task_Flag                   0x20000015   Data           1  md_connect.o(.data)
    MD_Connect_TX_Flag                       0x20000016   Data           1  md_connect.o(.data)
    crc16_ccitt_table                        0x20000018   Data         512  md_connect.o(.data)
    DTTDYS                                   0x20000218   Data           1  md_connect.o(.data)
    zhtningzhuangtai                         0x20000219   Data           1  md_connect.o(.data)
    KBAddr_Init                              0x2000021a   Data           4  md_connect.o(.data)
    CMD_APN                                  0x20000220   Data          50  pos_connect.o(.data)
    POS_Connect_TX_Buff                      0x20000252   Data        2000  pos_connect.o(.data)
    POS_Connect_TX_Flag                      0x20000a22   Data           1  pos_connect.o(.data)
    POS_RX_RNGData                           0x20000a24   Data           4  pos_connect.o(.data)
    FrameNow                                 0x20000a28   Data           2  pos_connect.o(.data)
    FrameTimeout                             0x20000a2a   Data           1  pos_connect.o(.data)
    FlashType                                0x20000a2c   Data           1  at45db.o(.data)
    ii                                       0x20000a2e   Data           2  at45db.o(.data)
    resultF                                  0x20000a30   Data           1  at45db.o(.data)
    CRCTemp                                  0x20000a31   Data           1  at45db.o(.data)
    DiskFileOpen_Flag                        0x20000a38   Data           1  log.o(.data)
    File_Len                                 0x20000a40   Data           8  log.o(.data)
    SysconfigFileName                        0x20000a48   Data          20  log.o(.data)
    EndLen                                   0x20000a5c   Data           2  log.o(.data)
    StartLen                                 0x20000a5e   Data           2  log.o(.data)
    LogName                                  0x20000a60   Data         125  log.o(.data)
    KeyNumBefore                             0x20000add   Data           1  surface.o(.data)
    KeyNumconfirm_Flag                       0x20000ade   Data           1  surface.o(.data)
    KeyNum0                                  0x20000adf   Data           1  surface.o(.data)
    KeyNum1                                  0x20000ae0   Data           1  surface.o(.data)
    KeyNum                                   0x20000ae1   Data           1  surface.o(.data)
    Multiplex_Port_RX_Flag                   0x20000ae2   Data           1  multiplex_port.o(.data)
    Multiplex_Port_TX_Flag                   0x20000ae3   Data           1  multiplex_port.o(.data)
    Multiplex_Port_RX_Buff                   0x20000ae4   Data        1000  multiplex_port.o(.data)
    Multiplex_Port_TX_Buff                   0x20000ecc   Data        1000  multiplex_port.o(.data)
    Multiplex_Port_DMA_RX_Len                0x200012b4   Data           1  multiplex_port.o(.data)
    TXHData                                  0x200012bc   Data       28248  txh.o(.bss)
    STM32CPU                                 0x20008114   Data          12  txh.o(.bss)
    s_uniGlobal                              0x20008120   Data        1208  fram.o(.bss)
    MD_Connect_TX_Buff                       0x200085d8   Data        2400  md_connect.o(.bss)
    MD_Connect_RX_Buff                       0x20008f38   Data        4000  md_connect.o(.bss)
    LORA_Set                                 0x20009ed8   Data          20  md_connect.o(.bss)
    HY_SendBuff                              0x20009eec   Data          50  md_connect.o(.bss)
    MD_RX_RNGData                            0x20009f20   Data          16  md_connect.o(.bss)
    POS_Connect_RX_Buff                      0x20009f30   Data        2000  pos_connect.o(.bss)
    POS2MD_Buff                              0x2000a700   Data        2000  pos_connect.o(.bss)
    F_uniGlobal                              0x2000aed0   Data         531  at45db.o(.bss)
    OLED_GRAM                                0x2000b0e3   Data        1152  oled.o(.bss)
    __initial_sp                             0x2000f568   Data           0  startup_stm32f4xx.o(STACK)



==============================================================================

Memory Map of the image

  Image Entry point : 0x08008189

  Load Region LR_IROM1 (Base: 0x08008000, Size: 0x0003a5f4, Max: 0x00080000, ABSOLUTE, COMPRESSED[0x000395b8])

    Execution Region ER_IROM1 (Exec base: 0x08008000, Load base: 0x08008000, Size: 0x00039338, Max: 0x00080000, ABSOLUTE)

    Exec Addr    Load Addr    Size         Type   Attr      Idx    E Section Name        Object

    0x08008000   0x08008000   0x00000188   Data   RO          398    RESET               startup_stm32f4xx.o
    0x08008188   0x08008188   0x00000000   Code   RO         4134  * .ARM.Collect$$$$00000000  mc_w.l(entry.o)
    0x08008188   0x08008188   0x00000004   Code   RO         4501    .ARM.Collect$$$$00000001  mc_w.l(entry2.o)
    0x0800818c   0x0800818c   0x00000004   Code   RO         4504    .ARM.Collect$$$$00000004  mc_w.l(entry5.o)
    0x08008190   0x08008190   0x00000000   Code   RO         4506    .ARM.Collect$$$$00000008  mc_w.l(entry7b.o)
    0x08008190   0x08008190   0x00000000   Code   RO         4508    .ARM.Collect$$$$0000000A  mc_w.l(entry8b.o)
    0x08008190   0x08008190   0x00000008   Code   RO         4509    .ARM.Collect$$$$0000000B  mc_w.l(entry9a.o)
    0x08008198   0x08008198   0x00000004   Code   RO         4516    .ARM.Collect$$$$0000000E  mc_w.l(entry12b.o)
    0x0800819c   0x0800819c   0x00000000   Code   RO         4511    .ARM.Collect$$$$0000000F  mc_w.l(entry10a.o)
    0x0800819c   0x0800819c   0x00000000   Code   RO         4513    .ARM.Collect$$$$00000011  mc_w.l(entry11a.o)
    0x0800819c   0x0800819c   0x00000004   Code   RO         4502    .ARM.Collect$$$$00002712  mc_w.l(entry2.o)
    0x080081a0   0x080081a0   0x00000024   Code   RO          399    .text               startup_stm32f4xx.o
    0x080081c4   0x080081c4   0x00000062   Code   RO         4137    .text               mc_w.l(ldiv.o)
    0x08008226   0x08008226   0x00000024   Code   RO         4139    .text               mc_w.l(llsshr.o)
    0x0800824a   0x0800824a   0x00000024   Code   RO         4141    .text               mc_w.l(memcpya.o)
    0x0800826e   0x0800826e   0x00000018   Code   RO         4143    .text               mc_w.l(strcat.o)
    0x08008286   0x08008286   0x0000000e   Code   RO         4145    .text               mc_w.l(strlen.o)
    0x08008294   0x08008294   0x0000001e   Code   RO         4147    .text               mc_w.l(strncmp.o)
    0x080082b2   0x080082b2   0x0000014e   Code   RO         4412    .text               mf_w.l(dadd.o)
    0x08008400   0x08008400   0x000000e4   Code   RO         4414    .text               mf_w.l(dmul.o)
    0x080084e4   0x080084e4   0x000000de   Code   RO         4416    .text               mf_w.l(ddiv.o)
    0x080085c2   0x080085c2   0x0000002c   Code   RO         4418    .text               mf_w.l(ffltl.o)
    0x080085ee   0x080085ee   0x00000022   Code   RO         4420    .text               mf_w.l(dflti.o)
    0x08008610   0x08008610   0x0000001a   Code   RO         4422    .text               mf_w.l(dfltui.o)
    0x0800862a   0x0800862a   0x00000028   Code   RO         4424    .text               mf_w.l(dfltl.o)
    0x08008652   0x08008652   0x00000042   Code   RO         4426    .text               mf_w.l(ffixl.o)
    0x08008694   0x08008694   0x0000003e   Code   RO         4428    .text               mf_w.l(dfixi.o)
    0x080086d2   0x080086d2   0x0000004a   Code   RO         4430    .text               mf_w.l(dfixl.o)
    0x0800871c   0x0800871c   0x00000026   Code   RO         4432    .text               mf_w.l(f2d.o)
    0x08008742   0x08008742   0x00000038   Code   RO         4434    .text               mf_w.l(d2f.o)
    0x0800877a   0x0800877a   0x00000062   Code   RO         4522    .text               mc_w.l(uldiv.o)
    0x080087dc   0x080087dc   0x0000001e   Code   RO         4524    .text               mc_w.l(llshl.o)
    0x080087fa   0x080087fa   0x00000020   Code   RO         4526    .text               mc_w.l(llushr.o)
    0x0800881a   0x0800881a   0x00000002   PAD
    0x0800881c   0x0800881c   0x0000009c   Code   RO         4535    .text               mc_w.l(strtod.o)
    0x080088b8   0x080088b8   0x00000000   Code   RO         4537    .text               mc_w.l(iusefp.o)
    0x080088b8   0x080088b8   0x0000006e   Code   RO         4538    .text               mf_w.l(fepilogue.o)
    0x08008926   0x08008926   0x000000ba   Code   RO         4540    .text               mf_w.l(depilogue.o)
    0x080089e0   0x080089e0   0x0000002e   Code   RO         4544    .text               mf_w.l(dscalb.o)
    0x08008a0e   0x08008a0e   0x00000002   PAD
    0x08008a10   0x08008a10   0x00000030   Code   RO         4548    .text               mf_w.l(cdrcmple.o)
    0x08008a40   0x08008a40   0x00000024   Code   RO         4550    .text               mc_w.l(init.o)
    0x08008a64   0x08008a64   0x0000000a   Code   RO         4553    .text               mc_w.l(isspace_c.o)
    0x08008a6e   0x08008a6e   0x00000002   PAD
    0x08008a70   0x08008a70   0x00000360   Code   RO         4555    .text               mc_w.l(scanf_fp.o)
    0x08008dd0   0x08008dd0   0x00000040   Code   RO         4559    .text               mc_w.l(_sgetc.o)
    0x08008e10   0x08008e10   0x000000a2   Code   RO         4562    .text               mf_w.l(dsqrt.o)
    0x08008eb2   0x08008eb2   0x00000002   PAD
    0x08008eb4   0x08008eb4   0x00000030   Code   RO         4564    .text               mf_w.l(cdcmple.o)
    0x08008ee4   0x08008ee4   0x00000028   Code   RO         4566    .text               mc_w.l(ctype_c.o)
    0x08008f0c   0x08008f0c   0x00000018   Code   RO         4569    .text               mf_w.l(dfltul.o)
    0x08008f24   0x08008f24   0x00000056   Code   RO         4579    .text               mc_w.l(__dczerorl2.o)
    0x08008f7a   0x08008f7a   0x0000001c   Code   RO         3171    i.AT45DBDataCheck   at45db.o
    0x08008f96   0x08008f96   0x00000002   PAD
    0x08008f98   0x08008f98   0x00000138   Code   RO         3172    i.AT45DBItemRead    at45db.o
    0x080090d0   0x080090d0   0x000000e8   Code   RO         3173    i.AT45DBItemWrite   at45db.o
    0x080091b8   0x080091b8   0x00000050   Code   RO         3175    i.AT45DB_Init       at45db.o
    0x08009208   0x08009208   0x000000c0   Code   RO         3176    i.AT45DB_ReadPage   at45db.o
    0x080092c8   0x080092c8   0x00000038   Code   RO         3177    i.AT45DB_SendByte   at45db.o
    0x08009300   0x08009300   0x0000008c   Code   RO         3178    i.AT45DB_SetPageByte  at45db.o
    0x0800938c   0x0800938c   0x000000a4   Code   RO         3179    i.AT45DB_WriteBuff  at45db.o
    0x08009430   0x08009430   0x000000a4   Code   RO         3180    i.AT45DB_WritePage  at45db.o
    0x080094d4   0x080094d4   0x0000001a   Code   RO         2746    i.BCC_CheckSum      md_connect.o
    0x080094ee   0x080094ee   0x00000014   Code   RO         2747    i.Bluesky_Decrypt   md_connect.o
    0x08009502   0x08009502   0x00000060   Code   RO         2748    i.Bluesky_Encrypt   md_connect.o
    0x08009562   0x08009562   0x00000002   PAD
    0x08009564   0x08009564   0x0000003c   Code   RO         3362    i.CH376ByteLocate   file_sys.o
    0x080095a0   0x080095a0   0x00000064   Code   RO         3363    i.CH376ByteRead     file_sys.o
    0x08009604   0x08009604   0x00000068   Code   RO         3364    i.CH376ByteWrite    file_sys.o
    0x0800966c   0x0800966c   0x00000014   Code   RO         3369    i.CH376DiskConnect  file_sys.o
    0x08009680   0x08009680   0x0000000e   Code   RO         3374    i.CH376FileClose    file_sys.o
    0x0800968e   0x0800968e   0x00000014   Code   RO         3375    i.CH376FileCreate   file_sys.o
    0x080096a2   0x080096a2   0x00000026   Code   RO         3378    i.CH376FileOpen     file_sys.o
    0x080096c8   0x080096c8   0x0000000a   Code   RO         3382    i.CH376GetFileSize  file_sys.o
    0x080096d2   0x080096d2   0x00000002   PAD
    0x080096d4   0x080096d4   0x00000020   Code   RO         3383    i.CH376GetIntStatus  file_sys.o
    0x080096f4   0x080096f4   0x0000003c   Code   RO         3384    i.CH376Read32bitDat  file_sys.o
    0x08009730   0x08009730   0x00000038   Code   RO         3385    i.CH376ReadBlock    file_sys.o
    0x08009768   0x08009768   0x00000016   Code   RO         3386    i.CH376ReadVar32    file_sys.o
    0x0800977e   0x0800977e   0x00000002   PAD
    0x08009780   0x08009780   0x00000028   Code   RO         3387    i.CH376ReadVar8     file_sys.o
    0x080097a8   0x080097a8   0x00000028   Code   RO         3389    i.CH376SendCmdDatWaitInt  file_sys.o
    0x080097d0   0x080097d0   0x00000020   Code   RO         3390    i.CH376SendCmdWaitInt  file_sys.o
    0x080097f0   0x080097f0   0x000000a8   Code   RO         3392    i.CH376SetFileName  file_sys.o
    0x08009898   0x08009898   0x00000038   Code   RO         3395    i.CH376WriteReqBlock  file_sys.o
    0x080098d0   0x080098d0   0x00000040   Code   RO         3396    i.CH376WriteVar32   file_sys.o
    0x08009910   0x08009910   0x00000038   Code   RO         2944    i.CRC_Check         pos_connect.o
    0x08009948   0x08009948   0x00000046   Code   RO         2749    i.CheckSum          md_connect.o
    0x0800998e   0x0800998e   0x0000001c   Code   RO         2750    i.CheckSum8         md_connect.o
    0x080099aa   0x080099aa   0x00000008   Code   RO            2    i.DMA1_Stream3_IRQHandler  stm32f4xx_it.o
    0x080099b2   0x080099b2   0x00000008   Code   RO            3    i.DMA1_Stream4_IRQHandler  stm32f4xx_it.o
    0x080099ba   0x080099ba   0x00000008   Code   RO            4    i.DMA1_Stream6_IRQHandler  stm32f4xx_it.o
    0x080099c2   0x080099c2   0x00000008   Code   RO            5    i.DMA1_Stream7_IRQHandler  stm32f4xx_it.o
    0x080099ca   0x080099ca   0x00000008   Code   RO            6    i.DMA2_Stream6_IRQHandler  stm32f4xx_it.o
    0x080099d2   0x080099d2   0x00000008   Code   RO            7    i.DMA2_Stream7_IRQHandler  stm32f4xx_it.o
    0x080099da   0x080099da   0x00000002   PAD
    0x080099dc   0x080099dc   0x00000034   Code   RO          728    i.DMA_ClearFlag     stm32f4xx_dma.o
    0x08009a10   0x08009a10   0x00000016   Code   RO          730    i.DMA_Cmd           stm32f4xx_dma.o
    0x08009a26   0x08009a26   0x00000002   PAD
    0x08009a28   0x08009a28   0x00000158   Code   RO          731    i.DMA_DeInit        stm32f4xx_dma.o
    0x08009b80   0x08009b80   0x0000003a   Code   RO          741    i.DMA_ITConfig      stm32f4xx_dma.o
    0x08009bba   0x08009bba   0x00000002   PAD
    0x08009bbc   0x08009bbc   0x00000058   Code   RO          742    i.DMA_Init          stm32f4xx_dma.o
    0x08009c14   0x08009c14   0x00000098   Code   RO         3101    i.DS1307_Init       ds1307.o
    0x08009cac   0x08009cac   0x00000088   Code   RO         3102    i.DS1307_Read       ds1307.o
    0x08009d34   0x08009d34   0x0000007c   Code   RO         3103    i.DS1307_Write      ds1307.o
    0x08009db0   0x08009db0   0x00000038   Code   RO         2945    i.DartCRC16         pos_connect.o
    0x08009de8   0x08009de8   0x00000030   Code   RO         2947    i.Decode_Data       pos_connect.o
    0x08009e18   0x08009e18   0x00000008   Code   RO            8    i.EXTI0_IRQHandler  stm32f4xx_it.o
    0x08009e20   0x08009e20   0x00000008   Code   RO            9    i.EXTI15_10_IRQHandler  stm32f4xx_it.o
    0x08009e28   0x08009e28   0x00000008   Code   RO           10    i.EXTI1_IRQHandler  stm32f4xx_it.o
    0x08009e30   0x08009e30   0x0000000c   Code   RO          853    i.EXTI_ClearITPendingBit  stm32f4xx_exti.o
    0x08009e3c   0x08009e3c   0x00000028   Code   RO          857    i.EXTI_GetITStatus  stm32f4xx_exti.o
    0x08009e64   0x08009e64   0x00000094   Code   RO          858    i.EXTI_Init         stm32f4xx_exti.o
    0x08009ef8   0x08009ef8   0x00000030   Code   RO         2949    i.Encrypt_Data      pos_connect.o
    0x08009f28   0x08009f28   0x00000184   Code   RO         2614    i.FMItemRead        fram.o
    0x0800a0ac   0x0800a0ac   0x0000014c   Code   RO         2615    i.FMItemWrite       fram.o
    0x0800a1f8   0x0800a1f8   0x00000158   Code   RO         2616    i.FM_Data_Init      fram.o
    0x0800a350   0x0800a350   0x00000080   Code   RO         2617    i.FM_IO_Configuration  fram.o
    0x0800a3d0   0x0800a3d0   0x000000ec   Code   RO         2618    i.FM_Init           fram.o
    0x0800a4bc   0x0800a4bc   0x0000006c   Code   RO         2619    i.FM_ReadData       fram.o
    0x0800a528   0x0800a528   0x00000038   Code   RO         2620    i.FM_SPI1_SendByte  fram.o
    0x0800a560   0x0800a560   0x00000060   Code   RO         2621    i.FM_SPI_Configuration  fram.o
    0x0800a5c0   0x0800a5c0   0x00000088   Code   RO         2622    i.FM_WriteData      fram.o
    0x0800a648   0x0800a648   0x0000001c   Code   RO         2623    i.FRamDataCheck     fram.o
    0x0800a664   0x0800a664   0x000000d4   Code   RO         3810    i.FindKey           surface.o
    0x0800a738   0x0800a738   0x00000250   Code   RO         3648    i.FindSysconfigFile  log.o
    0x0800a988   0x0800a988   0x00000100   Code   RO         1100    i.GPIO_DeInit       stm32f4xx_gpio.o
    0x0800aa88   0x0800aa88   0x00000090   Code   RO         1101    i.GPIO_Init         stm32f4xx_gpio.o
    0x0800ab18   0x0800ab18   0x00000046   Code   RO         1102    i.GPIO_PinAFConfig  stm32f4xx_gpio.o
    0x0800ab5e   0x0800ab5e   0x00000012   Code   RO         1105    i.GPIO_ReadInputDataBit  stm32f4xx_gpio.o
    0x0800ab70   0x0800ab70   0x00000004   Code   RO         1108    i.GPIO_ResetBits    stm32f4xx_gpio.o
    0x0800ab74   0x0800ab74   0x00000004   Code   RO         1109    i.GPIO_SetBits      stm32f4xx_gpio.o
    0x0800ab78   0x0800ab78   0x00000010   Code   RO         3811    i.GetKeyNum         surface.o
    0x0800ab88   0x0800ab88   0x00000044   Code   RO           11    i.HardFault_Handler  stm32f4xx_it.o
    0x0800abcc   0x0800abcc   0x00000010   Code   RO         2536    i.IWDG_ReloadCounter  stm32f4xx_iwdg.o
    0x0800abdc   0x0800abdc   0x00000020   Code   RO         2751    i.InteiHEXCheck     md_connect.o
    0x0800abfc   0x0800abfc   0x00000010   Code   RO         3649    i.Log_Init          log.o
    0x0800ac0c   0x0800ac0c   0x00000268   Code   RO         3650    i.Log_Task          log.o
    0x0800ae74   0x0800ae74   0x00014358   Code   RO         2752    i.MD_ConnectRXTask  md_connect.o
    0x0801f1cc   0x0801f1cc   0x00008cc4   Code   RO         2753    i.MD_ConnectTXTask  md_connect.o
    0x08027e90   0x08027e90   0x000000a0   Code   RO         2754    i.MD_Connect_BCDTou64  md_connect.o
    0x08027f30   0x08027f30   0x00000054   Code   RO         2755    i.MD_Connect_DMARX1_IRQHandler  md_connect.o
    0x08027f84   0x08027f84   0x00000044   Code   RO         2756    i.MD_Connect_DMARX2_IRQHandler  md_connect.o
    0x08027fc8   0x08027fc8   0x00000044   Code   RO         2757    i.MD_Connect_DMARX3_IRQHandler  md_connect.o
    0x0802800c   0x0802800c   0x00000048   Code   RO         2758    i.MD_Connect_DMARX4_IRQHandler  md_connect.o
    0x08028054   0x08028054   0x00000060   Code   RO         2759    i.MD_Connect_DMATX1_IRQHandler  md_connect.o
    0x080280b4   0x080280b4   0x00000060   Code   RO         2760    i.MD_Connect_DMATX2_IRQHandler  md_connect.o
    0x08028114   0x08028114   0x00000064   Code   RO         2761    i.MD_Connect_DMATX3_IRQHandler  md_connect.o
    0x08028178   0x08028178   0x00000064   Code   RO         2762    i.MD_Connect_DMATX4_IRQHandler  md_connect.o
    0x080281dc   0x080281dc   0x00000340   Code   RO         2763    i.MD_Connect_DMA_Configuration  md_connect.o
    0x0802851c   0x0802851c   0x00000148   Code   RO         2764    i.MD_Connect_IO_Configuration  md_connect.o
    0x08028664   0x08028664   0x00000060   Code   RO         2765    i.MD_Connect_Init   md_connect.o
    0x080286c4   0x080286c4   0x000000ec   Code   RO         2766    i.MD_Connect_NVIC_Configuration  md_connect.o
    0x080287b0   0x080287b0   0x00000022   Code   RO         2767    i.MD_Connect_TXDataCheck  md_connect.o
    0x080287d2   0x080287d2   0x00000002   PAD
    0x080287d4   0x080287d4   0x00000224   Code   RO         2768    i.MD_Connect_USART_Configuration  md_connect.o
    0x080289f8   0x080289f8   0x00000074   Code   RO         2769    i.MD_Connect_u64ToBCD  md_connect.o
    0x08028a6c   0x08028a6c   0x00000a80   Code   RO         2770    i.MD_Port_Init      md_connect.o
    0x080294ec   0x080294ec   0x00000374   Code   RO         2771    i.MD_Port_LORASet   md_connect.o
    0x08029860   0x08029860   0x000007d4   Code   RO         3946    i.Multiplex_PortRXTask  multiplex_port.o
    0x0802a034   0x0802a034   0x000007fc   Code   RO         3947    i.Multiplex_PortTXTask  multiplex_port.o
    0x0802a830   0x0802a830   0x00000074   Code   RO         3948    i.Multiplex_Port_Choose  multiplex_port.o
    0x0802a8a4   0x0802a8a4   0x00000050   Code   RO         3949    i.Multiplex_Port_DMARX_IRQHandler  multiplex_port.o
    0x0802a8f4   0x0802a8f4   0x0000006c   Code   RO         3950    i.Multiplex_Port_DMATX_IRQHandler  multiplex_port.o
    0x0802a960   0x0802a960   0x000000c4   Code   RO         3951    i.Multiplex_Port_DMA_Configuration  multiplex_port.o
    0x0802aa24   0x0802aa24   0x00000084   Code   RO         3952    i.Multiplex_Port_IO_Configuration  multiplex_port.o
    0x0802aaa8   0x0802aaa8   0x000001ac   Code   RO         3953    i.Multiplex_Port_Init  multiplex_port.o
    0x0802ac54   0x0802ac54   0x0000003e   Code   RO         3954    i.Multiplex_Port_NVIC_Configuration  multiplex_port.o
    0x0802ac92   0x0802ac92   0x00000002   PAD
    0x0802ac94   0x0802ac94   0x0000008c   Code   RO         3956    i.Multiplex_Port_USART_Configuration  multiplex_port.o
    0x0802ad20   0x0802ad20   0x00000078   Code   RO          404    i.NVIC_Init         misc.o
    0x0802ad98   0x0802ad98   0x00000014   Code   RO          406    i.NVIC_SetVectorTable  misc.o
    0x0802adac   0x0802adac   0x00000028   Code   RO         3679    i.OLED_Clear        oled.o
    0x0802add4   0x0802add4   0x000000ac   Code   RO         3686    i.OLED_DrawLine     oled.o
    0x0802ae80   0x0802ae80   0x00000078   Code   RO         3687    i.OLED_DrawPoint    oled.o
    0x0802aef8   0x0802aef8   0x00000174   Code   RO         3688    i.OLED_Init         oled.o
    0x0802b06c   0x0802b06c   0x00000016   Code   RO         3689    i.OLED_Pow          oled.o
    0x0802b082   0x0802b082   0x000000a2   Code   RO         3690    i.OLED_ProgressBar  oled.o
    0x0802b124   0x0802b124   0x00000050   Code   RO         3691    i.OLED_Refresh      oled.o
    0x0802b174   0x0802b174   0x00000038   Code   RO         3692    i.OLED_SPI2_SendByte  oled.o
    0x0802b1ac   0x0802b1ac   0x0000013c   Code   RO         3693    i.OLED_ShowChar     oled.o
    0x0802b2e8   0x0802b2e8   0x00000144   Code   RO         3694    i.OLED_ShowNum      oled.o
    0x0802b42c   0x0802b42c   0x000000d6   Code   RO         3695    i.OLED_ShowPicture  oled.o
    0x0802b502   0x0802b502   0x00000050   Code   RO         3696    i.OLED_ShowString   oled.o
    0x0802b552   0x0802b552   0x00000002   PAD
    0x0802b554   0x0802b554   0x00000058   Code   RO         3697    i.OLED_WR_Byte      oled.o
    0x0802b5ac   0x0802b5ac   0x000000b0   Code   RO         2625    i.PCBEncryption_Check  fram.o
    0x0802b65c   0x0802b65c   0x00004b48   Code   RO         2954    i.POS_ConnectRXTask  pos_connect.o
    0x080301a4   0x080301a4   0x000021d8   Code   RO         2955    i.POS_ConnectTXTask  pos_connect.o
    0x0803237c   0x0803237c   0x00000078   Code   RO         2956    i.POS_Connect_DMARX_IRQHandler  pos_connect.o
    0x080323f4   0x080323f4   0x00000020   Code   RO         2957    i.POS_Connect_DMATX_IRQHandler  pos_connect.o
    0x08032414   0x08032414   0x000000c0   Code   RO         2958    i.POS_Connect_DMA_Configuration  pos_connect.o
    0x080324d4   0x080324d4   0x0000006c   Code   RO         2959    i.POS_Connect_IO_Configuration  pos_connect.o
    0x08032540   0x08032540   0x000002b4   Code   RO         2960    i.POS_Connect_Init  pos_connect.o
    0x080327f4   0x080327f4   0x0000003e   Code   RO         2961    i.POS_Connect_NVIC_Configuration  pos_connect.o
    0x08032832   0x08032832   0x00000002   PAD
    0x08032834   0x08032834   0x0000005c   Code   RO         2962    i.POS_Connect_USART_Configuration  pos_connect.o
    0x08032890   0x08032890   0x00000064   Code   RO         2706    i.Pluse_InPut_EXTI_Configuration  pluse_input.o
    0x080328f4   0x080328f4   0x000000ec   Code   RO         2707    i.Pluse_InPut_IO_Configuration  pluse_input.o
    0x080329e0   0x080329e0   0x0000007c   Code   RO         2708    i.Pluse_InPut_IRQHandler  pluse_input.o
    0x08032a5c   0x08032a5c   0x000000c0   Code   RO         2709    i.Pluse_InPut_Init  pluse_input.o
    0x08032b1c   0x08032b1c   0x0000003c   Code   RO         2710    i.Pluse_InPut_NVIC_Configuration  pluse_input.o
    0x08032b58   0x08032b58   0x00000098   Code   RO         3276    i.Pluse_Putout_IO_Configuration  pluse_putout.o
    0x08032bf0   0x08032bf0   0x00000008   Code   RO         3277    i.Pluse_Putout_Init  pluse_putout.o
    0x08032bf8   0x08032bf8   0x0000001a   Code   RO         3957    i.Price_DataCheck   multiplex_port.o
    0x08032c12   0x08032c12   0x00000002   PAD
    0x08032c14   0x08032c14   0x0000016c   Code   RO         3870    i.Print_Num         printf.o
    0x08032d80   0x08032d80   0x00000018   Code   RO         3398    i.Query376Interrupt  file_sys.o
    0x08032d98   0x08032d98   0x00000020   Code   RO         1194    i.RCC_AHB1PeriphClockCmd  stm32f4xx_rcc.o
    0x08032db8   0x08032db8   0x00000020   Code   RO         1196    i.RCC_AHB1PeriphResetCmd  stm32f4xx_rcc.o
    0x08032dd8   0x08032dd8   0x00000020   Code   RO         1197    i.RCC_AHB2PeriphClockCmd  stm32f4xx_rcc.o
    0x08032df8   0x08032df8   0x00000020   Code   RO         1203    i.RCC_APB1PeriphClockCmd  stm32f4xx_rcc.o
    0x08032e18   0x08032e18   0x00000020   Code   RO         1205    i.RCC_APB1PeriphResetCmd  stm32f4xx_rcc.o
    0x08032e38   0x08032e38   0x00000020   Code   RO         1206    i.RCC_APB2PeriphClockCmd  stm32f4xx_rcc.o
    0x08032e58   0x08032e58   0x00000020   Code   RO         1208    i.RCC_APB2PeriphResetCmd  stm32f4xx_rcc.o
    0x08032e78   0x08032e78   0x000000e8   Code   RO         1215    i.RCC_GetClocksFreq  stm32f4xx_rcc.o
    0x08032f60   0x08032f60   0x00000024   Code   RO         2420    i.RNG_Cmd           stm32f4xx_rng.o
    0x08032f84   0x08032f84   0x0000000c   Code   RO         2424    i.RNG_GetRandomNumber  stm32f4xx_rng.o
    0x08032f90   0x08032f90   0x0000003c   Code   RO         3183    i.ReadDFStatus      at45db.o
    0x08032fcc   0x08032fcc   0x00000090   Code   RO         3184    i.ReadDriverID      at45db.o
    0x0803305c   0x0803305c   0x000000e8   Code   RO         3399    i.SPI2_Init         file_sys.o
    0x08033144   0x08033144   0x00000038   Code   RO         3400    i.SPI2_ReadWriteByte  file_sys.o
    0x0803317c   0x0803317c   0x00000018   Code   RO         1476    i.SPI_Cmd           stm32f4xx_spi.o
    0x08033194   0x08033194   0x00000058   Code   RO         1483    i.SPI_I2S_DeInit    stm32f4xx_spi.o
    0x080331ec   0x080331ec   0x00000012   Code   RO         1484    i.SPI_I2S_GetFlagStatus  stm32f4xx_spi.o
    0x080331fe   0x080331fe   0x00000006   Code   RO         1487    i.SPI_I2S_ReceiveData  stm32f4xx_spi.o
    0x08033204   0x08033204   0x00000004   Code   RO         1488    i.SPI_I2S_SendData  stm32f4xx_spi.o
    0x08033208   0x08033208   0x0000003c   Code   RO         1489    i.SPI_Init          stm32f4xx_spi.o
    0x08033244   0x08033244   0x0000001c   Code   RO         2966    i.SUMCRC            pos_connect.o
    0x08033260   0x08033260   0x00000040   Code   RO         1633    i.SYSCFG_EXTILineConfig  stm32f4xx_syscfg.o
    0x080332a0   0x080332a0   0x000000d8   Code   RO         2580    i.SYSTimer_IRQHandler  time_count.o
    0x08033378   0x08033378   0x000000e8   Code   RO          361    i.SetSysClock       system_stm32f4xx.o
    0x08033460   0x08033460   0x0000000c   Code   RO         3402    i.Spi376OutByte     file_sys.o
    0x0803346c   0x0803346c   0x00000084   Code   RO         2772    i.StrToFloat        md_connect.o
    0x080334f0   0x080334f0   0x0000004c   Code   RO         2773    i.StrToInt          md_connect.o
    0x0803353c   0x0803353c   0x0000019c   Code   RO         3812    i.Sureface_Wait_TimeUpData  surface.o
    0x080336d8   0x080336d8   0x00000010   Code   RO         3813    i.SurfaceJump       surface.o
    0x080336e8   0x080336e8   0x000026f4   Code   RO         3814    i.SurfaceTast       surface.o
    0x08035ddc   0x08035ddc   0x00000044   Code   RO         3815    i.Surface_Copy_16   surface.o
    0x08035e20   0x08035e20   0x0000002c   Code   RO         3816    i.Surface_Init      surface.o
    0x08035e4c   0x08035e4c   0x00000028   Code   RO          408    i.SysTick_CLKSourceConfig  misc.o
    0x08035e74   0x08035e74   0x00000068   Code   RO          363    i.SystemInit        system_stm32f4xx.o
    0x08035edc   0x08035edc   0x00000008   Code   RO           12    i.TIM2_IRQHandler   stm32f4xx_it.o
    0x08035ee4   0x08035ee4   0x00000006   Code   RO         1686    i.TIM_ClearFlag     stm32f4xx_tim.o
    0x08035eea   0x08035eea   0x00000018   Code   RO         1692    i.TIM_Cmd           stm32f4xx_tim.o
    0x08035f02   0x08035f02   0x00000002   PAD
    0x08035f04   0x08035f04   0x00000190   Code   RO         1697    i.TIM_DeInit        stm32f4xx_tim.o
    0x08036094   0x08036094   0x00000022   Code   RO         1713    i.TIM_GetITStatus   stm32f4xx_tim.o
    0x080360b6   0x080360b6   0x00000012   Code   RO         1717    i.TIM_ITConfig      stm32f4xx_tim.o
    0x080360c8   0x080360c8   0x00000084   Code   RO         1764    i.TIM_TimeBaseInit  stm32f4xx_tim.o
    0x0803614c   0x0803614c   0x000000c0   Code   RO          323    i.TXH_Init          txh.o
    0x0803620c   0x0803620c   0x000008c4   Code   RO          324    i.TXH_Task          txh.o
    0x08036ad0   0x08036ad0   0x00000330   Code   RO         2581    i.Timer_Init        time_count.o
    0x08036e00   0x08036e00   0x00000022   Code   RO         2582    i.Timer_NVIC_Configuration  time_count.o
    0x08036e22   0x08036e22   0x00000008   Code   RO           13    i.UART4_IRQHandler  stm32f4xx_it.o
    0x08036e2a   0x08036e2a   0x00000008   Code   RO           14    i.UART5_IRQHandler  stm32f4xx_it.o
    0x08036e32   0x08036e32   0x00000008   Code   RO           15    i.USART1_IRQHandler  stm32f4xx_it.o
    0x08036e3a   0x08036e3a   0x00000008   Code   RO           16    i.USART2_IRQHandler  stm32f4xx_it.o
    0x08036e42   0x08036e42   0x00000008   Code   RO           17    i.USART3_IRQHandler  stm32f4xx_it.o
    0x08036e4a   0x08036e4a   0x00000008   Code   RO           18    i.USART6_IRQHandler  stm32f4xx_it.o
    0x08036e52   0x08036e52   0x00000012   Code   RO         2234    i.USART_ClearFlag   stm32f4xx_usart.o
    0x08036e64   0x08036e64   0x00000018   Code   RO         2238    i.USART_Cmd         stm32f4xx_usart.o
    0x08036e7c   0x08036e7c   0x00000012   Code   RO         2239    i.USART_DMACmd      stm32f4xx_usart.o
    0x08036e8e   0x08036e8e   0x00000002   PAD
    0x08036e90   0x08036e90   0x000000b4   Code   RO         2240    i.USART_DeInit      stm32f4xx_usart.o
    0x08036f44   0x08036f44   0x0000001a   Code   RO         2241    i.USART_GetFlagStatus  stm32f4xx_usart.o
    0x08036f5e   0x08036f5e   0x00000054   Code   RO         2242    i.USART_GetITStatus  stm32f4xx_usart.o
    0x08036fb2   0x08036fb2   0x0000004a   Code   RO         2244    i.USART_ITConfig    stm32f4xx_usart.o
    0x08036ffc   0x08036ffc   0x000000d4   Code   RO         2245    i.USART_Init        stm32f4xx_usart.o
    0x080370d0   0x080370d0   0x00000024   Code   RO         3403    i.Wait376Interrupt  file_sys.o
    0x080370f4   0x080370f4   0x00000028   Code   RO         4360    i.__0sprintf$8      mc_w.l(printf8.o)
    0x0803711c   0x0803711c   0x00000030   Code   RO         4459    i.__ARM_fpclassify  m_wm.l(fpclassify.o)
    0x0803714c   0x0803714c   0x00000004   PAD
    0x08037150   0x08037150   0x00000038   Code   RO         4078    i.__hardfp_atof     m_wm.l(atof.o)
    0x08037188   0x08037188   0x000003c4   Code   RO         4461    i.__hardfp_log      m_wm.l(log.o)
    0x0803754c   0x0803754c   0x00000004   PAD
    0x08037550   0x08037550   0x00000130   Code   RO         4096    i.__hardfp_log10    m_wm.l(log10.o)
    0x08037680   0x08037680   0x00000c50   Code   RO         4108    i.__hardfp_pow      m_wm.l(pow.o)
    0x080382d0   0x080382d0   0x000000f8   Code   RO         4475    i.__kernel_poly     m_wm.l(poly.o)
    0x080383c8   0x080383c8   0x00000030   Code   RO         4439    i.__mathlib_dbl_divzero  m_wm.l(dunder.o)
    0x080383f8   0x080383f8   0x00000014   Code   RO         4440    i.__mathlib_dbl_infnan  m_wm.l(dunder.o)
    0x0803840c   0x0803840c   0x00000014   Code   RO         4441    i.__mathlib_dbl_infnan2  m_wm.l(dunder.o)
    0x08038420   0x08038420   0x00000020   Code   RO         4442    i.__mathlib_dbl_invalid  m_wm.l(dunder.o)
    0x08038440   0x08038440   0x00000020   Code   RO         4443    i.__mathlib_dbl_overflow  m_wm.l(dunder.o)
    0x08038460   0x08038460   0x00000020   Code   RO         4445    i.__mathlib_dbl_underflow  m_wm.l(dunder.o)
    0x08038480   0x08038480   0x0000000c   Code   RO         4529    i.__read_errno      mc_w.l(errno.o)
    0x0803848c   0x0803848c   0x0000000e   Code   RO         4573    i.__scatterload_copy  mc_w.l(handlers.o)
    0x0803849a   0x0803849a   0x00000002   Code   RO         4574    i.__scatterload_null  mc_w.l(handlers.o)
    0x0803849c   0x0803849c   0x0000000e   Code   RO         4575    i.__scatterload_zeroinit  mc_w.l(handlers.o)
    0x080384aa   0x080384aa   0x00000006   Code   RO         2626    i.__set_PRIMASK     fram.o
    0x080384b0   0x080384b0   0x00000006   Code   RO         3185    i.__set_PRIMASK     at45db.o
    0x080384b6   0x080384b6   0x00000002   PAD
    0x080384b8   0x080384b8   0x0000000c   Code   RO         4530    i.__set_errno       mc_w.l(errno.o)
    0x080384c4   0x080384c4   0x0000000e   Code   RO         4557    i._is_digit         mc_w.l(scanf_fp.o)
    0x080384d2   0x080384d2   0x00000002   PAD
    0x080384d4   0x080384d4   0x00000404   Code   RO         4365    i._printf_core      mc_w.l(printf8.o)
    0x080388d8   0x080388d8   0x00000024   Code   RO         4366    i._printf_post_padding  mc_w.l(printf8.o)
    0x080388fc   0x080388fc   0x0000002e   Code   RO         4367    i._printf_pre_padding  mc_w.l(printf8.o)
    0x0803892a   0x0803892a   0x0000000a   Code   RO         4369    i._sputc            mc_w.l(printf8.o)
    0x08038934   0x08038934   0x0000000c   Code   RO         4051    i.delay_init        delay.o
    0x08038940   0x08038940   0x00000044   Code   RO         4052    i.delay_ms          delay.o
    0x08038984   0x08038984   0x00000042   Code   RO         4053    i.delay_us          delay.o
    0x080389c6   0x080389c6   0x00000002   PAD
    0x080389c8   0x080389c8   0x00000028   Code   RO         2775    i.do_crc            md_connect.o
    0x080389f0   0x080389f0   0x00000018   Code   RO         4455    i.fabs              m_wm.l(fabs.o)
    0x08038a08   0x08038a08   0x00000040   Code   RO         3104    i.iic_ack           ds1307.o
    0x08038a48   0x08038a48   0x00000040   Code   RO         3105    i.iic_noack         ds1307.o
    0x08038a88   0x08038a88   0x00000060   Code   RO         3106    i.iic_readbyte      ds1307.o
    0x08038ae8   0x08038ae8   0x00000068   Code   RO         3107    i.iic_sendbyte      ds1307.o
    0x08038b50   0x08038b50   0x00000034   Code   RO         3108    i.iic_start         ds1307.o
    0x08038b84   0x08038b84   0x00000034   Code   RO         3109    i.iic_stop          ds1307.o
    0x08038bb8   0x08038bb8   0x0000005c   Code   RO         3110    i.iic_wait4ack      ds1307.o
    0x08038c14   0x08038c14   0x00000010   Code   RO         4463    i.log               m_wm.l(log.o)
    0x08038c24   0x08038c24   0x0000006c   Code   RO         3404    i.mInitCH376Host    file_sys.o
    0x08038c90   0x08038c90   0x0000006c   Code   RO          300    i.main              main.o
    0x08038cfc   0x08038cfc   0x00000044   Code   RO         3959    i.mystrstr          multiplex_port.o
    0x08038d40   0x08038d40   0x0000006e   Code   RO         4491    i.sqrt              m_wm.l(sqrt.o)
    0x08038dae   0x08038dae   0x00000014   Code   RO         3405    i.xReadCH376Data    file_sys.o
    0x08038dc2   0x08038dc2   0x00000002   PAD
    0x08038dc4   0x08038dc4   0x00000040   Code   RO         3406    i.xWriteCH376Cmd    file_sys.o
    0x08038e04   0x08038e04   0x00000012   Code   RO         3407    i.xWriteCH376Data   file_sys.o
    0x08038e16   0x08038e16   0x0000000b   Data   RO          326    .constdata          txh.o
    0x08038e21   0x08038e21   0x00000003   PAD
    0x08038e24   0x08038e24   0x00000bec   Data   RO         2628    .constdata          fram.o
    0x08039a10   0x08039a10   0x0000006a   Data   RO         2777    .constdata          md_connect.o
    0x08039a7a   0x08039a7a   0x00000002   PAD
    0x08039a7c   0x08039a7c   0x00004fa2   Data   RO         2968    .constdata          pos_connect.o
    0x0803ea1e   0x0803ea1e   0x00000002   PAD
    0x0803ea20   0x0803ea20   0x00000244   Data   RO         3187    .constdata          at45db.o
    0x0803ec64   0x0803ec64   0x00001e10   Data   RO         3699    .constdata          oled.o
    0x08040a74   0x08040a74   0x0000079c   Data   RO         3817    .constdata          surface.o
    0x08041210   0x08041210   0x00000088   Data   RO         4111    .constdata          m_wm.l(pow.o)
    0x08041298   0x08041298   0x00000038   Data   RO         4464    .constdata          m_wm.l(log.o)
    0x080412d0   0x080412d0   0x00000008   Data   RO         4477    .constdata          m_wm.l(qnan.o)
    0x080412d8   0x080412d8   0x00000040   Data   RO         4567    .constdata          mc_w.l(ctype_c.o)
    0x08041318   0x08041318   0x00000020   Data   RO         4571    Region$$Table       anon$$obj.o


    Execution Region RW_IRAM1 (Exec base: 0x20000000, Load base: 0x08041338, Size: 0x0000f568, Max: 0x00030000, ABSOLUTE, COMPRESSED[0x00000280])

    Exec Addr    Load Addr    Size         Type   Attr      Idx    E Section Name        Object

    0x20000000   COMPRESSED   0x00000010   Data   RW         1238    .data               stm32f4xx_rcc.o
    0x20000010   COMPRESSED   0x00000002   Data   RW         2629    .data               fram.o
    0x20000012   COMPRESSED   0x0000020c   Data   RW         2778    .data               md_connect.o
    0x2000021e   COMPRESSED   0x00000002   PAD
    0x20000220   COMPRESSED   0x0000080b   Data   RW         2969    .data               pos_connect.o
    0x20000a2b   COMPRESSED   0x00000001   PAD
    0x20000a2c   COMPRESSED   0x00000006   Data   RW         3188    .data               at45db.o
    0x20000a32   COMPRESSED   0x00000006   PAD
    0x20000a38   COMPRESSED   0x000000a5   Data   RW         3651    .data               log.o
    0x20000add   COMPRESSED   0x00000005   Data   RW         3818    .data               surface.o
    0x20000ae2   COMPRESSED   0x000007d3   Data   RW         3960    .data               multiplex_port.o
    0x200012b5   COMPRESSED   0x00000003   PAD
    0x200012b8   COMPRESSED   0x00000004   Data   RW         4531    .data               mc_w.l(errno.o)
    0x200012bc        -       0x00006e64   Zero   RW          325    .bss                txh.o
    0x20008120        -       0x000004b8   Zero   RW         2627    .bss                fram.o
    0x200085d8        -       0x00001958   Zero   RW         2776    .bss                md_connect.o
    0x20009f30        -       0x00000fa0   Zero   RW         2967    .bss                pos_connect.o
    0x2000aed0        -       0x00000213   Zero   RW         3186    .bss                at45db.o
    0x2000b0e3        -       0x00000480   Zero   RW         3698    .bss                oled.o
    0x2000b563   COMPRESSED   0x00000005   PAD
    0x2000b568        -       0x00004000   Zero   RW          396    STACK               startup_stm32f4xx.o


==============================================================================

Image component sizes


      Code (inc. data)   RO Data    RW Data    ZI Data      Debug   Object Name

      1578         90        580          6        531       9054   at45db.o
       146          0          0          0          0       1511   delay.o
       936         72          0          0          0       5693   ds1307.o
      1506        108          0          0          0      16640   file_sys.o
      2034        102       3052          2       1208       9341   fram.o
      1224        106          0        165          0       3293   log.o
       108         18          0          0          0       2003   main.o
    125938       2750        106        524       6488      56720   md_connect.o
       180         22          0          0          0       2312   misc.o
      5404        258          0       2003          0      11799   multiplex_port.o
      2046         70       7696          0       1152      11227   oled.o
       712         60          0          0          0       3089   pluse_input.o
       160         22          0          0          0       1152   pluse_putout.o
     29470       1254      20386       2059       4000      25158   pos_connect.o
       364          6          0          0          0       1136   printf.o
        36          8        392          0      16384        820   startup_stm32f4xx.o
       564         40          0          0          0       4677   stm32f4xx_dma.o
       200         18          0          0          0       2344   stm32f4xx_exti.o
       496         36          0          0          0       4561   stm32f4xx_gpio.o
       196         10          0          0          0     338654   stm32f4xx_it.o
        16          6          0          0          0        541   stm32f4xx_iwdg.o
       456         60          0         16          0       7159   stm32f4xx_rcc.o
        48         12          0          0          0       1124   stm32f4xx_rng.o
       200         12          0          0          0       4439   stm32f4xx_spi.o
        64          4          0          0          0        696   stm32f4xx_syscfg.o
       614         82          0          0          0       4775   stm32f4xx_tim.o
       636         32          0          0          0       6628   stm32f4xx_usart.o
     10740       1134       1948          5          0      10205   surface.o
       336         32          0          0          0       1477   system_stm32f4xx.o
      1066         36          0          0          0       1974   time_count.o
      2436         74         11          0      28260      14004   txh.o

    ----------------------------------------------------------------------
    189944       6534      34210       4792      58028     564206   Object Totals
         0          0         32          0          0          0   (incl. Generated)
        34          0          7         12          5          0   (incl. Padding)

    ----------------------------------------------------------------------

      Code (inc. data)   RO Data    RW Data    ZI Data      Debug   Library Member Name

        56         12          0          0          0        132   atof.o
       184         44          0          0          0        744   dunder.o
        24          0          0          0          0        124   fabs.o
        48          0          0          0          0        124   fpclassify.o
       980         92         56          0          0        440   log.o
       304         44          0          0          0        200   log10.o
       248          0          0          0          0        152   poly.o
      3152        296        136          0          0        352   pow.o
         0          0          8          0          0          0   qnan.o
       110          0          0          0          0        148   sqrt.o
        86          0          0          0          0          0   __dczerorl2.o
        64          0          0          0          0         84   _sgetc.o
        40          6         64          0          0         68   ctype_c.o
         0          0          0          0          0          0   entry.o
         0          0          0          0          0          0   entry10a.o
         0          0          0          0          0          0   entry11a.o
         4          0          0          0          0          0   entry12b.o
         8          4          0          0          0          0   entry2.o
         4          0          0          0          0          0   entry5.o
         0          0          0          0          0          0   entry7b.o
         0          0          0          0          0          0   entry8b.o
         8          4          0          0          0          0   entry9a.o
        24         12          0          4          0        136   errno.o
        30          0          0          0          0          0   handlers.o
        36          8          0          0          0         68   init.o
        10          0          0          0          0         68   isspace_c.o
         0          0          0          0          0          0   iusefp.o
        98          0          0          0          0         84   ldiv.o
        30          0          0          0          0         68   llshl.o
        36          0          0          0          0         68   llsshr.o
        32          0          0          0          0         68   llushr.o
        36          0          0          0          0         68   memcpya.o
      1160         50          0          0          0        420   printf8.o
       878         12          0          0          0        216   scanf_fp.o
        24          0          0          0          0         68   strcat.o
        14          0          0          0          0         68   strlen.o
        30          0          0          0          0         80   strncmp.o
       156         12          0          0          0        120   strtod.o
        98          0          0          0          0         92   uldiv.o
        48          0          0          0          0         68   cdcmple.o
        48          0          0          0          0         68   cdrcmple.o
        56          0          0          0          0         88   d2f.o
       334          0          0          0          0        148   dadd.o
       222          0          0          0          0        100   ddiv.o
       186          0          0          0          0        176   depilogue.o
        62          0          0          0          0         80   dfixi.o
        74          0          0          0          0         80   dfixl.o
        34          0          0          0          0         76   dflti.o
        40          0          0          0          0         80   dfltl.o
        26          0          0          0          0         76   dfltui.o
        24          0          0          0          0         76   dfltul.o
       228          0          0          0          0         96   dmul.o
        46          0          0          0          0         80   dscalb.o
       162          0          0          0          0        100   dsqrt.o
        38          0          0          0          0         68   f2d.o
       110          0          0          0          0        168   fepilogue.o
        66          0          0          0          0         76   ffixl.o
        44          0          0          0          0         92   ffltl.o

    ----------------------------------------------------------------------
      9878        600        264          4          0       6056   Library Totals
        18          4          0          0          0          0   (incl. Padding)

    ----------------------------------------------------------------------

      Code (inc. data)   RO Data    RW Data    ZI Data      Debug   Library Name

      5106        488        200          0          0       2416   m_wm.l
      2906        108         64          4          0       1844   mc_w.l
      1848          0          0          0          0       1796   mf_w.l

    ----------------------------------------------------------------------
      9878        600        264          4          0       6056   Library Totals

    ----------------------------------------------------------------------

==============================================================================


      Code (inc. data)   RO Data    RW Data    ZI Data      Debug   

    199822       7134      34474       4796      58028     545270   Grand Totals
    199822       7134      34474        640      58028     545270   ELF Image Totals (compressed)
    199822       7134      34474        640          0          0   ROM Totals

==============================================================================

    Total RO  Size (Code + RO Data)               234296 ( 228.80kB)
    Total RW  Size (RW Data + ZI Data)             62824 (  61.35kB)
    Total ROM Size (Code + RO Data + RW Data)     234936 ( 229.43kB)

==============================================================================

